:100000000C94AD0E0C94D50E0C94D50E0C94D50E0C
:100010000C94D50E0C94D50E0C94D50E0C94D50ED4
:100020000C94D50E0C94D50E0C94D8130C94376107
:100030000C94F7630C9464610C94D50E0C943714F3
:100040000C94C6130C94D50E0C94D50E0C94D50EAE
:100050000C94D50E0C94D50E0C94D50E0C94D50E94
:100060000C946F640C947C140C94C9610C94B0646F
:100070000C94D50E0C94D50E0C94D50E0C94D50E74
:100080000C94D50E0C94D50E0C94D50E08160C16A7
:10009000CD15D315D915D915D9150016041608167E
:1000A0000C16101614161816CB398B399639A5393B
:1000B000AB39AF39B439773E8D3E9B3EB03EBE3E44
:1000C000CD3EDF3E053F2E3F3C3F623F803F8E3FAF
:1000D0009C3FAA3F015DF05CEA5CF25CF65CFA5C76
:1000E000ED5CFE5C045DDD65DF65E265E765FA6594
:1000F0000B661B66266638664A664F6668666B66E0
:100100006F667166736678667C6688668C669466D0
:100110009B669F66A166A566A766A966AB66AF6685
:10012000B366B866BD66C266C766CC66204F6C64AF
:100130002056657273696F6E20454550524F4D20B1
:100140002020434845434B2053455454494E475380
:100150002F43414C494200416C61726D73204469E8
:100160007361626C656400506C65617365205265F3
:10017000736574205377697463686573005468729B
:100180006F74746C65206E6F742069646C650052C6
:1001900065736574207468726F74746C650045458E
:1001A00050524F4D206C6F77206D656D004C4F4164
:1001B00044494E47006D537461636B206F666C6FEA
:1001C00077006D537461636B2075666C6F77004DBB
:1001D00045535341474500707265737320616E79D2
:1001E000204B657900507265737320616E79206BC6
:1001F000657920746F20736B697000032D2D2D7845
:100200003E30783C307C787C663E30663C307C66A4
:100210007C633120633220633320633420633520D4
:1002200063362063372063382063392063313063BD
:1002300031316331326331336331346331356331AA
:100240003600034F46464142535255735255254599
:100250004C73454C25544873544825414C73414CCC
:100260002550312050312550322050322550332036
:10027000503325002D2D2D004348002D2D2D20001D
:100280000450312020503220205033202048414C4F
:100290004646554C4C4359433143594332435943E5
:1002A0003350504D3150504D3250504D3350504DD1
:1002B0003450504D3550504D3650504D3750504DB4
:1002C00038434831204348322043483320434834A0
:1002D0002043483520434836204348372043483898
:1002E0002043483920434831304348313143483175
:1002F0003243483133434831344348313543483140
:100300003633504F534756312047563220475633E5
:100310002047563420475635204756362047563713
:1003200020002D2D2D2D000000642810070301044E
:1003300052554420454C45205448522041494C20B8
:1003400000414C4552540000010203000201030326
:10035000010200030201004F4E20004F46460003F9
:10036000544852525544454C45494430494431491A
:10037000443241494C47454154524E5357315357EB
:1003800032535733535734535735535736535737E0
:1003900053573853573953574153574253574300D4
:1003A0001B1E272D36394B4E636C7278878D939CBC
:1003B000B1B4C6C9D2D8E1E453706C6173680080EF
:1003C00040000000000000000000000000000000ED
:1003D000000000000000000000000000000000001D
:1003E000000000000000000000000000000000000D
:1003F00000000000000000000000000000000000FD
:1004000000000000000000000000000080C0E0E0EC
:10041000F0F8F8FCFCFCF8F8F8F0400000000000F0
:10042000808080000000000000000000000000004C
:1004300000000000000080C0C0E0E0E0F0F0F0E06C
:10044000C00000000000C0F8FFFF9F878383838304
:10045000838383838383838383838383838383836C
:1004600083830383808383838383838383838383DF
:10047000838383838383838383838383C3E3733F00
:100480001F0000000080E0F0F8FCFEFFFFFFFF7F90
:100490003F1F1F0F0783C3E1E1E0E0C0000E1F3FD5
:1004A0007F7FFFF3E0E0800000000000000000001C
:1004B0000080F0FCFEFFFFFFFF7F3F0F0301010103
:1004C00000000080F0FEFFFFC7C1C1C1C1C1C1C1B2
:1004D000C1C1C1C1C1C1C1C1C1C1C1C1C1C1C101CC
:1004E000C1F0FEFF3F0F070F0D0D0D1D1919191952
:1004F0003131313171616161E1C1C1C181000000FF
:1005000080E0F8FCFFFFFFFF2F170F038180C0E0A2
:10051000F0F8FCFEFFFFFFFFFFFF7F01000000007F
:1005200000000001010307070E1E1C3870E0F0F800
:10053000FEFFFF7F1F0F030001000000000000000E
:1005400000000000000000000000000000000000AB
:10055000000000000000000000000000000000009B
:10056000000000000000000000000000000000008B
:100570000000000000000000000000000000007EFD
:10058000FFFFFFFFFFFFFBF8FCFCFEFF7F3F1F0F9D
:1005900007C3FFFFFFFFFFFF7F0700000000000011
:1005A0000000000000000000C0E0F8FEFFFF7F1F19
:1005B0000F1F3D7CF8F8F0E0800000000000000014
:1005C000000000000000000000000000000000002B
:1005D000000000000000000000000000000000001B
:1005E000000000000000000000000000000000000B
:1005F00000000000000000000000000000000000FB
:10060000000101010101030707070301000000E0E9
:10061000FCFFFFFFFFFF1F030000000000000000C1
:10062000000000C0F078DE2713090E070300000069
:10063000000000000001030F7FFFFC7878F8000045
:10064000000000000000000000808080808080802A
:10065000808000808000808000000000000000801A
:10066000808080808080808080808080808080808A
:1006700080000000000000000000000000000000FA
:1006800000000000000000000000000080F0FEFFFD
:10069000FFFFFF3F0F010000000000000000C0E06E
:1006A000381E0F03000100000000000000000000E1
:1006B0000000000000000000000000000303010033
:1006C0000000000000000000000E0E020202020204
:1006D0000303000F0F000F0F080808080808080F91
:1006E0000F08080808080F0F000000000F0F000097
:1006F00000000000000000000000000000000000FA
:1007000000000000000000000000C0F8BFFFFFFF75
:100710001F7F010000000000000000F0FCFF7F7858
:100720003000000000000000000000000000000099
:1007300000000000000000000000000000000000B9
:1007400000000000000000000000000000000000A9
:100750000000000000000000000000000000000099
:100760000000000000000000000000000000000089
:100770000000000000000000000000000000000079
:100780000000000000000000301C070E0F070100F1
:100790000000000000000000000000000000000059
:1007A0000000000000000000000000000000000049
:1007B0000000000000000000000000000000000039
:1007C0000000204D4F443A202020202020002053BC
:1007D000564E3A20657239782D72383038005449B7
:1007E0004D453A2031313A34343A34390044415499
:1007F000453A2031322E31312E32303133005645D8
:1008000052533A2056312E323139312D4D696B65B4
:100810000022047C5E54546D000345787045784690
:10082000466E654D65644372730011544F54000168
:1008300053544B115354250001544D4511545357F3
:10084000005354415400035B4D454E555D20746F79
:10085000207265667265736800746D61696E0F6DF4
:100860007300746D7231204A69747465720F757308
:1008700000746D72314C6174206D696E0F75730078
:10088000746D72314C6174206D61780F7573005313
:1008900054415432004D6F6465002052455441006C
:1008A000014368616E6E656C204F7264657200432F
:1008B000726F73735472696D00456E61626C65206E
:1008C00050504D53494D0042616E64476170005372
:1008D0007469636B5363726F6C6C00506F74536315
:1008E000726F6C6C00416C61726D205761726E6941
:1008F0006E67004D656D6F7279205761726E696E1B
:10090000670044656661756C7420537700546872A3
:100910006F74746C65205761726E696E67005370F6
:100920006C617368204E616D650053706C61736813
:100930002073637265656E004C69676874206F6E22
:100940002053746B204D76004C69676874206F6685
:1009500066206166746572004261636B6C696768EA
:100960007420696E76657274004C696768742073D0
:10097000776974636800466C617368206F6E2062EB
:10098000656570004265657020636F756E74646F95
:10099000776E004D696E75746520626565700054F0
:1009A00068726F74746C6520726576657273650029
:1009B000496E616374697669747920616C61726DE6
:1009C000136D0042617474657279207761726E698B
:1009D0006E6700436F6E74726173740020486170BB
:1009E00074696320537472656E6774680020537075
:1009F00065616B657220506974636800566F6C7531
:100A00006D65000A4265657065722020202050697E
:100A100053706B72202020204265657072566F699A
:100A20006365506953706B566F6963654D656761A7
:100A3000536F756E642000536F756E64204D6F6444
:100A40006500065175696574204E6F4B6579207895
:100A500053686F727453686F7274204E6F726D209A
:100A6000204C6F6E672020784C6F6E6720004265C7
:100A700065706572004F776E6572204E616D65001E
:100A8000000900524144494F20534554555000033A
:100A90006D6F64650A2520737263202073770043AD
:100AA000616C004D756C7469706C696572000363EC
:100AB000683163683263683363683400036F666665
:100AC000202B3D203A3D0007536C61766500000302
:100AD00003030300545241494E45520056455253B8
:100AE000494F4E005472696D2D202B0005204D6535
:100AF0006E75204578697420446F776E20202055EC
:100B0000705269676874204C6566740044494147B7
:100B10000012424700414E4100034D4F56452053BD
:100B20005449434B532F504F5453000553455420C1
:100B30004D4944504F494E5400035B4D454E555D61
:100B400020544F2053544152540043414C49425287
:100B50004154494F4E000966726565004D4F44454A
:100B60004C53454C00434F4C204469726563746993
:100B70006F6E0041494C20446972656374696F6E01
:100B800000454C4520446972656374696F6E00537B
:100B9000776173682052696E6700436F6C6C6563A0
:100BA0007469766500062D2D2D20202031323020ED
:100BB000202031323058202031343020202039306C
:100BC00020202020005377617368205479706500DD
:100BD0000048454C492053455455500020464D008F
:100BE00001524554410020464D30004D4F4445537D
:100BF000005472696D730053776974636800000371
:100C0000464C204D4F444500015245544100032DB0
:100C10002D2D503120503220503320475634475626
:100C20003547563647563700566F6C756D6520430D
:100C30006F6E74726F6C004175746F204C696D69D2
:100C40007473005432546854726967005472616955
:100C50006E657200452E204C696D697473000350F7
:100C60004F534E45470053686966742053656C00C6
:100C700050504D20317374204368616E0003416D04
:100C8000654A61704575720020436F756E747279A4
:100C900000034431364438204C52500020547970BF
:100CA0006500094C50342F4C5035202044534D32B0
:100CB0006F6E6C792044534D322F44534D5800448D
:100CC000534D20547970650042696E642020526152
:100CD0006E67650050504D2046724C656E0D6D5329
:100CE0006563000B52784E756D000434434820361E
:100CF000434820384348203130434831324348315B
:100D00003443483136434800137553001175536519
:100D100063000650504D2020205058582020204479
:100D2000534D32202050504D31362050504D5349B4
:100D30004D0050726F746F00524554413132330090
:100D40004265657020436E74005472696D2053775C
:100D50000006457870202020457846696E65466912
:100D60006E6520204D656469756D436F61727365B2
:100D7000005472696D20496E6300542D4578706F80
:100D800000542D5472696D000A436F756E742044CF
:100D90006F776E436F756E7420557020200054720B
:100DA00069676765724200547269676765720056C9
:100DB0006F69636520496E646578114D454E550035
:100DC0004E616D6500000900010000000000000098
:100DD0000602010053455455500052414E474520EC
:100DE000434845434B20525353493A000642494E2B
:100DF00044494E47004475706C69636174696E675D
:100E0000206D6F64656C0044454C455445204D4F42
:100E100044454C004455504C4943415445204D4FA6
:100E200044454C004472537732004472537731008A
:100E30000257656967687400024578706F00044462
:100E40005220486900044452204C6F7700044452F9
:100E5000204D696400004558504F2F445200012B2B
:100E60002A52004D495845520003202020202020BE
:100E700020200044454C455445204D49583F00032F
:100E80005B4D454E555D0B5B455849545D0003591C
:100E900045530B4E4F005072657373205B455849A4
:100EA000545D20746F2061626F7274004D61782010
:100EB0006D69786572732072656163683A203332B8
:100EC0000002536C6F77202055700002536C6F77CF
:100ED0002020446F776E000244656C617920557064
:100EE000000244656C617920446F776E00084164AC
:100EF0006420202020204D756C7469706C795265D7
:100F0000706C6163652000024D756C74707800022E
:100F10005761726E696E6700025377697463680087
:100F20004375727665000D44696666000254726905
:100F30006D0002466C4D6F64657472696D00024607
:100F40006978204F6666736574004F6666736574D2
:100F500000466D5472696D56616C00025765696791
:100F600068740002536F75726365004544495420EC
:100F70004D49582000032D2D2D783E30783C307C93
:100F8000787C663E30663C307C667C633120633220
:100F90002063332063342063352063362063372099
:100FA0006338206339206331306331316331326318
:100FB0003133633134633135633136000D4F6E00A8
:100FC000072D2D2D2D202020763E6F667320207654
:100FD0003C6F667320207C767C3E6F66737C767CEB
:100FE0003C6F6673414E44202020204F5220202029
:100FF0002020584F522020202076313D3D7632204F
:101000007631213D76322076313E7632202076319F
:101010003C7632202076313E3D76322076313C3DA2
:1010200076322054696D654F6666005300000343B5
:101030005553544F4D205357495443484553000688
:101040004F4E202020204F4646202020424F54481B
:101050002020313553656373333053656373363005
:101060005365637356617269626C005653000720C2
:1010700038205365637331322053656373313620F2
:1010800053656373004E756D62657220566F6963B8
:1010900065205377000000025341464554592053C0
:1010A0005749544348455300434C454152204D490C
:1010B000584553205B4D454E555D0054454D504CB1
:1010C0004154455300032D2D2D52746D45746D54BC
:1010D000746D41746D52454E525544454C455448CB
:1010E0005241494C5031205032205033206331203E
:1010F00063322063332063342063352063362063FA
:1011000037206338206339206331306331316331F4
:1011100032633133633134633135633136004756DE
:10112000000001474C4F42414C205641525300436E
:101130004F5059205452494D205B4D454E555D004E
:1011400000034C494D4954530043560043555256F1
:10115000455300505245534554000043555256459F
:1011600000032D2D2D494E56004756005B4D454E30
:10117000555D205748454E20444F4E450053454C41
:1011800045435400434F5059004D4F564500444588
:101190004C455445004544495400494E534552542A
:1011A00000434F5059004D4F56450044454C45545F
:1011B0004500B1490D234E229B2ED021B524C144B8
:1011C000EE25BB2BF4281941244EC63F3943D14F9D
:1011D00089407C2212081200081C0808081C08001C
:1011E00000082200490022080000000000227F229F
:1011F00000000008220049002208000008220049DF
:10120000002208000000227F2200000000000822C7
:1012100000490022080000081C0808081C080006F5
:101220005761726E31205761726E3220436865617A
:10123000702052696E672020536369466920526F9F
:10124000626F742043686972702054616461202069
:10125000437269636B74536972656E20416C6D43B0
:101260006C6B5261746174615469636B20204861D6
:1012700070746331486170746332486170746333B1
:101280000054696D65720054524530313241470057
:10129000204142434445464748494A4B4C4D4E4FF6
:1012A000505152535455565758595A6162636465A8
:1012B000666768696A6B6C6D6E6F70717273747556
:1012C000767778797A303132333435363738395F5A
:1012D0002D2E00FEFFFDF6F7F8F9FAFBFC042D2D8C
:1012E0002D2D54494D3154494D3242415454477685
:1012F0007231477672324776723347767234477668
:101300007235477672364776723700537769746361
:1013100068205761726E696E670067656E777269E3
:101320007465206572726F7200454550524F4D20B2
:10133000466F726D617474696E6700426164204526
:101340004570726F6D204461746100434845434BA2
:10135000204D495820534F5552434553004D4F445B
:10136000454C2020202020004D45202020202020FA
:10137000202000454550524F4D206F766572666CB7
:101380006F7700E2AEA1A6A4A2C02F258122AF00F4
:10139000000000000000000000000000000000004D
:1013A000000000000000000000000000000000330A
:1013B0003B1F0F00000000C0C0C0C0C0C0C0C0C004
:1013C000C00000000000000000000000000000005D
:1013D00000000000000000183C3C18000000000065
:1013E000000080C0E070381C0C0C0E0703010000E8
:1013F0000000000000FCFE87C3E377FEFC00000F46
:101400001F3B3130381F0F00000C0EFFFF000000A3
:1014100000000030303F3F3030000000000C0E076D
:1014200083C3E77E3C00003C3E3733313030300030
:10143000000303C3C3C3E7FE3C000030303030304C
:10144000391F0F0000C0E070381C0EFFFF000003C2
:1014500003030303033F3F00003F3F33333373E392
:10146000C300000C1C383030381F0F0000FCFEC7D2
:10147000C3C3C78E0C00000F1F383030391F0F0058
:10148000000303C3E3733B1F0F000000003F3F0056
:1014900000000000003CFEE7C3C3E7FE3C00000F75
:1014A0001F393030391F0F00003C7EE7C3C3E7FE11
:1014B000FC0000000030381C0E07030000183C3C04
:1014C00018000000000000060F0F0600000000F0EA
:1014D000F8DCCEC7C7CEDCF8F03F3F0000000000CC
:1014E000003F3FFFFFC3C3C3C3C3E7FE3C3F3F30E2
:1014F00030303030391F0FFCFE0703030303070EA3
:101500000C0F1F3830303030381C0CFFFF03030342
:10151000070E1CF8F03F3F303030381C0E0703FF39
:10152000FFC3C3C3C3C3C303033F3F3030303030B6
:10153000303030FFFFC3C3C3C3C3C303033F3F0007
:1015400000000000000000FCFE0703C3C3C3C7CEB9
:10155000CC0F1F3830303030303F3FFFFFC0C0C0AD
:10156000C0C0C0FFFF3F3F0000000000003F3F0041
:10157000000303FFFF03030000000030303F3F3053
:10158000300000000000000303FFFF03030C1C38C1
:101590003030381F0F0000FFFFC0E0F0381C0E078E
:1015A000033F3F000103070E1C3830FFFF0000001F
:1015B00000000000003F3F3030303030303030FF2E
:1015C000FF0E1CF8F81C0EFFFF3F3F00000000005C
:1015D000003F3FFFFF3870E0C08000FFFF3F3F004B
:1015E00000000103033F3FFCFE070303030307FE64
:1015F000FC0F1F3830303030381F0FFFFFC3C3C31C
:10160000C3C3E77E3C3F3F0000000000000000FC39
:10161000FE070303030307FEFC0F1F383033371E9A
:101620001C3F33FFFFC3C3C3C3C3E77E3C3F3F0040
:101630000003070E1C38303C7EE7C3C3C3C3C78E0C
:101640000C0C1C3830303030391F0F03030303FFFC
:10165000FF03030303000000003F3F00000000FF02
:10166000FF000000000000FFFF0F1F383030303057
:10167000381F0FFFFF000000000000FFFF03070EF0
:101680001C38381C0E0703FFFF000000000000FF9D
:10169000FF0F1F38381F1F38381F0F0F1F38F0E09B
:1016A000E0F0381F0F3C3E0703010103073E3C3FBB
:1016B0007FE0C08080C0E07F3F000000013F3F012D
:1016C00000000003030383C3E3733B1F0F3C3E375B
:1016D00033313030303030000000000000000000B6
:1016E000003030303030303030303000003030308A
:1016F000303070E0C00C1E3F33333333333F3FFF95
:10170000FFC0E070303070E0C03F3F3030303030EC
:10171000381F0FC0E070303030303000000F1F38FD
:1017200030303030381C0CC0E070303070E0C0FF1A
:10173000FF0F1F3830303030303F3FC0E070303066
:10174000303070E0C00F1F3B33333333330303C0FB
:10175000C0FCFEC7C303070E0C00003F3F000000A3
:10176000000000F0F89C0C0C0C0C0CFCFC0001338D
:10177000333333333B1F0FFFFFC0E070303070E076
:10178000C03F3F0000000000003F3F00003030F34A
:10179000F300000000000030303F3F303000000018
:1017A0000000003030F3F300000C1C383030381FDC
:1017B0000F0000FFFF0080C0E0703000003F3F03DB
:1017C000070F1C3830000000000303FFFF0000007B
:1017D00000000030303F3F30300000F0F03070E06B
:1017E000E07070E0C03F3F0000030300003F3FF0A7
:1017F000F0C0E070303070E0C03F3F0000000000FB
:10180000003F3FC0E0703030303070E0C00F1F3814
:1018100030303030381F0FF0F03030303030F0E002
:10182000C03F3F0303030303030100C0E0F0303077
:1018300030E0C0F0F000010303030303033F3FF077
:10184000F0C0E070303070E0C03F3F0000000000AA
:10185000000000C0E0F03030303030000030313374
:10186000333333333F1E0C3030FFFF303000000085
:101870000000000F1F383030381C0CF0F000000062
:10188000000000F0F00F1F383030381C0C3F3FF0E4
:10189000F0000000000000F0F003070E1C38381CB8
:1018A0000E0703F0F0000000000000F0F00F1F38FA
:1018B000381C1C38381F0F3070E0C08080C0E070CA
:1018C0003030381C0F07070F1C3830F0F080000054
:1018D000000000F0F0000133333333333B1F0F308F
:1018E00030303030B0F0F0703030383C3E3733318B
:1018F00030303000000000000000006F00000700E2
:101900000700147F147F14242A7F2A1223130864EB
:101910006236495522500005030000001C22410098
:101920000041221C0014083E081408083E08080064
:10193000503000000808080808006060000020100F
:10194000080402003E49453E0000427F40006251CB
:1019500049460041494936001814127F0027454581
:1019600039003E49493200017905030036494936BC
:10197000000649291E0000363600000056360000D9
:1019800008142241141414141441221408000201F2
:1019900051090600060909067E0909097E7F4949A1
:1019A00049363E414141227F4141221C7F494949FC
:1019B000417F090909013E4149497A7F0808087FAA
:1019C00000417F41002040413F017F081422417FB8
:1019D000404040407F020C027F7F0408107F3E4160
:1019E00041413E7F090909063E4151215E7F0919A7
:1019F0002946264949493201017F01013F404040C3
:101A00003F1F2040201F3F4030403F6314081463B5
:101A100007087008076151494543007F41410002B2
:101A2000040810200041417F0004020102044040EC
:101A3000404040000102040020545454787F484440
:101A400044383844444420384444487F385454543B
:101A500018087E0901020C5252523E7F0804047895
:101A600000447D40002040443D007F102844000099
:101A7000417F40007C041804787C080404783844D2
:101A80004444387C14141408081414187C7C08048A
:101A900004084854545420043F4440203C40402013
:101AA0007C1C2040201C3C4020403C442810284402
:101AB0000C5050503C4464544C44000836410000E3
:101AC000007F000000413608000808221C08081C9E
:101AD00022080840800804201002019CCE003264D5
:101AE000E2F1003264645A505A6450463C46649CA9
:101AF000141E465A536572766F20546573740047FE
:101B000079726F2053657475700048656C69205355
:101B10006574757000456C65766F6E5C44656C74B9
:101B20006100562D5461696C00537469636B7920B0
:101B3000542D43757400542D4375740053696D70B2
:101B40006C6520342D4348003C1B361B291B221B8F
:101B5000151B0A1BFF1AF41A0000891112239B326D
:101B60002446AD573665BF74488CC19D5AAFD3BE6D
:101B70006CCAE5DB7EE9F7F88110080193331A227D
:101B8000A5562C47B7753E64C99C408DDBBF52AE4D
:101B9000EDDA64CBFFF976E802218B30100299135D
:101BA0002667AF763444BD554AADC3BC588ED19F2D
:101BB0006EEBE7FA7CC8F5D983310A20911218033D
:101BC000A7772E66B5543C45CBBD42ACD99E508F0D
:101BD000EFFB66EAFDD874C904428D5316619F700D
:101BE0002004A9153227BB364CCEC5DF5EEDD7FCED
:101BF0006888E1997AABF3BA85520C4397711E60FD
:101C0000A1142805B3373A26CDDE44CFDFFD56ECCC
:101C1000E9986089FBBB72AA06638F7214409D51DC
:101C20002225AB343006B9174EEFC7FE5CCCD5DDAC
:101C30006AA9E3B8788AF19B87730E6295501C41BC
:101C4000A3352A24B1163807CFFF46EEDDDC54CD8C
:101C5000EBB962A8F99A708B088481951AA793B69C
:101C60002CC2A5D33EE1B7F04008C919522BDB3A8C
:101C7000644EED5F766DFF7C899400859BB712A65C
:101C8000ADD224C3BFF136E0C1184809D33B5A2A6C
:101C9000E55E6C4FF77D7E6C0AA583B4188691973C
:101CA0002EE3A7F23CC0B5D14229CB38500AD91B4C
:101CB000666FEF7E744CFD5D8BB502A4999610871C
:101CC000AFF326E2BDD034C1C3394A28D11A580B2C
:101CD000E77F6E6EF55C7C4D0CC685D71EE597F4EC
:101CE0002880A1913AA3B3B2444ACD5B5669DF780C
:101CF000600CE91D722FFB3E8DD604C79FF516E4DC
:101D0000A9902081BBB332A2C55A4C4BD7795E68EB
:101D1000E11C680DF33F7A2E0EE787F61CC495D5BB
:101D20002AA1A3B03882B193466BCF7A5448DD59CB
:101D3000622DEB3C700EF91F8FF706E69DD414C59B
:101D4000ABB122A0B9923083C77B4E6AD5585C49AB
:101D5000E33D6A2CF11E780F536911241FBECFEFAB
:101D6000D0E1DEBFCDBF11E0A0E0B1E0E8ECF4EDE2
:101D700002C005900D92A632B107D9F71DE0A6E288
:101D8000B1E001C01D92A038B107E1F71DE1CAE53D
:101D9000DDE104C02297FE010E94116AC835D10717
:101DA000C9F70E9483670C94626A0C940000E7E60E
:101DB000F5E040E0842F806487B9369A3699FECFEB
:101DC00024B135B1369A3699FECF84B195B1820FE0
:101DD000931F819391934F5F483061F70895E0918D
:101DE000400594E0E99FF0011124E80FF11DE95B43
:101DF000FC4F84918F5F0895853050F0883020F03B
:101E00008E3020F482E0089581E0089583E0089503
:101E100080E008952AE0829FC001112483519E4FE3
:101E2000089525E0829FC0011124835D9C4F089591
:101E30008F929F92AF92BF92DF92EF92FF920F9399
:101E40001F93CF93DF93C82FD62F5A01122FF02E56
:101E5000822F8470D82E57FF10C0882311F08CE198
:101E600001C08FE0212F4DE26D2F9C2F981B892FF1
:101E70000E946458B194A194B108212F2F214AE304
:101E80006D2F8C2F0E9464586CE370E0C5010E9496
:101E9000BA694B015C01012F00619B0140E050E0F9
:101EA00062E0E62E6D2F8C2F0E94335ADD2011F058
:101EB0008AE101C08FE00F2D0061950140E050E004
:101EC00092E0E92E6D2F8C0F0E94335ADF91CF9153
:101ED0001F910F91FF90EF90DF90BF90AF909F9078
:101EE0008F900895CF93DF93D62FC22F206250E0BA
:101EF0000E94435BC7FD09C02C2F46E76D2F8091E0
:101F0000810CDF91CF910C946458DF91CF910895AB
:101F1000242F40913C010C94720F0F93022F24FF49
:101F200003C00F7E9CE201C094E2411106C024E090
:101F300042E253E00E94F6580FC0453028F42FEFDC
:101F4000240F4FE253E006C0941730F02BEF240F1C
:101F500040E852E00E9418590F9108950F93CF93D3
:101F6000DF93C82FD62F022F411104C024E04BE786
:101F700052E00EC04A3010F086E101C081E18C0FC2
:101F800050E0202F6D2F0E94435B22E048E752E093
:101F90006D2F8C2F0E94F658DF91CF910F910895ED
:101FA0000F931F93CF93DF93D62FC42F022F16E0EA
:101FB000180F442339F0463141F04A3E81F44BE595
:101FC00053E005C044E752E002C047E553E06D2FFF
:101FD000812FDF91CF911F910F910C942C5947FFC6
:101FE00004C041E20E946458C1952FEF2C0F4FE5C9
:101FF00053E06D2F812F0E941859DF91CF911F91CF
:102000000F910895EF92FF920F931F93CF93DF9359
:10201000D82F162FF42EE22EC091DE0181E0821718
:1020200008F442C02C2F27FD2195203168F4042F9D
:1020300042E452E08D2F0E941859CF3FCCF52F2D4E
:1020400041E2612F8AEF19C0253230F41C1614F4D6
:1020500041EF22C04FE020C0CA339CF0C353042F8D
:102060002C2F4BEF51E08D2F0E941859C0310CF4EA
:10207000D6502F2D45E2612F82E18D0F0E946458CA
:1020800017C0242F4DE682E18D0F0E9464581C1664
:1020900014F44CED01C044E24C0F2F2D612F8AEF58
:1020A0008D0F0E94D00F04C082E0281313C004C01B
:1020B000E11010C0C13071F42F2D40914E04612FFA
:1020C0008AEF8D0FDF91CF911F910F91FF90EF90CD
:1020D0000C94D00FDF91CF911F910F91FF90EF9053
:1020E00008958C3038F4E82FF0E0EE0FFF1FEE5526
:1020F000F84F22C08431C0F4482F50E0DA01AA0F13
:10210000BB1FA05FBE4F2D913C91803148F4FA0176
:10211000EE0FFF1FEA5EFA4F80819181281B390B79
:10212000C901880F991F0895843248F4E82FF0E020
:10213000EE0FFF1FE65AF84F8081918108958E328D
:1021400018F484520C94991C80E090E008950E9449
:102150007F678111FCCF1092B20C08950F931F93EB
:10216000CF93DF938C01EB010E94145824E041E4EB
:1021700053E060E082E20E942C59B80180E20E94A4
:102180004C59BE0188E20E944C5965EE71E080E333
:102190000E944C59DF91CF911F910F910C94EA5BF3
:1021A0000F93262F00E04FE553E060E10E9418599D
:1021B0000F910895CF93DF93D6E1C0E08D2F0E9459
:1021C000CC5CCC0FC82BD150DE30C1F78C2FDF9107
:1021D000CF9108950F931F93CF93DF93082FC3EDF3
:1021E000D1E01AE0499124E0602F812F0E946458C9
:1021F000155F1837B9F7DF91CF911F910F910895AF
:102200001F93CF93DF93EC01162F0E941458BE0149
:1022100088E10E944C59111109C047ED51E068E373
:102220008CE10E94525941E453E002C04FEC51E06E
:1022300024E060E082E20E942C59DF91CF911F914F
:102240000C94EE5B61E00E9400110C94EA5B70E07C
:10225000882399F090E0019725E0289FF001299FBD
:10226000F00D1124E60FF71FEE0FFF1FE856FB4F8E
:10227000808191818B509E4F0895FB01EE0FFF1FCF
:10228000EE5FFE4F0190F081E02D8081992787FD60
:10229000909508951F93CF93DF93D82F162FC4E006
:1022A000DD2399F0612F8D2F0E9427119C01253F7E
:1022B00081E0380764F08BE0820F8D1710F08CE01E
:1022C000820FC15029F0D82FEBCFC0E001C0CD2F35
:1022D0008C2FDF91CF911F910895CF93C62F0E942D
:1022E0004A116C2FCF910C9427110F931F93CF930A
:1022F000DF93EA01062F10E08823B9F00E944A110B
:10230000882399F090E0019725E0289FF001299F0C
:10231000F00D1124E00FF11FEE0FFF1FE856FB4FE9
:10232000C55FD140D183C08317C0CE0183589F4F72
:102330008B3F910540F01C161D061CF4CDE7D0E044
:1023400002C0C3E8DFEFF801EE0FFF1FEE5FFE4FA4
:102350000190F081E02DC08386E0DF91CF911F9145
:102360000F910C94C152AF92BF92CF92DF92EF9235
:10237000FF920F931F93CF93DF938C017B016A0130
:10238000A22EB090B3019B2D9F7D943439F08091A3
:102390008007882309F481C0933439F4E801219639
:1023A00083E10E94D86685E00BC0953419F0923421
:1023B00009F076C0E801219784E10E94D86684E0A4
:1023C0000E94CC5C81115EC0E114F104E1F481E073
:1023D000C816D104C1F480E6B81619F08EE2B8121E
:1023E00012C010928007C1E00115110509F0C0E08C
:1023F000D0E08B2D0E941B5D8EE2B81203C081E0FD
:102400008093B407B12C40913F0150914001C41B0F
:10241000D50B8091B407833031F48091BC01C80F93
:10242000D11D87FDDA95CC16DD0644F48B2D0E9474
:102430001B5D83E10E94D866E6010AC0CE15DF0568
:102440003CF48B2D0E941B5D84E10E94D866E7015D
:10245000C017D107A1F0209751F48B2D0E940B5D7E
:1024600017FF02C083E101C084E10E94D8668A2D73
:1024700083700E94C15281E08093470113C0109283
:10248000470110C0CC27DD27C01BD10B85E00E947F
:102490001B5D84E00E941B5D97CF953409F48ACFC1
:1024A000E80192CFCE01DF91CF911F910F91FF9064
:1024B000EF90DF90CF90BF90AF900895552747FDE4
:1024C0005095772767FD7095992787FD90950E9415
:1024D000B311089522E00C945E12462F22E060E0D2
:1024E0000C945E1221E00C945E12462F21E060E015
:1024F0000C945E12E0914901F0E0EE0FFF1FE45BE7
:10250000FE4F808191810895E0914901F0E0EE0F46
:10251000FF1FE65BFE4F918380838FEB8093480122
:102520000895E5EBF7E0108E168A158A178A08954C
:10253000E3E5FDE037A1303180F420A541E0420F12
:1025400040A7DF01A20FB11DA20FB11D8D939C9377
:10255000403108F010A63F5F37A3089590E08C5FEC
:102560009E4F0C94981290E00C9498128093BE01A8
:1025700090E040970C949812FC0190914B0580A13B
:1025800091FF74C091A1882311F0946001C09B7FDA
:1025900091A386A1813059F5C79A37A121A1332390
:1025A00021F181A541E0480F41A7DF01A80FB11D2E
:1025B000A80FB11D8D919C9195A384A3403108F083
:1025C00011A6315037A397FD02C031E101C038E2B6
:1025D00033A32C7F97FD226021A381A18BBBC798D9
:1025E0008FE182A382E086A308952BBB48C08111AE
:1025F0000CC0C79A81A1836081A38BBB8091820CA0
:102600008D3308F43CC086E02FC0823009F438C016
:1026100081A18BBBC79ABF9800C0000000C086B3E1
:102620008078BF9A96A1933049F4882329F083A13A
:10263000815083A3811123C084E016C0943021F41B
:102640008823E9F083E00EC0953039F483A18150EE
:1026500083A3811114C081E007C0963081F48823E0
:1026600071F084E183A385E086A309C090914805B9
:1026700096FB992790F9891711F0C79A0895C79882
:1026800008951BBA8FE18ABB00C099B38FEF8ABB54
:10269000E4EBF1E08781882311F080E202C0892F0A
:1026A000807E8483292F207C8081281759F08074B4
:1026B000880F90783181891711F0315001C03F5F48
:1026C0003183208382819381891711F083838183F1
:1026D00008959091400590FD02C093E08927E82F6E
:1026E000F0E0E055F84FE081E7FDE95FE595E5951D
:1026F000E5951E1624F0EE2321F0E19502C080E856
:1027000001C080E0E8300CF0E7E0FF27E7FDF0953E
:10271000E95DFC4FE491EE2319F099E090935401A8
:102720008E2B0895833021F0811103C083E001C016
:1027300080E0E82FF0E0EE0FFF1FE959FA4F8081AB
:1027400091810895FF920F931F93CF93DF93F12C04
:10275000C0E0D0E08F2D0E949213092F10E0C00F2F
:10276000D11FF39484E0F812F5CFCE01DF91CF9121
:102770001F910F91FF9008950E949213209142059E
:1027800020FF03C0919581959109089578941F9237
:102790000F920FB60F9211248F93809126018F5FB5
:1027A000809326018F910F900FBE0F901F90189568
:1027B00078941F920F920FB60F9211242F938F933C
:1027C0009F93EF93FF93F89487B78F7B87BF78949D
:1027D00020917D0180917F0190914B05882359F0D4
:1027E00090FF07C080917D0D820F80937D0D87FF44
:1027F00002C01B9A01C01B9891FF2AC080918008DB
:10280000811126C0E3E5FDE086A1823009F583A1B0
:10281000882311F081501BC021A1C79A82A180FD9D
:1028200009C02D7F84A195A196FD2260880F991F74
:1028300095A384A381E082278BBB81A3C79882A143
:10284000815082A3811104C083E086A385E083A325
:10285000F89487B7806487BF7894FF91EF919F9138
:102860008F912F910F900FBE0F901F901895789415
:102870001F920F920FB60F9211242F933F934F93F5
:102880005F936F937F938F939F93AF93BF93EF93D8
:10289000FF9381B7845681BF8BE791E00E940D655D
:1028A0000E942A5D8091BF0C82608093BF0CEAE099
:1028B000F1E08081815011F0808304C084E6808340
:1028C00081E081838281815011F0828304C08AE09B
:1028D000828381E08383FF91EF91BF91AF919F91BC
:1028E0008F917F916F915F914F913F912F910F90B9
:1028F0000FBE0F901F90189578941F920F920FB6ED
:102900000F9211242F933F934F935F936F937F9375
:102910008F939F93AF93BF93EF93FF93209180008A
:1029200030918100F89480917D008F7D80937D00AF
:1029300078948091600590916105A901481B590B1D
:10294000CA019695879530936105209360059C0197
:10295000215A3F402F3D3E4220F481E080932701E1
:102960002CC0E09127012FEF2E0F283030F59C016D
:102970002152334027373540F0F424E62093BD013F
:1029800021E02E0F20932701F0E0EE0FFF1FEA5DFC
:10299000FE4F9C012C5D354040914605465F429FAD
:1029A000C001439F900D11246AE070E00E94BA6953
:1029B0007183608302C010922701F89480917D009A
:1029C000806280937D007894FF91EF91BF91AF91E9
:1029D0009F918F917F916F915F914F913F912F9137
:1029E0000F900FBE0F901F9018959C0155E03595E4
:1029F00027955A95E1F7280F391FAC01440F452F51
:102A0000441F550B241B350B892F990F990B859566
:102A1000820F931F08959DE7980F9B3F88F08E5774
:102A2000E82FF0E0EE0FFF1FE657FB4F808186177F
:102A30001CF46083862F0895481714F44083842F74
:102A4000089544E66CE90C940B15982F8091E401ED
:102A500084FF03C081E0923009F080E0089591E0A6
:102A6000823009F090E0892F089549E284029001B4
:102A70001124359527953595279587FD815C86FB33
:102A8000880F880B80F9A901481B510987FD5395D0
:102A9000CA0108954F925F926F927F928F929F9298
:102AA000AF92BF92CF92DF92EF92FF920F931F935C
:102AB000CF93DF93782E642E45E0461508F4D5C0F9
:102AC000882309F4D0C056E1851721F08AEE7812E8
:102AD00003C0CBC081E0CDC096E197150CF4C5C012
:102AE000872D87FD81958A3040F4825F0E94CC5CFF
:102AF00017140CF4BEC091E01DC08A50282F30E09E
:102B00006901CC0CDD1C8601020F131F075D1B4FF2
:102B1000F80182818F7009F4A8C0A9014A5A5E4F5A
:102B20007A0155E0651208C0F701908117140CF482
:102B300098C081E089279DC0F801508041800E94A3
:102B4000FC0E81110AC08FEF850D0E947110EC01FF
:102B5000F80181810E94351511C0823059F48FEF40
:102B6000850D0E947110EC01F801818181500E9455
:102B7000711004C080E090E0C0E0D0E0F801228154
:102B80002F70822E912CF4013197EE30F10508F070
:102B90006EC0EA5BFF4F0C940F6AD7FF39C0D19526
:102BA000C195D10935C0D7FF37C0D195C195D1099D
:102BB00033C0D1E0D60D4D2F60E0852D0E944A151F
:102BC000C82F4D2F60E0842D0E944A15F801228104
:102BD0002F70253069F4CC2309F449C0882309F407
:102BE00046C0F8018281982F907F69F591E036C048
:102BF000263019F4C111F5CFF1CF982F9C2720C0B2
:102C0000C817D907A1F5EDCFC817D90751F72FC0BD
:102C10008C179D0734F32BC0C817D90714F327C0AE
:102C2000C817D907F4F623C08C179D07D4F61FC028
:102C3000F601EE59FE4F91819095991F9927991FA2
:102C40009111CFCF0BC082958F7089300CF08F5FC0
:102C500041E0460D60E00E944A15982FF7019083ED
:102C600065CF892F06C0862F04C080E002C090E0A7
:102C7000F5CFDF91CF911F910F91FF90EF90DF90F3
:102C8000CF90BF90AF909F908F907F906F905F900C
:102C90004F90089540E060E080912D050E944A1514
:102CA000811114C08091390190913A01892B71F4FE
:102CB0001092730D8091820C90916605981751F0D7
:102CC0008093660583E59DE00C94BC1281E08093BF
:102CD000730DF0CF08952091390130913A012115FB
:102CE000310511F021503109882319F080914405F4
:102CF00001C080E090913801992329F090914C0512
:102D0000891708F4892F4AEF849FC0011124880F86
:102D1000991F8217930708F4C90190933A01809391
:102D200039010C944A16CF92DF92EF92FF920F93E3
:102D30001F93CF93DF938091830C9091840C90919B
:102D40006505282F291B20933B018093650560E0D2
:102D50008BE597E00E94643380913B01882309F45E
:102D6000C5C2E5EBF7E0878980FF0DC0808D91E05B
:102D7000980F908F943638F08356808F8589968986
:102D80000196968B858B8091BD01882319F0815027
:102D90008093BD0180E00E94C5520E9414580E9499
:102DA000605C182F482F4F70E42E5AEFE50EC0914B
:102DB000E501C43021F0C33019F4C4E001C0C8E01B
:102DC00087E08E1508F4A1C0812F807F803209F43E
:102DD0009CC0E091400594E0E99FF00111248E2D04
:102DE0008695E80FF11DE95BFC4F049180915C052D
:102DF00080FF03C083E0801B082F602F8091770540
:102E00000E944A11F82E602F0E946D119C01C11181
:102E10000CC0EC0197FF04C0CC27DD27C81BD90BE1
:102E2000D595C795D595C795CF5F023061F4809150
:102E3000E40180FF59C281E0C2E09091420590FF19
:102E400003C0C19501C080E0DD27C7FDD095E0FE3D
:102E500003C0C20FD31F04C0A9014C1B5D0BEA01C4
:102E6000209721F09D2F932797FF11C081110FC04C
:102E7000232B69F040E050E0602F8F2D0E947511E8
:102E8000812F0E941B5D86E10E94D8663DC09E0195
:102E900024583F4F293F310580F4AE01602F8F2D1C
:102EA0000E947511D7FF03C0D195C195D109D59561
:102EB000C795D595C7954C2F21C01C161D061CF42F
:102EC0004DE750E002C043E85FEF602F8F2D0E9476
:102ED0007511CE0183589F4F8B3F9105A8F4D7FF02
:102EE00003C0D195C195D109D7FD2396AE01559563
:102EF000479555954795519541955109445C65E134
:102F00008BE791E00E94C26510E0EDE3F1E0809173
:102F1000AE079091AF0720813181281B390B37FF15
:102F200002C0215E3F4F65E0359527956A95E1F730
:102F30002115310561F024813581281B390B37FFBC
:102F400002C02F5F3F4F35952795918380839583EE
:102F500084838091420585FF02C020E030E0338306
:102F60002283C4EBD1E02D818981821B8F3F09F43C
:102F700080E087FD8F5F85958887982F990F920F46
:102F80009D83812B0E946B1680915805895FE0918B
:102F90004901F0E0EE0FFF1FE65BFE4F208131811B
:102FA000245E3B4309F044C028852223B1F09E8172
:102FB000332727FD3095290F311D97FD3A952E3780
:102FC000310514F09DE705C023389FEF39071CF445
:102FD00093E89E8301C02E831886E0914F049E2FB4
:102FE000907E31F1E295E695E770F0E0E430F1058E
:102FF00054F4EE0FFF1FE855F84F208131813C5FFC
:1030000060E078E00CC0EE0FFF1FE657FB4F208119
:10301000332727FD309523583F4F6AEF70E047E094
:10302000429FC001439F900D11240E94A669862FE4
:103030009091BE0189130E94B6128091480587FFC6
:103040003BC0809155018823B9F1809154018823B8
:10305000A9F18091640587FD03C08F5F80936405AB
:1030600082E00E946913982F9F7789F02091640570
:10307000921720F510926405111120C0182F109599
:10308000111F1127111F83E6811B182F17C083E022
:103090000E946913982F9F7789F0209164059217F9
:1030A00068F410926405111109C0182F1095111FB2
:1030B0001127111F1C5902C01092540181E0809306
:1030C000550100917705E090BA01FF24E7FCF094E8
:1030D000CBE8D4E09AE0C92ED12C6881662309F4AC
:1030E00040C0653030F46150802F0E946D11BC01EA
:1030F0002BC0653041F1E62FF0E0EE0FFF1F6A3084
:1031000048F4EA56F84F6081718177FF0EC0695F1D
:103110007F4F0BC06D3078F4EA56F84F2081318133
:1031200037FF02C0295F3F4FB901B3E0759567953E
:10313000BA95E1F709C0E859F84F80819181B6014D
:103140000E94BA6901C0B70163382FEF72072CF0F3
:103150006D3771051CF06DE701C063E8FE01319722
:103160006083229644E0C939D40709F0B6CF809134
:10317000D1019091D2010097B1F060E00E9400115E
:103180000E947F6790916305992339F0811125C0D2
:103190001092D2011092D10120C08823F1F081E079
:1031A000809363051AC010926305C0914801CC2337
:1031B00031F01092480187E10E94D8661C2F1093CD
:1031C000B301E0914901F0E0EE0FFF1FE65BFE4F17
:1031D0000190F081E02D812F09950E94EE5BC09156
:1031E00065008BE791E00E94F964882311F084E187
:1031F00005C080917F0D882321F0815080937F0D41
:1032000006C0809163008695817080937E0D8091C9
:103210007E0D8093CF01882309F464C08091480516
:1032200085FD60C0CF7EC09365008091820C8F7158
:10323000823009F054C08091750590917605AC01FB
:10324000F4E0440F551FFA95E1F797FD0796BC018E
:10325000E3E075956795EA95E1F720912C05332712
:1032600027FD30952A5F3F4F629FC001639F900DFD
:10327000729F900D1124840F951F2091420526FD09
:1032800005C0609100017091010102C060EF70E023
:103290000E94A66980913C01680F711D6F5F7F4F8E
:1032A0007595679560933C0180916205805F80937E
:1032B0006205811114C080912B05681780F4623378
:1032C00070F06EE281E10E94DE668091420583FF2C
:1032D00006C082E390E090933A0180933901109206
:1032E000380104C0C0619FCF80E0A7CDDF91CF91AE
:1032F0001F910F91FF90EF90DF90CF900895CF93A3
:10330000DF93C62F2091D001222339F09093D20170
:103310008093D101DF91CF91089560E00E94001168
:10332000C11103C080912A0501C089E10E94DB5BC5
:1033300067E182E10E94DE660E94A710D1E00E9450
:103340007F67882321F0DF91CF910C94A7108091A3
:10335000BF0C833019F4A8951092BF0C40E060E0D8
:1033600080912D050E944A15811106C08091440567
:10337000811102C0CC2329F0D093730D0E944A160C
:10338000DECF1092730DFACF90914901911103C0D5
:10339000811106C00CC0811103C08FEF890F01C0DD
:1033A00080E0809349018EEB80934801089560E0AE
:1033B00082EC91E00C947F19E0914901E43028F00F
:1033C00060E085EB91E00C947F192FEB209348018E
:1033D000EF5FE0934901F0E0EE0FFF1FE65BFE4F69
:1033E0009183808308951F93CF93DF93C0EAD4E045
:1033F00090E0888111E0190F882341F040E060E0FF
:103400000E944A15882311F0812F05C0912F2A961A
:10341000143079F780E0DF91CF911F910895BF922A
:10342000CF92DF92EF92FF920F931F93CF93DF9390
:1034300080912601C2B7909126018913F9CFD0E07F
:10344000D82B80914F048F7150E1D52ED81A0E944D
:10345000D70E1EE517B90E9441130E94931617B9A3
:10346000369A3699FECF84B195B104964091000109
:103470005091010167E0649F9001659F300D112418
:10348000820F931F43E0969587954A95E1F79093B5
:103490000101809300018091BF0C833019F4A8953D
:1034A0001092BF0C2091260182B79091260129131A
:1034B000F9CF90E0922B8C1B9D0B2091D60630917A
:1034C000D7062817390720F49093D7068093D6069D
:1034D00080910D01882309F4DAC080915E059091F6
:1034E0005F05019690935F0580935E05CD2CFFE00C
:1034F000FC1508F476C00C2D10E0E801CC0FDD1FA0
:10350000C05BDB4F8881E82EE294E69437E0E3224B
:10351000F98095E09E1550F0EAEFEF1538F4EF2DA5
:10352000F0E0EE0FFF1FE656FD4FF0808F7109F4BB
:1035300056C040E060E00E944A15B82E80910D010F
:1035400001541E4F823009F448C08E2D857051F40D
:10355000F8018081811106C0BB2021F08F2D90E001
:103560000E9498128FEF8E0D823058F4F8018081FE
:10357000813099F5B11031C0F2E0EF122AC0F39416
:1035800028C085E08E1550F4F8018081811125C096
:10359000BB2019F189810E94BF1C1FC0F2E0FE15FB
:1035A000E0F4BB20D1F084E0E81631F095E0E916B4
:1035B00031F066E970E005C06CE271E002C068E5D8
:1035C00072E080915E0590915F050E94A669892B4B
:1035D00021F48F2D90E00E949812F801B082C394DC
:1035E00086CFB9E2EB2EB4E0FB2E02E611E0F70144
:1035F000C2808C2D8F700E94FC0E8330E1F5F801A3
:10360000C081D181209771F4F701C081C7FD06C048
:10361000C095FAE0CF02E001112419C0DD27C7FDF3
:10362000D09515C0D7FF12C0219689F4F701C1814A
:10363000C7FD06C0CF5FFAE0CF02E001112406C04B
:10364000DD27C7FDD095C095D09501C021978C2D61
:10365000807F71F08C2D82958F7089300CF08F5F98
:1036600040E060E00E944A15811102C0CFEFDFEF19
:10367000F801D183C083F3E0EF0EF11C0E5F1F4F02
:1036800081E00A37180709F0B2CF10920D0180913E
:103690000B01882309F47BC080915D058F5E982F14
:1036A000977F903618F490935D0503C087708093E0
:1036B0005D05C3EDD1E0F12CFD1409F45FC08E016E
:1036C00003581D4FF8018081982F907C9034C9F4E5
:1036D000880F880F40E060E0859585950E944A1527
:1036E000882379F080914B0580FF05C0FE01E258E8
:1036F000FD4F608101C061E046E48BE791E00E94EC
:10370000C265F8018081982F907C9038A1F52091B6
:103710005D05880F880F859585958731E4F0992799
:1037200087FD909547978130910539F0823091055A
:1037300041F0892B01F5237001C0207F21111BC0AE
:1037400003C027702230B9F4FE01E258FD4F80819A
:103750000E94BF1C10C020FD0EC040E060E00E942F
:103760004A15882341F0FE01E258FD4F80818058C0
:1037700090E00E949812F39422969ECF10920B0133
:1037800080915401882319F0815080935401DF9176
:10379000CF911F910F91FF90EF90DF90CF90BF904E
:1037A00008951F93CF93DF93D82F162FC42FB901FD
:1037B0000E944C59112329F06FE08C2F0E946D124A
:1037C000C82F4C2F50E0212F6D2F80E60E94435BC5
:1037D0008C2FDF91CF911F910895813649F40E947B
:1037E0001B5D81E00E94C41989E191E40E94DC190B
:1037F0006CEA7EE080E10E944C5966E97EE080E25E
:103800000C944C59CF93C82F8091BD0C80FF03C0FE
:103810006CEE7DE002C06AED7DE088E10E944C59CB
:10382000C13629F41092BD0C80E00E94C419809129
:103830000E08815080930E08811104C081E0CF9161
:103840000C94D866CF910895FF920F931F93CF9356
:10385000DF93182FF62E0AE08AE0189FE00111246A
:10386000C351DE4F2FE130E0211B3109029FA0013F
:10387000039F500D1124BE01CE010A960E94306AAA
:10388000FF2049F0BE016A5071094AE050E0CE01C4
:103890000E94306A0AC0FE0111920A95E9F78091F0
:1038A0001C088883898384E68A8310931E08DF912D
:1038B000CF911F910F91FF9008959C01220F331F0C
:1038C000280F391F9595879595958795280F391F4E
:1038D000959587959595879595958795820F931FD3
:1038E0000895429643E7489F9001499F300D112467
:1038F000C901E6E095958795EA95E1F7089581E09D
:103900000895E82FFF27E7FDF095ED52FD4EE49175
:10391000862F992787FD909583589F4FEE5FE23061
:1039200038F42AE0AC01249FC001259F900D11249A
:103930000895E82FFF27E7FDF095ED52FD4EE49145
:10394000ED3F4CF4EE0FFF0BE256FB4F80819927C1
:1039500087FD90950895ED3F59F074F0EF3F09F021
:103960005CF4EE0FFF0BE754F84F838994890895B8
:1039700080913C0190E0089580E090E00895CF921E
:10398000DF92EF92FF92F82E0E94991CEF2DFF27F5
:10399000E7FDF095ED52FD4EE491ED3F09F15CF449
:1039A000E63FDCF0EE0FFF0BE256FB4F80819927DC
:1039B00087FD909512C0EF3F09F07CF46CE370E056
:1039C0000E94BA696B017C0146E260E0C6010E9478
:1039D000E766C70160E045E305C060E040E002C083
:1039E00061E044E2FF90EF90DF90CF900C94E766A7
:1039F000BF92CF92DF92EF92FF920F931F93CF93DC
:103A0000DF93F82ED62EC42EE901102F8E2D817053
:103A1000B82EE0FE12C000E021E0240F4DED52E18F
:103A20008F2D0E94185912FD03C088E18F0D06C02A
:103A30008CE18F0D98EFD90E01C08F2D9E2D9870BF
:103A4000E3FC1F7BEC2DFF27E7FDF095ED52FD4ECB
:103A5000C49022E02C0D223088F412FF8450B11063
:103A6000865F1770012F212FAE016D2D86500E94A9
:103A7000180FC3E3CC0D8AEFF80E0AC0992311F09A
:103A80008DE38F0D212FAE016D2D0E94435BC0E2AF
:103A90008E2D867069F0E2FE04C08AE08F0D1B7FD8
:103AA00002C08091810C212F4C2F6D2D0E946458F3
:103AB0008C2FDF91CF911F910F91FF90EF90DF90AE
:103AC000CF90BF9008950F931F93CF93DF93C82F8C
:103AD000D62F042F122F49E651E10E942C5940E3C2
:103AE000400F212F6D2F8CE08C0FDF91CF911F9114
:103AF0000F910C946458DF92EF92FF920F931F93F3
:103B0000CF93DF93182FF62EC42FD22EDE2DD37035
:103B1000A1F08091B301803881F48DE7840F8B3F51
:103B200040F0E42FF0E0EE0FFF1FE257FC4FC081A2
:103B300001C0CEE782E00E94C1528DE78C0F2E2D8E
:103B40008B3FA0F043E84C0F6F2D8EEE810F0E944B
:103B5000631DDD2309F122E042E850E06EE770E0EA
:103B60008C2F90E00E94B311C82F16C04C2F552700
:103B700047FD50956F2D812F0E94435BDD2361F03F
:103B8000402F6D2D8C2FDF91CF911F910F91FF90C2
:103B9000EF90DF900C946A128C2FDF91CF911F91E0
:103BA0000F91FF90EF90DF900895CF93DF939EE009
:103BB000899FE0011124C358DC4F40E060E08C8510
:103BC0000E944A15882349F040E060E08D850E94FC
:103BD0004A15811104C081E003C080E001C082E089
:103BE000DF91CF910895EF92FF920F931F93CF93A0
:103BF000DF93F82EE62EC42FD42FD695062F0D1B5B
:103C0000182F1D1B602F812F0E94E7596D2F6E0DFD
:103C10004C2F812F0E94E4594C2F602F8D2F8F0D38
:103C20000E94E7594C2F602F812FDF91CF911F9178
:103C30000F91FF90EF900C94E45921E0AC0160E00B
:103C400080E00C942C591F93CF93DF93182FCEE074
:103C5000D1E08FE898E00E941D1E1136B1F068F4A3
:103C60001036D1F48FEF888319821092D706109204
:103C7000D60687E10E94D8660FC0123619F01336B7
:103C800021F00AC088E99EE102C084EE9BE3DF9147
:103C9000CF911F910C94841260E878E088E00E9434
:103CA0004C594981469550E068E084E50E94525B9A
:103CB00061E778E080E10E944C594881469550E0E8
:103CC00060E184E50E94525B62E678E088E10E9450
:103CD0004C59498150E08881481B510957FF02C067
:103CE0004F5F5F4F5595479568E184E50E94525BB1
:103CF00069E578E080E20E944C598091D606909167
:103D0000D70629E1289FA001299F500D112456951F
:103D100047955695479520E360E284E50E94435B12
:103D200066E478E088E3DF91CF911F910C944C59C1
:103D30000F931F93CF93DF93182FC5EBD7E081E448
:103D400098E00E941D1E113678F0133628F01336C5
:103D500059F483E29EE102C084EE9BE3DF91CF91B0
:103D60001F910F910C94841268E378E088E00E9420
:103D70004C594A815B8100E020E068E08AE20E94C1
:103D8000180F4C815D8120E068E08EE40E94180FDE
:103D90006FE278E080E10E944C594E815F8120E023
:103DA00060E18AE20E94180F4885598514E0569513
:103DB00047951A95E1F720E060E18EE40E94180F24
:103DC0006AE278E080E00E944C594881598120E005
:103DD00060E08EE40E94180F4EE76CE382E00E94E0
:103DE000E45943E26CE185E00E94E759CBE043E00F
:103DF0006BE38C2F0E94E759CA5FC338C1F710915B
:103E0000D9068091D806893710F4C0E001C0C12FCF
:103E1000D6E00CE3EC2FF0E0E652F94F4081602F42
:103E2000641B8D2F0E94E759CF5FC83708F0C0E0B0
:103E3000C11719F0DF5FDE3769F7DF91CF911F916E
:103E40000F91089591E0211101C090E0442319F0F1
:103E500047E553E002C04BE553E0292F0C942C5961
:103E60000F9301E0211101C000E0242F41E651E150
:103E70000E9418590F9108957F928F929F92AF924E
:103E8000BF92CF92DF92EF92FF920F931F93CF9347
:103E9000DF93EC01162FD42E4901B0905A074091C0
:103EA000AA075091AB072091AC073091AD07EDE325
:103EB000F1E086819781841B950B97FDCF96A6E054
:103EC00095958795AA95E1F7682F80937D07808562
:103ED0009185821B930B97FDCF9676E095958795FC
:103EE0007A95E1F7982F80937B07662311F057832B
:103EF0004683992311F03187208780917C078111B7
:103F000004C08091420585FF06C010927D07109283
:103F10007B0710927C0720917D07211108C08091BA
:103F20007B07811104C082819381892B61F080918C
:103F300044053AEF839FC0011124880F991F909385
:103F40003A018093390181149104B1F18881811182
:103F500097C18091B407882309F49DC1813009F489
:103F6000ACC12111B1C1153609F4D1C1143609F41F
:103F7000D8C1772473948091B407811102C082E084
:103F8000782E402F50E0272D60E08FE70E94435BA2
:103F90000A3008F47EC10FE6272D4FE260E0802F43
:103FA0000E9464584D2D50E04F5F5F4F272D60E019
:103FB0008FEF800F0E94435BE114F10451F0988170
:103FC0008C2D9C1508F4892FF701E80FF11DE49161
:103FD00001C0E0E08091B407813081F58091BC019F
:103FE00018166CF4BE1610F4B39411F588818A1576
:103FF00018F48F5F888301C01882B12C19C0882300
:10400000B9F0B11014C08881882319F081508883D9
:1040100001C0A882E114F10459F098818C2D9C15FF
:1040200008F4892FF701E80FF11DB49001C0BA948C
:104030001092BC011E3249F483E005C0833029F49C
:104040001E3219F481E08093B407E114F10451F0B9
:1040500098818C2D9C1508F4892FF701E80FF11D2C
:10406000549101C050E080918007811145C080913A
:104070007B07882301F14881481B47FD40E08A2DDA
:1040800090E0242F332727FD3095281739070CF0AF
:104090004A2D4883E114F10459F0C41608F44C2D5C
:1040A000F701E40FF11DE491EB1518F4BE2E01C0E9
:1040B000B12C10927B0728812223F1F080917D079B
:1040C0008823D1F0B81AB7FCB12C8B2D992787FD26
:1040D0009095E114F10479F03C2D2C1508F4322F61
:1040E000F701E30FF11DE4912E2F30E082179307C3
:1040F0001CF0BE2E01C0B12C103669F190F41234C0
:1041000009F473C028F41132A9F11E3221F197C0CD
:10411000143409F446C008F476C0153409F451C0CB
:104120008EC0153609F451C040F4133609F46EC040
:10413000D8F5123609F45CC082C01E38C1F01F3BAE
:1041400031F0113809F07BC01092800721C018822D
:104150001092800738C08881882309F470C081E0FC
:1041600090918007911180E08093800768C08EE86D
:104170000E941B5D80918007882319F010928007B0
:104180005EC08881882311F0892831F41092B40729
:1041900080E00E94C41953C087E10E94D86618824B
:1041A0004EC0B51609F44BC0EF2809F448C0809101
:1041B0008007811144C0B51610F4B39411C0B12C1E
:1041C0000FC0B11002C0B12C3AC0EF28C1F18091EC
:1041D0008007811134C0BB2011F0BA9401C0B52E04
:1041E000552369F11092B3012AC088818A1539F1EB
:1041F00080918007811123C088818A1510F48F5F18
:104200000DC018820EC088818823C9F08091800774
:10421000811115C08881882319F08150888301C0DD
:10422000A882E114F10479F288818C1508F4C82E73
:10423000F701EC0DF11DE490EB1408F4BE2C809115
:10424000800781110AC021E080913F0190914001D7
:10425000892B09F420E0822F01C081E080937F0741
:10426000B0925A07DF91CF911F910F91FF90EF907D
:10427000DF90CF90BF90AF909F908F907F900895E8
:1042800080918007811103C081E08093B407712C75
:1042900072CE05E781CE8091BC01181624F08823E8
:1042A00019F015E601C014E61092BC011E3209F0A7
:1042B00058CE81E08093B40705C01E3209F051CE7C
:1042C0001092B40710E04DCE8091800781114BCE43
:1042D000ED2DE21BE7FDE0E0202F30E08E2F992747
:1042E00087FD90958217930714F0EFEFE00FFF27FB
:1042F000E7FDF0958D2D90E0E817F90729F0EE0F16
:10430000FF1FE80DF91D1EC010927D072CCED110A5
:1043100001C0D02EF401ED0DF11DED0DF11D329710
:1043200011C02D2D30E0802F90E00197281739071C
:104330001CF411E01D0D01C010E0810E911C810ED6
:10434000911CF40185919491DF91CF911F910F9170
:10435000FF90EF90DF90CF90BF90AF909F908F90A5
:104360007F900C948412AF92CF92EF92FF920F93B2
:10437000AE2CC12CE12CF12C0E943C1F0F91FF9020
:10438000EF90CF90AF900895EF920F93E42E00E05E
:1043900020E030E040E00E94B3210F91EF900895BB
:1043A000BF92CF92DF92EF92FF920F931F93CF9322
:1043B000DF93C82F85E19BE00E941D1EEE24E3944D
:1043C00006E022EB31E144E06C2F86E098E00E94A9
:1043D000B321B090060810925501C2EAD7E010E070
:1043E00000E0C12CB4E0DB2EE12CF12C41E4612F84
:1043F00088E10E94F35841E3400F612F8EE10E9453
:10440000F358802F0E949213AC01612F8AE20E9420
:104410005559073081F0A881B98124E630E00E9427
:104420006E69A70196010E94F069A901612F8AE5D2
:104430000E94525B0AC081E0B81611F040E201C050
:1044400041E2612F8AE50E94880F0F5F185F229674
:10445000083061F661E17BE088E20E944C594091AE
:1044600000015091010160E388E70E94525B81E006
:10447000B8120AC0B0927C074FE761E880912C0522
:104480000E94721280932C05DF91CF911F910F91A2
:10449000FF90EF90DF90CF90BF900895EF920F9331
:1044A000CF93C82F8CED9AE00E941D1EE12C06E0F0
:1044B00022EB31E142E06C2F84E098E00E94B321CE
:1044C0006EEC77E080E10E944C596EEF77E088E176
:1044D0000E944C596DEE77E080E20E944C596EEDDF
:1044E00077E088E20E944C5962EC77E080E3CF915C
:1044F0000F91EF900C944C597F928F929F92AF92B4
:10450000BF92CF92DF92EF92FF920F931F93CF93C0
:10451000DF93C82F83E291E10E941D1ED7E0AD2EEC
:10452000CC24C39411E2E12E11E1F12E0BE02EEB2D
:1045300031E14AE06C2F85E198E00E943C1FA09099
:10454000150870905A070BE8E02E04E0F02ECAE838
:10455000D4E0CC24C394D12C18E0B12C6EE171E1ED
:10456000812F0E944C5940E34C0D612F8CE00E943A
:10457000F358912CAC14BD0441F4791006C080911D
:104580008007811105C021E001C020E0812C03C01B
:1045900022E088248394911013C0022FF701208118
:1045A00045EC50E1612F88E40E9418598820C1F041
:1045B0006CE1F70180810E946D12F701808310C0C9
:1045C0004881552747FD5095612F8CE60E94435B3B
:1045D000882031F04DE763E888810E946A12888361
:1045E0009394F2E09F12C6CF185F82E0E80EF11CB0
:1045F0002296EFEFCE1ADE0A103409F0AFCFDF912A
:10460000CF911F910F91FF90EF90DF90CF90BF90CF
:10461000AF909F908F907F9008957F928F929F92FE
:10462000AF92BF92CF92DF92EF92FF920F931F93C0
:10463000CF93DF93D82E84ED9AE00E941D1E66E092
:10464000A62E75E0C72EEEECEE2EEAE0FE2E06E07A
:1046500022EB31E141E06D2D83E098E00E943C1FA8
:10466000C090030880905A078091630081FF04C0C6
:1046700067EC7AE088E1FCC0CA94809180078823C7
:1046800019F053E0952E02C099249394C6E3D5E027
:10469000B12C10E1AA24A394AB0C20E04A2D612F89
:1046A00080E00E948D0FF12CCB1002C08F1411F00E
:1046B00000E001C0092D802F8270782E92E0F9165B
:1046C00009F444C0E3E0FE1609F455C0F1E0E980C6
:1046D000FF16D1F0E294E694E69443E0E4222E2D16
:1046E0004CEB5AE0612F88E10E941859772009F4B9
:1046F0005AC062E08E2D0E9475128295880F880F35
:10470000807C99819F731FC0EE0CEE0CE594E594BC
:104710008E2D9DE08902F0011124F7FD3396AF0143
:104720005595479555954795202F612F82E40E9416
:10473000435B7720C1F14FE161EE8E2D0E94721232
:104740008F739981907C982B99832DC0E880EE2DF2
:10475000E770EE2E2E2F4EEA5AE0612F88E40E9479
:104760001859772001F163E08E2D0E947512877031
:104770009881987F16C0E880E594E594E594202F11
:104780004E2D612F8AE50E94D00F772061F04FE017
:1047900061EF8E2D0E947212880F880F880F98810A
:1047A0009770982B9883F394F4E0FF127DCF185FF5
:1047B0002296AF1611F0BA2C6DCF63EA7AE080E34F
:1047C0000E944C5984E0C8120AC048E266EF80910A
:1047D00046050E9472128093460521E201C020E244
:1047E00040914605552747FD5095465F5F4F60E372
:1047F0008EE40E94435BEE24E39495E0C912E12C21
:104800002E2D4FE95AE068E380E00E942C5908E21F
:1048100011E0CEE2D5E020E3F22EF8014191519172
:104820008F0169917991461B570B440F551F20E268
:1048300068E38F2D0E94435BF8E1FF0E80E9F812D8
:10484000ECCFEE2091F090E6D9120FC088E0E8E2BC
:10485000F1E0AEE2B5E001900D928A95E1F781E0DA
:104860000E94C15287E10E94D8666FE87AE088E032
:10487000DF91CF911F910F91FF90EF90DF90CF903C
:10488000BF90AF909F908F907F900C944C591F9346
:10489000CF93DF93C82FD62F142F47E16CE20E94ED
:1048A000F31D43E06BE28C2F0E94E75943E06CE27A
:1048B0008FEF8C0F0E94E459812F69EF0E94986955
:1048C000282F245D8D2F67E00E94986945E0622FB4
:1048D0008C0FDF91CF911F910C94F31DCF92DF923B
:1048E000EF92FF920F931F93CF93DF93C0EBD7E02C
:1048F000498168818AE20E9447244A816B8186E56A
:104900000E944724C2EAD7E02896FAE3FF2E0DE57D
:1049100010E0A7E3CA2E899199919C5FB8010E948B
:10492000BA69DD24D394D60EEC2CE61A4D2D6E2DEB
:104930008F2D0E94E7594D2D6E2D81E08F0D0E9425
:10494000E7594D2D6E2D82E08F0D0E94E75985E0CD
:10495000F80E89E4F812DFCFDF91CF911F910F910C
:10496000FF90EF90DF90CF900895DF92EF92FF924B
:104970000F931F93CF93DF93F82E8AE49BE00E945E
:104980001D1EEE24E39406E022EB31E145E06F2D9D
:1049900087E098E00E94B32110920708CEEDD7E09F
:1049A00010E0812F0E949213488159818417950746
:1049B0000CF4AC01499359932C853D852817390790
:1049C0000CF49C013D872C87143060F0FE01709739
:1049D000240F351F37FF02C02F5F3F4F35952795B6
:1049E000318320831F5F1730E1F68091FA078093AF
:1049F0007C0790E2F91621F08FEBF8120EC00BC085
:104A00008F5F8093FA07833041F487E10E94D86674
:104A100081E00E94C1521092FA078091FA0781301A
:104A200089F050F0823009F072C010925501CDEF3C
:104A3000D4E0EEEDF7E01FC069E37BE088E10E947F
:104A40004C5965C0C0EDD7E0D12C08E9E02E0AE34F
:104A5000F02E08E615ECFF86EE861D8F0C8F8D2D4F
:104A60000E94921389939993D39497E0D912F3CF2C
:104A70006BE27BE043C061917191848595859B01D8
:104A8000281B390B37FF03C031952195310923339A
:104A900031053CF1DF0150974D915C91598348837A
:104AA0009A01261B370BB90137FF02C0615C7F4FAB
:104AB00016E0759567951A95E1F7261B370B3F872A
:104AC0002E87841B950B9C0197FF02C0215C3F4FF2
:104AD000B6E035952795BA95E1F7821B930B9D8F2C
:104AE0008C8F229687E0EC3EF80729F60E94BF5192
:104AF000909328058093270569E17BE080E10E947F
:104B00004C594CE651E168E182E10E945259DF9133
:104B1000CF911F910F91FF90EF90DF900C946E2436
:104B2000FF920F931F93CF93DF93182F062FEA0165
:104B3000F22E222321F061E00E947512182FBE018F
:104B4000802F0E944C592F2D412F602F86E60E9406
:104B5000221F812FDF91CF911F910F91FF90089518
:104B6000CF93C1E09C2F981B892F0E949025C81BD2
:104B70008C2FCF910895FF920F931F93CF93DF93C4
:104B8000182F062FEA01F22E222321F061E00E9465
:104B90006D12182FBE01802F0E944C592F2D412FCE
:104BA000602F86E60E94221F812FDF91CF911F91F7
:104BB0000F91FF9008951F93CF93DF93D62F122F5D
:104BC0000E94BB25C82F212F482F6D2F86E60E94FB
:104BD000301F8C2FDF91CF911F910895AF92CF920C
:104BE000EF92FF920F93CF93DF93C82F81ED9BE05D
:104BF0000E941D1E96E0A92EC12C20EDE22E2BE076
:104C0000F22E0BE02EEB31E141E06C2F8AE098E0D0
:104C10000E943C1FC0910A08D091E901D295D69517
:104C2000D77065EC7BE088E00E944C59C13089F474
:104C300064E08D2F0E946D12D82F982F9295990FB6
:104C4000907E8091E9018F71892B8093E90101E0C9
:104C500001C000E02D2F45EA5BE068E084E50E949A
:104C600018596AE97BE080E10E944C59C23049F44E
:104C700064E28091EA010E946D128093EA0121E0D2
:104C800001C020E04091EA0160E184E50E948D0FBF
:104C90006FE87BE088E10E944C59C33049F464E638
:104CA0008091EB010E946D128093EB0121E401C021
:104CB00020E44091EB0150E068E184E50E94435B11
:104CC00021E0C43009F020E08091E90141E85BE097
:104CD00060E282FB882780F90E94DB259091E90140
:104CE00080FB92F99093E90121E0C53009F020E0C2
:104CF0008091E90143E75BE068E283FB882780F964
:104D00000E94DB259091E90180FB93F99093E901E2
:104D100021E0C63009F020E08091E90145E65BE042
:104D200060E3829581700E94DB259091E90180FB10
:104D300094F99093E901DF91CF910F91FF90EF905B
:104D4000CF90AF900895CF93482FCAE02AE0829F7A
:104D5000C001112483519E4F2FE130E0241B310903
:104D6000C29FA001C39F500D1124BC01665F7F4FFD
:104D70000E94306AE3E2F3E0DF011D92CA95E9F791
:104D800082E00E94C152CF910C9452530F93CF9363
:104D9000C42F0E94D00F002339F046E16AEE8C2F19
:104DA000CF910F910C946A128C2FCF910F9108958F
:104DB0000F931F93CF93DF93D82F162FC42F022F5B
:104DC00047FF08C041E28AEF8D0F0E94645886E0D9
:104DD0008C1BC82F2C2F45E75FE0612F8D2F0E9481
:104DE0001859DF91CF911F910F9108950F931F9341
:104DF000CF93DF93182F062F0E940A0FEC01111199
:104E000008C001110FC08881882379F181508883FF
:104E10002CC0113288F5103219F4002329F02CC06F
:104E2000002311F01F5F01C01150812F0E940A0F53
:104E3000FC0198818FEF890F8031F0F420812131BE
:104E4000D8F4291302C08BE007C0002301F390318E
:104E500060F49F5F988309C0815029F09081288178
:104E600021939993F9CF10931D0882E0DF91CF91A0
:104E70001F910F910C94C152DF91CF911F910F910F
:104E8000089580912303882329F08DEE9BE10E94F1
:104E9000DC1981E00895BC0188E00E944C596EE85D
:104EA0007EE088E20E944C596FE77EE080E30C943C
:104EB0004C59CF93C82F813669F08F3B39F080363B
:104EC00099F4809157070E94A32604C080E00E94B5
:104ED000D8660AC08C2F0E941B5D81E00E94C41915
:104EE00089E191E40E94DC1983E79EE0CF910C9464
:104EF0004B270F93CF93C82F4FE060ED77E0809161
:104F000053070E94355200E12AE040ED57E060E18E
:104F100081E00E94F6584FE360E182E40E94F3587A
:104F200080915407882319F084E19EE002C087E055
:104F30009EE00E944B27C13651F1CF3B19F0C0369D
:104F400091F505C080E0CF910F910C94D8668091C7
:104F500054078823A9F085EF9DE00E9422118091DB
:104F600053070E946C52882339F087E10E94D8666B
:104F700082E08093540709C080E00E94D86605C093
:104F8000809153078F5F0E949C5580E601C081E6A7
:104F90000E941B5D81E00E94C41983E19DE2CF91D4
:104FA0000F910C94DC19CF910F9108959091BC0151
:104FB00081E0191624F0911101C080E081951092D2
:104FC000BC010895CF93C82F0E94D6279091560711
:104FD0002091B3012136E1F028F4203249F02E323D
:104FE00039F008C0233671F038F02E3889F002C04D
:104FF00081E00FC0181624F49C1730F49F5F04C0A2
:10500000882311F0911191509093560780E001C0D0
:1050100082E0CF9108950F931F93CF93DF93EC011C
:10502000062F000F000F000F18E0011788F069E647
:105030007EE0812F0E944C59AE01612F88E10E94D1
:105040005259FE01849121968111FBCF185FEDCF5B
:105050002AEF210F40E367E082E1DF91CF911F91BA
:105060000F910C94555BCF92DF92EF92FF92CF930A
:10507000DF93FC01EB019C01DC010E945F699B0155
:10508000AC01DE010E947569272F382F492F552763
:10509000DF010E9475696B017C014CE0F694E79496
:1050A000D794C7944A95D1F724E630E02C1B3D0BEA
:1050B0000E945F696E5C7F4F8F4F9F4F6C0D7D1D0F
:1050C0008E1D9F1D24E630E040E050E00E94CE6936
:1050D000C901DF91CF91FF90EF90DF90CF900895BD
:1050E0001F93CF93DF936115710529F1192F111FBC
:1050F0001127111F19F091958195910977FF10C023
:10510000719561957109C0E0D4E09E01281B390BAF
:10511000C9010E9433289E01281B390BC90102C016
:105120000E943328112329F022273327281B390B0B
:1051300001C09C01C901DF91CF911F910895EF92A9
:105140000F93CF93DF93962F642F322F402F882316
:10515000E1F121E001E0C0911B088EE0C89FE00171
:105160001124C358DC4F333631F44C85892F0E940B
:10517000C6268C8734C0323631F44D85892F0E9483
:10518000C6268D872CC0E42FF0E0E30FF11DE30F5E
:10519000F11DEE0FFF1FEE0DF11DEC0FFD1FEF01D6
:1051A000411108C0E22E04E62CE94881892F0E94B3
:1051B0007B1D09C048814C59E22E04E620E0892F6E
:1051C0000E947B1D845688830AC001E0E0913F0164
:1051D000F0914001EF2B09F400E020E0BCCFDF911B
:1051E000CF910F91EF9008952F923F924F925F923F
:1051F0006F927F928F929F92AF92BF92CF92DF92E7
:10520000EF92FF920F931F93CF93DF9300D000D0C4
:105210001F92CDB7DEB7182F86E59EE00E941D1EB7
:10522000B5E0AB2EC12C05E5E02E0EE0F02E0BE034
:105230002EEB31E143E0612F8FE098E00E943C1FAC
:10524000F0900F08F1101092550100911B0821E019
:10525000F2120BC020E043E060E0802F0E945E125B
:10526000082F80931B0821E001C020E041E0400F9F
:1052700068E080E00E948D0F802F0E94D51DD82EFF
:1052800031E0831731F082E0D81206C065E47EE099
:1052900005C06DE47EE002C06EE37EE088E00E941F
:1052A0004C59E02FF0E0EE0FFF1FEE55F84F408114
:1052B0005181453651052CF44C395F4F24F012E0F2
:1052C00003C010E001C011E0802F0E94251581115C
:1052D00010E068E37EE080E10E944C59112319F050
:1052E00081E0E2E0FE1280E0EE24E39400E02D2D68
:1052F00048E168E10E949F28113019F081E0F2E056
:10530000FF1280E0E12C00E02D2D48E160E30E94D7
:105310009F2860E37EE080E20E944C59112319F03F
:1053200081E023E0F21280E0EE24E39401E02D2DF1
:1053300048E268E10E949F28113019F081E033E0D3
:10534000F31280E0E12C01E02D2D48E260E30E94A1
:105350009F286AE27EE080E30E944C5981E094E05D
:10536000F91280E0E12C00E023E640E36EE10E94C8
:105370009F2864E27EE088E30E944C5981E0E5E0EA
:10538000FE1280E0E12C00E022E648E36EE10E949C
:105390009F2840911B08FEE04F9FA001112424E0AC
:1053A000D29E400D511D11244D525E4FFA01E6551B
:1053B000FE4FDA01A555BE4F1C91DA01A455BE4F30
:1053C000FC9034E6F30EDA01A355BE4F0C910C5954
:1053D00080810E942115682E812F0E942115782E30
:1053E00044E660E08F2D0E940B15982E44E660E0A5
:1053F000802F0E940B15882E80911B080E94251576
:10540000E62DFF27E7FDF095FD83EC83092D11279D
:1054100007FD1095882309F45DC0C12CD12C7601BD
:10542000B12C61E2262E312C74E6472E512C6C8172
:105430007D81D701C601B595A795979587950E945F
:105440007028880F991FB1010E94BA69609FC0013E
:10545000619F900D709F900D11245FE3A52EAB0C02
:10546000B2010E94A669F0E4F61B6F2F8A2D0E94FC
:1054700097598B2D8370B394811108C06FE38A2DE7
:105480000E9497596B2D8FE30E94975921E2C20E1B
:10549000D11CE11CF11C3EE3B312C9CFE0911B0803
:1054A000F0E0EE0FFF1FEE55F84F00811181C801AB
:1054B00061E270E00E94BA69862F4EE361E0825A91
:1054C0000E94E75980911B080E942515882309F442
:1054D0009CC069C0E12CF12C512C81E2C82ED12C4A
:1054E00094E6A92EB12C872D992787FD90959B8353
:1054F0008A83282C332427FC30946C817D81C7015A
:105500000E947028B6010E94BA69609FC001619F25
:10551000900D709F900D1124BEE54B2E450CB501EA
:105520000E94A66990E2961B692F842D0E949759CC
:10553000E52DE370E983E11109C060E2842D0E944A
:10554000975960E2650D8EE50E9497596A817B81CB
:10555000C7010E947028B6010E94BA69629DC0010D
:10556000639D900D729D900D1124AEE54A2E451855
:10557000B5010E94A669605E842D0E949759F98149
:10558000F11109C060E2842D0E94975960E265190B
:105590008EE50E949759539421E2E20EF11C3FE1FF
:1055A0005312ABCF7BCFC8019C5F97FD01966C81F6
:1055B0007D81959587950E9470289C01220F331F4D
:1055C000A92D97FCAD5FA595A595BB27A7FDB09527
:1055D0000E94576929E130E040E050E00E94F06904
:1055E00069017A01C90161E270E00E94BA6980E450
:1055F000861B4EE3682F8FE30E94E459C601D7FC57
:1056000001967C01F594E7942EC0101611060CF457
:10561000762C672D772767FD7095C8010E9470284A
:105620001016110614F4A92D01C0A82DA7FDAD5F19
:10563000A595A5959C01BB27A7FDB0950E9457692C
:1056400029E130E040E050E00E94F0697901C901B1
:1056500061E270E00E94BA6980E2861B4EE3682F27
:105660008FE30E94E45989E1809FA001819F500D42
:10567000112457FF02C041505F4F852F880F880BC0
:10568000452F582F60E382E70E94525B89E18E9D8F
:10569000A0018F9D500D112457FF02C041505F4F54
:1056A000852F880F880B452F582F68E084E50F90D1
:1056B0000F900F900F900F90DF91CF911F910F914E
:1056C000FF90EF90DF90CF90BF90AF909F908F9022
:1056D0007F906F905F904F903F902F900C94525B13
:1056E00090E0E92FF0E0E057FD4EE491E81721F05B
:1056F000EE2321F09F5FF5CF892F089580E0089574
:10570000823430F4E82FF0E0E057FD4E84910895A4
:1057100080E20895FF920F931F93CF93DF93C82FDA
:10572000D62FF42E122F622F842F0E942711FC01F6
:10573000E53F81E0F80794F09BE09E0F9F1510F085
:105740009CE09E0F40E3490F202F6D2F8C2FDF919F
:10575000CF911F910F91FF900C946458212F48E036
:105760005CE06D2F8C2F0E941859DF91CF911F9113
:105770000F91FF900895BF92CF92DF92EF92FF9228
:105780000F931F93CF93DF93C82F8BEE9BE00E9464
:105790001D1E24E0E22E0BE02EEB31E142E06C2FE7
:1057A0008BE098E00E94B321D0900B08C03611F036
:1057B000CE3669F4DD2059F08FEF8D0D80932008EF
:1057C0008C2F0E941B5D82E49CE20E94DC1966EE35
:1057D0007BE080E10E944C59DAE5C0E000E02C2F2C
:1057E00040EE5BE060E18D2F0E941859CF5FDA5FD9
:1057F000C430A1F7C3EDD1E098E1F92E11E0BB244C
:10580000B3941D11B12C6CED7BE08F2D0E944C598F
:1058100040E3410F6F2D82E10E94F3582B2DFE01D2
:10582000E353FD4F40816F2D8AE20E94D00F8AE53D
:10583000C82EE12C0B2D2E2D412F6F2D8C2D0E946B
:105840008A2BE39486E0C80E84E0E812F3CF1F5F52
:1058500088E0F80E2A96153091F60E94F319682F09
:10586000660F660F660F615F29E04AE180E0DF9115
:10587000CF911F910F91FF90EF90DF90CF90BF904D
:105880000C94555B8F929F92AF92BF92CF92DF9212
:10589000EF92FF920F931F93CF93DF93C82F8090C7
:1058A00020082AE0829E40011124C40188569B4FA3
:1058B0004C0180E09CE00E941D1EAA24A394CC24ED
:1058C000C3945EEFE52E5BE0F52E00E020E030E0D3
:1058D00040E06C2F8CE098E00E943C1F4091200833
:1058E0004F5C60E080E30E94F358B0900C0868E0E1
:1058F000F62ED12CBD1007C080918007882329F097
:1059000042E0E42E04C0E12C02C0EE24E394D11066
:1059100010C067EF7BE08F2D0E944C590E2D2E2D6D
:10592000F40140856F2D80E30E94C626F401808734
:105930004DC061EF7BE08F2D0E944C5930E3C32EA8
:1059400010E080915A07811711F000E001C00E2D80
:10595000409120084F5F212F6F2D8C2D0E948A2BA4
:10596000EE2071F180915A0781132AC080917F0740
:10597000882331F1E401C10FD11DC10FD11DE88190
:10598000F981CF018B509E4F843FF1E09F0714F4C3
:1059900084EF91E022E048EF51E064EF71E00E9473
:1059A000B311AC0180914701882351F0443F21E0BD
:1059B000520711F440E050E0455F5140598348835D
:1059C0001F5F86E0C80E143009F0BBCFD39498E077
:1059D000F90EE2E0DE128ECFDF91CF911F910F9191
:1059E000FF90EF90DF90CF90BF90AF909F908F90FF
:1059F0000895CF93C62F0E941B5D0E945253C093FF
:105A000029058C2F0E9462538091DD010E94AE1205
:105A100082E080930D0181E00E94C1520E945253A6
:105A200081E0CF9108958F929F92AF92BF92CF92D3
:105A3000DF92EF92FF920F931F93CF93DF93182F74
:105A40008CE59BE00E941D1EF09009088091520792
:105A5000811109C081E08093B4074FE0612F89E094
:105A600098E00E94C42166E57BE080E00E944C59EA
:105A70000E94BF54AC0160E086E60E94525BB09089
:105A8000090880915407823021F41092080810927E
:105A90005407CB2DDD27C7FDD095809181079E014E
:105AA000281B3109C901181619066CF09E012150F6
:105AB000310937FF02C020E030E020938107E0E1A8
:105AC000AE2E812C3EC025303105CCF39E012450F2
:105AD00031092B3031058CF32AE030E0EECF00E1C4
:105AE00096012F5F3F4F442737FD4095542F72E0BA
:105AF000E72E6A2D82E10E94335A8091290598127F
:105B000005C04AE26A2D81E00E94F3584FE060ED43
:105B100077E0892D0E943552CC15DD05E1F48091A6
:105B200008088823C1F001E12FE040ED57E06A2D1D
:105B300088E10E94F658839438E0A30E86E0881628
:105B400061F090908107980CC92CD12CCC15DD0503
:105B500031F601E1C5CF00E1E7CF809152078823FC
:105B600009F453C09091290580910908981302C047
:105B700003E001C004E0602F8DE791E10E940B2853
:105B80008FEF800F0E94E227D82E00915607602FDA
:105B9000660F660F660F685F20E044E288E10E94AE
:105BA0007A5921E0D21228C0011110C06091090871
:105BB00060932905812F0E94F92C80915207823031
:105BC00009F581EC94E40E9484121CC0033031F486
:105BD000812F0E941B5D1092540704C0013049F4CC
:105BE00000935407B092530789E797E20E94DC19AB
:105BF00009C0D092080806C032E0D31256C0812FE7
:105C00000E941B5D1092520750C0163638F41436AD
:105C1000A0F4103649F1113649F047C01138B1F1FE
:105C20001F3BC1F11E3609F040C01EC0809108081C
:105C30008823D9F11092080838C0909129058091E5
:105C40000908981749F0812F0E941B5D1092560792
:105C500082E08093520729C01092B407153609F0EC
:105C600051C08CE792E250C080910808882319F057
:105C70001092080808C0812F0E941B5D10925607E1
:105C800081E080935207109280070FC081E00E944C
:105C9000C4190BC010920808109252078091290570
:105CA0008093090881E00E94C552809108088823EA
:105CB00071F1FB1461F161E06B0D81E08F0D0E94C9
:105CC0007A558091290590E0C817D90719F4F09208
:105CD000290509C02F2D332727FD309528173907AF
:105CE000B1F4B092290581E0DF91CF911F910F911E
:105CF000FF90EF90DF90CF90BF90AF909F908F90EC
:105D00000C94C15281EC94E40E948412CECFDF91B6
:105D1000CF911F910F91FF90EF90DF90CF90BF90A8
:105D2000AF909F908F90089521E0411101C020E035
:105D3000405D0C946458EF920F931F93CF93DF93C1
:105D4000C82F8CE09BE00E941D1EE12C06E022EB98
:105D500031E143E06C2F85E098E00E94B321D0E070
:105D6000C0E0C43018F018EF1D0F01C01D2F8FE0E8
:105D70008C0F0E94CC5C082FCF5F20E04C2F612F4E
:105D80008AE20E94D00F402F612F84E40E94942E5B
:105D9000D85FC93031F7D8E3C0E08C2F0E94CC5CCB
:105DA000182F00E02C2F4CEE5AE06D2F80E00E945F
:105DB0001859412F6D2F80E20E94942ECF5FD8504A
:105DC000C63059F744EE5AE068E184E50E94525922
:105DD00016E0C0E2D0E02D2F44ED51E16C2F84E5B8
:105DE0000E941F58812F0E94CC5C482F6C2F8CE69C
:105DF0000E94942E81E0810F0E94CC5C482F6C2F72
:105E000088E70E94942EDF5FC85F1E5FD43019F7C9
:105E1000DF91CF911F910F91EF900895CF92DF9274
:105E2000EF92FF920F931F93CF93DF93D82E109191
:105E3000DE01F12EF7FCF194C5EBD7E0E0904E04C3
:105E40001A339CF0E12FEE0FFF0BE951F94F20813F
:105E500031813C5F37FF02C0215C3F4FA6E03595A2
:105E60002795AA95E1F7D22E2DC024E22F1550F5E3
:105E70002D853E854F855889242B352B4B855C8598
:105E8000242B352B8989282B8A89282B232B29F42D
:105E9000812F881F8827881F8A8B111614F48CED98
:105EA00001C084E2810F40E060E00E944A1588232F
:105EB00041F09A89911105C091E02989211190E062
:105EC000998B8A8BEE2039F040E060E08E2D0E94A5
:105ED0004A15882311F001E002C000E0D12C4D8565
:105EE0005E854F5F5F4F5E874D874F8558894D0DAB
:105EF000511D588B4F87F8942091830C3091840C5E
:105F000078948B859C85281B390B2436310508F441
:105F100025C18C599F4F9C878B872F853889ED85AC
:105F2000FE85C901BF010E94A669D62EC62E6E9FAE
:105F3000C0016F9F900D1124281B390B388B2F87C0
:105F40001E861D863FE03F1510F0198A0EC084E2C0
:105F50008F1558F0111614F481EF01C08FE0810FF6
:105F600040E060E00E944A15898B88819981019602
:105F7000998388834A815B814F5F5F4F5B834A834C
:105F8000CC2031F02E813F812F5F3F4F3F832E8306
:105F900021E0F21201C0F98A8989882341F00023A7
:105FA00031F02C813D812F5F3F4F3D832C83D69470
:105FB000288539852D0D311D398728870091E0010D
:105FC0001091E1011C8B0B8BF11002C01A8625C0C9
:105FD00081E0F81206C0E11018C0C801841B950BBF
:105FE0001AC08FE08F1528F0F0FC06C02E813F818B
:105FF00008C089E38F1548F4F4E036952795FA95A3
:10600000E1F7C801821B930B06C08C819D8198012A
:10601000281B390BC9019C8B8B8B8A85EB88FC88EC
:10602000813049F018F0823069F018C08091DE01AB
:106030008823A1F011C0F7FE11C00115110571F000
:1060400082E00BC035ECE3163FEFF30614F483E077
:106050008A870115110511F481E08A87898D9A8D4F
:106060008E159F0509F46EC08A85813009F05BC0EA
:106070008091420582FF35C00115110591F18EE135
:10608000E816F10419F469E289E10DC024E1E21691
:10609000F10419F46AE28AE106C03AE0E316F10479
:1060A00031F46BE28BE10E94DE6681E00EC086E097
:1060B000E816F1044CF4F7FC03C06E2D8CE1F3CF2D
:1060C0008CE10E94D866F1CF80E09091420593FF69
:1060D00008C0882331F082E390E090933A018093E6
:1060E00039018091DF0180FF04C0C8018E199F092A
:1060F00001C0C7016CE370E00E94BA69DC01CB010A
:106100004091420541FF1EC0AB2BE1F440914B058D
:1061100041FF07C0009761F046E260E00E94E76639
:1061200007C080E003C0823069F48CE10E94D86629
:106130008091420583FF06C082E390E090933A018C
:10614000809339018B899C899A8F898F2091DF01F7
:1061500020FF04C0081B190B1C8B0B8BDF91CF9108
:106160001F910F91FF90EF90DF90CF900895CF9304
:10617000DF938091DE01E82FE7FDE1959EEF9E0F12
:106180009E30B0F4E595EE0FFF0BE056F84F2081FE
:10619000318187FF05C080E094E0821B930B02C031
:1061A000C9019C5FC6E096958795CA95E1F702C044
:1061B00080E090E00E940E2F8091A6079091A707A3
:1061C0009C5FB6E096958795BA95E1F72091DF013F
:1061D00022FF0AC08530910538F02091CC072111AB
:1061E00003C023E02093CC07CCEFD7E0288139818E
:1061F0002F5F3F4F398328832A813B81280F391F26
:106200003B832A83F8948091830C9091840C78943A
:106210002C813D81AC01421B530B9A01283E334037
:1062200090F19D838C838091E2018F70823039F4EC
:1062300040E060E085E10E944A15811120C08A811A
:106240009B81688179810E94A6691B821A821982CA
:1062500018828091D806893718F48F5F8093D8060A
:10626000E091D90681E08E0F8093D906F0E0E652E6
:10627000F94F6083883738F01092D90604C087E060
:106280000E94D866DCCFDF91CF910895E5EBF7E06F
:106290001286138212821782168215821482118648
:1062A00010868091E0019091E101928F818F089595
:1062B000EF92FF920F931F93CF93DF93C62FD3E0FC
:1062C000ED2EE60E1AE5819F102D1124165FD0E207
:1062D000CE1598F4FF24F394FC0E40E060E08F2D7F
:1062E0000E944A15082F2C2F4FE553E06D2F812F68
:1062F0000E941859D85FCF2DEBCFDF91CF911F911E
:106300000F91FF90EF900895CF92DF92EF92FF925E
:10631000CF93DF936B017C01C0E1D0E040E050E817
:10632000E0E0F0E89A01DA010E945F69C616D7063C
:10633000E806F90610F44E275F27F695E7952197B2
:10634000209719F04E2B5F2BEDCFCA01DF91CF9133
:10635000FF90EF90DF90CF9008951F9341E0262F9C
:1063600030E0683050F440E055E0529FF001539F18
:10637000F00D1124E754FC4F0AC02850310959E0B0
:10638000529FF001539FF00D1124EF51FC4F9C5F81
:1063900097FD0DC0811528E0920784F0442319F081
:1063A00088E090E002C084E090E0E80FF91F2081CF
:1063B000332727FD3095322F222725C0442329F08B
:1063C000492F9927880F991F03C0492F469591702F
:1063D000242F30E0E20FF31F608140E052E0481BC1
:1063E000590B5595479564039001659F300D112415
:1063F0001181BC01759567951603A001179F500D7B
:106400001124240F351FC90169E170E00E94BA69A7
:10641000CB011F9108956F927F928F929F92AF92BE
:10642000BF92CF92DF92EF92FF920F931F93CF9381
:10643000DF93982EDD24D39480911F08883008F4D0
:10644000D12C8BE591E10E941D1EDD2011F089E029
:1064500001C085E0A82EC12CBAE5EB2EB1E1FB2EE0
:1064600000E020E030E040E0692D89E198E00E9402
:106470003C1F2FEB921202C01092180840911F0887
:1064800050E04F5F5F4F21E060E084E20E94435B99
:10649000C0911F08DD2061F08C2F90E0089729E063
:1064A000289FE001299FD00D1124CF51DC4F06C059
:1064B00045E0C49FE0011124C754DC4F60901908E7
:1064C0006A94CC2E7D2EAC2EBD2E05E010E0A0E10E
:1064D0008A2EE62CFF24E7FCF094F50141915F0140
:1064E00021E0C8010597E816F90609F020E05527D4
:1064F00047FD5095682D88E10E94435BDD2091F0B7
:10650000093081F021E0E016F10609F020E0FE01FB
:10651000E00FF11F4081552747FD5095682D80E31E
:106520000E94435BF8E08F0E0F5F1F4F28E382123B
:10653000D4CF11E04FEF641210E0212F43E551E179
:1065400068E08CE00E942C59112309F446C0909217
:10655000B30120E044E06CEF809118080E945E12C5
:106560008093180890914701992399F1DD2021F03B
:1065700090E164E049E003C098E062E045E054E661
:1065800085028001112470E0719561957109582F81
:1065900056039001579F300D112484E6829F4001DD
:1065A000839F900C1124EC2DF72D20E030E0A92ED4
:1065B000B12CC901880D991DB5010E94BA6961937A
:1065C000200F311F8E2F8C19841798F382E00E94C0
:1065D000C152C12C0CE91FEF34C044E66CE98E01B6
:1065E0000E0D1F1DF80180810E946A12F801808340
:1065F000F0CF85E090E02817390794F5C901F5E060
:10660000880F991FFA95E1F7DD2011F164E070E041
:106610000E94BA69B62EFE01E20FF31F8081F0E2FC
:106620008F02C0011124B8010E94BA69E216F30674
:1066300091F4625E25E045E08AE38B0D0E94555B94
:10664000C3942C2D30E0DD20A1F289E090E0D3CF7F
:1066500062E070E0DDCF615E23E043E08BE3EDCFED
:10666000C0E0DCEF10E0E0E2FE2E60911F08CE01FA
:106670000E94AD310CE3010F75E0969587957A95F0
:10668000E1F76F2D681B802F0E949759812F83702F
:1066900021F460E2802F0E9497591F5FA09610346A
:1066A00021F740E460E08CE5DF91CF911F910F91DD
:1066B000FF90EF90DF90CF90BF90AF909F908F9022
:1066C0007F906F900C94E7592F923F924F925F9278
:1066D0006F927F928F929F92AF92BF92CF92DF92F2
:1066E000EF92FF920F931F93CF93DF93CDB7DEB757
:1066F0006C970FB6F894DEBF0FBECDBF8B8F9C8F0B
:10670000162F80913B01882309F447C0E1E9EE2E62
:10671000E6E0FE2ED7017D0180917E07882319F0E7
:10672000815080937E070E94A213F7012381348158
:106730008217930741F0948383831282118281E050
:10674000809338012AC060914105665F31F18091E4
:106750003C01823310F1D70180818F5F80838031CB
:10676000E0F0F701818192810196928381831C92EE
:1067700047E751E0649F9001659F300D1124281771
:10678000390758F48F719927019739F486E00E94F0
:10679000B6126DE280E10E94DE660E94F3198093DA
:1067A0007705E091EB01E11103C0212C312C26C0CB
:1067B000A091A407B091A5074091A8075091A907FF
:1067C0009D010E9457696B017C019A01DA010E94C8
:1067D0005769C60ED71EE81EF91E8E2F0E9435156A
:1067E0009C01DC010E9457696C157D058E059F0593
:1067F000E0F6C701B6010E9484311C01809140057A
:10680000880F880F6DEFA62E64E0B62E9E012F5FD5
:106810003F4F3A87298740E556E05E874D87E12C58
:10682000F12C512C682F70E07A8B698B695B7C4F5F
:106830007D8B6C8B712F71707E8B7EE0472EC1013A
:10684000A0E0B0E08F8B988FA98FBA8F12701B8B4E
:106850006E2C8E2D0E949213D5011296BC87AB87A9
:10686000F50120813181821B930B9C01BC0188279B
:1068700077FD8095982F5AE0660F771F881F991F24
:106880005A95D1F71216130624F4FD01228D338D8B
:1068900004C0EB85FC85248535852436310514F448
:1068A00024E630E0442737FD4095542F0E94F069DC
:1068B00089012130FCEF3F073CF0011524E012076D
:1068C0002CF000E014E002C000E01CEF80914205D3
:1068D00080FF11C08091400581708F87188A82E007
:1068E00090E04F855889841B950BE816F90619F43A
:1068F00011950195110953E0561580F0C80144E047
:10690000959587954A95E1F7F701E055F84F808313
:10691000EC89FD89EE0DFF1D749001C0762CC72C0B
:10692000D12CF601EE0FFF1FEE55F84F11830083B7
:10693000C80117FD0F9624E0959587952A95E1F7F4
:10694000282F87FD219522307CF481E090E00C2CEB
:1069500001C0880F0A94EAF7211102C0982F03C0E2
:10696000909190069823592A63E0661508F4FAC0BE
:106970007E8971115AC08091DF0181FF56C04501A7
:1069800089E3880E911CF4018181807C09F44DC05B
:10699000F50181AD40E061E08595859585950E9482
:1069A0004A15882309F441C08091BD01882309F468
:1069B0003CC0D4018C918770E989FA89E80FF11DF8
:1069C000E95BFC4FE491F0E0DF01AA0FBB1FA85D7B
:1069D000BE4FEE0FFF1FE25DFA4F8D919C9120811B
:1069E0003181821B930B97FD0196AC01559547951C
:1069F000F4012181322F330F330F35953595340350
:106A0000C001359F900D11246FE170E00E94BA69BA
:106A1000660F771F660F771F2295269526952370A0
:106A2000213009F059C6060F171F2114310499F0BF
:106A3000872D8D7F813079F48091EB010E9435158F
:106A40009801DC010E9457692F89388D498D5A8D34
:106A50000E94F0698901872D0E94D51DA82E872DDF
:106A60000E942515B12C882311F1F501EE0FFF1FAF
:106A7000EE0FFF1F4C9CC0014D9C900D1124E80FA0
:106A8000F91FE358FC4F80810E942115682F77275A
:106A900067FD7095C8019C5F97FD01969595879558
:106AA0000E9470288C01000F111F912C24C081E0DE
:106AB000101611060CF480E0982E4C9CC0014D9CE1
:106AC000900D11249501220F331F220F331F820FC7
:106AD000931F8D529E4F890D911DFC01E655FE4F6F
:106AE00080810E942115682F772767FD7095C80166
:106AF0000E9470288C01C501880F991F880F991F6B
:106B00004C9C90014D9C300D1124820F931F8D528F
:106B10009E4F890D911DFC01E455FE4F808144E696
:106B200060E08C590E940B159801A82FBB27A7FD88
:106B3000B0950E94576924E630E040E050E00E94A2
:106B4000F0698901872D0E94251581111450662D49
:106B5000809177050E946D11880F991FA985BA85CC
:106B60008D939C93CC0CDD1CF601E85CF94F6F0112
:106B700011830083FB89FF23C1F023E02615A8F0D1
:106B8000872D0E942F1581110CC0065F1F4F053104
:106B9000110518F0D6011D921C92E985FA85118223
:106BA0001082AD85BE851D921C92BFEFEB1AFB0AC9
:106BB000ED85FE853296FE87ED8729853A852E5F25
:106BC0003F4F3A87298737E0E316F10419F0AB8489
:106BD000BC843ECE8091E40180FF25C062E08091BC
:106BE00077050E946D11282F8091420580FD219527
:106BF000332727FD3095432F532F23583F4F4F4FB7
:106C00005F4FA0E0B4E080913C0690913D06A81B48
:106C1000B90B0E94806920E034E040E050E00E941F
:106C2000F0693E832D831091E80115218091900633
:106C30008095812319F088E10E94D8661093900610
:106C400080E094E09093470680934606909349062F
:106C50008093480682E10E94CC5C811108C083E1E8
:106C60000E94CC5C882331F080E090E005C080E099
:106C70009CEF02C080E094E09093810680938006B0
:106C800028E231E0EEE2F5E000E516E060E0D9014F
:106C90008D919D919D01643020F440815181841B30
:106CA000950B880F991FD8018D939D938D016F5F70
:106CB0003296683061F720E636E0E6E9F6E0419189
:106CC000519161917191D9014D935D939D01B6E010
:106CD000E63DFB07A1F7EAE8F4E0A2E8B6E0808130
:106CE00028E08202C00111248D939D93329634E0F6
:106CF000E839F307A1F7E091EB01EE2309F447C06F
:106D0000A0913A06B0913B0640913E0650913F0655
:106D10009D010E9457696B017C019A01DA010E9472
:106D20005769C60ED71EE81EF91E8E2F0E94351514
:106D30008C019C01DC010E9457696C157D058E0554
:106D40009F0528F5C701B6010E94843120913A06BB
:106D500030913B066C01E12CF12CD8010E9457695F
:106D6000A70196010E94F06930933B0620933A06F2
:106D700020913E0630913F06D8010E945769A70135
:106D800096010E94F06930933F0620933E06609181
:106D9000E901862F807E09F4D2C04B89411111C0D0
:106DA00020913A0630913B068B819C81280F391F38
:106DB00080913E0690913F064F815885840F951F24
:106DC00004C080E090E020E030E0E8E3F6E04091AD
:106DD000EA01442349F0DF01A40FB11DA40FB11D46
:106DE00012974D915C9102C040E050E062FF03C0F9
:106DF00031952195310963FF03C0919581959109E2
:106E000064FF03C05195419551096295669567707D
:106E1000623009F44AC018F46130B1F090C06330B8
:106E200009F47DC0643009F08AC0BA01621B730B9B
:106E3000738B628B9A01280F391F358B248B481B6B
:106E4000590B578B468B7BC0BC0197FF02C0695F13
:106E50007F4FA3E075956795AA95E1F7DC01A61B26
:106E6000B70BBC0197FF02C061587F4F660F672FB9
:106E7000661F770BA61BB70B97FF02C081509C4F74
:106E8000BC01672F770F770B65956595CD01861B44
:106E9000970BBA01621B730B738B628B37FF02C0B7
:106EA0002F5F3F4F359527953FC0B90137FF02C08F
:106EB000695F7F4FA3E075956795AA95E1F7D901C2
:106EC000A61BB70BB90137FF02C061587F4F660F91
:106ED000672F661F770BA61BB70B37FF02C0215029
:106EE0003C4FB901672F770F770B659565959D012D
:106EF000261B370BBA01681B790B738B628B97FDCE
:106F0000019695958795840F951FAC01420F531FED
:106F1000558B448B821B930B978B868B10C0BA01C9
:106F2000621B730B738B628B240F351FA901480FF3
:106F3000591F558B448B281B390B378B268B80911F
:106F40003B0181110E94B73080E4E6E9F6E0DF0101
:106F50001D928A95E9F785EB93E090930301809366
:106F6000020186EB93E0909305018093040187EB87
:106F700093E0909307018093060188EB93E0909350
:106F8000090180930801E8EBF5E0FC87EB8728E72F
:106F900035E0388B2F8748E156E05E874D87312CEE
:106FA000212C832D0E940A0F7C01FC0182810E940A
:106FB00021158987D7018C918150803108F072C2E8
:106FC000ED85FE85D08040E061E0F70183810E947D
:106FD0004A15F70193812181992341F094EF920F93
:106FE000983020F49091BD01992311F0811112C0C5
:106FF00088EF820F823008F03FC2F70187818670E8
:10700000843009F439C280E0293009F03EC000E044
:107010001CEF3FC081E0D11080E0D82E8FEF820FAF
:10702000A82FB0E0FD01EE0FFF1FE85CF94F0081D3
:107030001181843150F0831540F4AA0FBB1FAA0FB1
:10704000BB1FAA56B94F0D911C91F7013781832FB1
:10705000807361F0832F82958370815041E050E00E
:1070600002C0440F551F8A95E2F7242A36FF10C04C
:10707000253070F4E22FF0E0EE0FFF1FE050FF4FDD
:10708000C70108969183808303C000E010E001C02F
:1070900081E0AD85BE858C93F7018781887459F4B2
:1070A0008085882341F04DE763E80E940B150E941C
:1070B0003515080F191FF701F681F98BF11105C07D
:1070C000F7018581882309F4EAC0AF85B889AD90BE
:1070D000BC90EB85FC8580819181A2819C014A2F27
:1070E000552747FD509529013A01D1100AC0BB2709
:1070F00057FDBA95A52F942F832F6801C81AD90A76
:107100003EC0F701878186708430D9F4E081F0E0D9
:10711000EE0FFF1FE25AF94FA081B18120E034E663
:107120000E946E692B013C01F985FF2351F02F2F3E
:10713000332727FD3095432F532F0E94F0692901F3
:107140003A01C301B20120E031E040E050E00E948A
:10715000F06950954095309521953F4F4F4F5F4FC7
:107160006801C20ED31EC114D10449F0F701858114
:10717000D7FE82958F70F4E68F9F50011124A114E1
:10718000B10491F080913B01882331F021E0A21AF3
:10719000B108A114B10441F0332777FC3A95272DAB
:1071A000162D052DC12CD12CAF85B889AD92BC927E
:1071B000C114D10409F46EC04801AA2497FCA0941C
:1071C000BA2CB989BB2309F461C080913B018823A3
:1071D000F1F1E985EE2379F02E2F27FD219530E09E
:1071E00040E050E060E070E080E293E00E94F069EF
:1071F000CA01B90104C060E070E080E293E0F701E9
:1072000026811C141D0444F090958095709561951D
:107210007F4F8F4F9F4F22952F7030E02115310502
:1072200091F0E4E6E29FA001E39F500D11249A0142
:10723000442737FD4095542F0E94F069420E531E9B
:10724000641E751E04C04424582C692C7A2CBB275C
:1072500077FCBA95A72D962D852D1C141D0434F4AA
:1072600088169906AA06BB0634F009C08815990548
:10727000AA05BB0524F44424582C692C7A2C332706
:1072800077FC3A95272D162D052D04C04424582C43
:10729000692C7A2CAB85BC854D925D926C92F7017E
:1072A000878187FF28C044E66CE984810E940B1522
:1072B000A82FBB27A7FDB0951A161B0644F417FF8D
:1072C0006AC024E630E02A1B3B0BD90109C01097A5
:1072D00009F461C0101611060CF05DC0AC59BF4F27
:1072E00098010E94576924E630E040E050E00E9497
:1072F000F069890150C0F7016481862F992787FDC5
:107300009095A92FB92F8730910590F5FC01EC5A83
:10731000FF4F0C940F6AF7018181893021F417FD2A
:1073200035C012500BC017FF36C01BC0F70181815A
:10733000893039F41016110664F11E5F000F111F19
:107340002AC0101611066CF026C017FF24C0119534
:107350000195110920C010161106DCF002C017FDBE
:1073600015C000E010E017C01016110694F00EC012
:1073700067FF06C0119501951109F6E0F61B6F2F06
:107380006750C8010E94AD318C0105C000E01CEFC0
:1073900002C000E014E0F701478140FD10C0818188
:1073A0009FEF980F943058F4FE013196E80FF11DCD
:1073B000E80FF11D329780819181080F191F980104
:1073C000F985AF2FBB27A7FDB0950E9457694B01E8
:1073D0005C014874483099F4F7018085882379F07E
:1073E0004DE763E80E940B150E94351524E630E056
:1073F000DC010E946E69860E971EA81EB91ED70179
:107400000C9110E001501109F70187818695837076
:10741000000F111F000F111F813071F0823029F110
:10742000F801EA56F94F80819181A281B381880EDB
:10743000991EAA1EBB1E19C0C501B40124E630E086
:1074400040E050E00E94F069F801EA56F94F60818F
:107450007181828193810E94886920E034E040E05C
:1074600050E00E94F06949015A01F801EA56F94FCB
:1074700080829182A282B38233942B853C852D5FDA
:107480003F4F3C872B874F8558894E5F5F4F588B06
:107490004F876D857E856F5F7F4F7E876D8770E23A
:1074A00037127FCD1091820C20FE05C0111103C050
:1074B0008EE10E94D86621FE07C0812F877F80342D
:1074C00019F48FE10E94D86622FE09C0812F877FC0
:1074D000803811F0103919F480E20E94D8668B8D43
:1074E00089879C8D9A8731E5232E34E0332EA2E8DC
:1074F000B7E0BE87AD87E6E9F6E0FC87EB87C12CF5
:10750000D12CCF868C2D0E94110F4C01FC01838160
:107510009481A0908304B12CA816B9063CF0B194D4
:10752000A194B108A816B9060CF45C01F4012181FC
:107530008501FAE02F02000D111D1124D4012C91B8
:10754000F5014AE02402E00DF11D11249F01285E9F
:10755000334008511C4F033E54E0150714F002EE6F
:1075600014E059012E316BEF360724F42EE1A22EE0
:107570002BEFB22E302F212F8017910714F4382FC4
:10758000292FE32EF22EEA14FB040CF47501AB85CF
:10759000BC854D905D906D907C90C301B20124E656
:1075A00030E040E050E00E94F069EB85FC852193DB
:1075B000319341935193FC87EB87AD85BE852D9325
:1075C0003D93BE87AD874114510461047104A9F055
:1075D00077FE04C0D701AA19BB0903C0D801AE19B0
:1075E000BF09A30192010E94806920EA36E841E0C8
:1075F00050E00E94F06929013A01C7010E94F51488
:107600007C01E40CF51CC8010E94F5148C01C50135
:107610000E94F5140E151F050CF47801E816F90602
:107620000CF47C01F4018281882319F0F194E19437
:10763000F10880914F048F71F0E1F81B2F852F170F
:10764000F8F4F601EE0FFF1FE05BFB4F9081892FEE
:10765000880F880F8595859599F0929596959695C2
:1076600093709D5F9370923058F040E060E00E940C
:107670004A15882329F0D1018C910E9435157C018F
:10768000F894E985FA85E192F192FA87E98778948E
:10769000FFEFCF1ADF0A22E0220E311C30E1C316C1
:1076A000D10409F02ECF6C960FB6F894DEBF0FBE52
:1076B000CDBFDF91CF911F910F91FF90EF90DF90A1
:1076C000CF90BF90AF909F908F907F906F905F9082
:1076D0004F903F902F900895223009F0A6C98B015A
:1076E000A4C9FF920F931F93CF93DF93CDB7DEB75B
:1076F000C054D1090FB6F894DEBF0FBECDBF63E012
:10770000CE0181960E94643361E0CE0101960E9411
:107710006433EFE2F3E09E012F5D3F4F8E010F5F78
:107720001F4F418152818081882329F0D9018D9199
:107730009C91D80104C0D8018D919C91D9016D9183
:107740007C91861B970B840F951F883EB3E09B07A7
:107750003CF489314CEF94073CF0482F892F02C04C
:1077600048EE83E0942F02C098E18CEF91838283EE
:1077700035962E5F3F4F0E5F1F4F83E0EF37F807C0
:1077800081F605EB13E0F12C8F2D0E942F1581114E
:1077900002C0D8011C92F3940F5F1F4FB4E0FB129C
:1077A000F3CF86E00E94C15281E00E94D866C05C9F
:1077B000DF4F0FB6F894DEBF0FBECDBFDF91CF9184
:1077C0001F910F91FF9008958F929F92AF92BF9259
:1077D000CF92DF92EF92FF920F931F93CF93DF939D
:1077E000C82F80913E05182F1F708073109255018D
:1077F000C038E9F198F4C33209F462C030F4C03201
:1078000061F1C23209F46AC0A8C0C53209F44DC0A2
:1078100008F441C0C13609F481C09FC0C43881F169
:1078200058F4C23809F467C008F483C088E99EE1BF
:107830000E94841283E864C0CE38C9F0CF3B09F4BB
:107840007EC0C53809F089C081E080937C0781EB58
:1078500099E40E94DC1985E81BC0133009F07DC053
:107860008091CC0791E089278093CC0766C081E0A6
:1078700080937C070E947A120E94DC198C2F08C02A
:1078800081E080937C0783E19DE20E94DC1984E81B
:107890000E941B5D62C0123009F05FC080911A081F
:1078A0008F5F833054F080E008C0123009F055C07B
:1078B00080911A08815087FD82E080931A084DC09C
:1078C0001F5F143008F010E0812B80933E0581E0AB
:1078D0000E94C15283E10E94D8663FC0112311F07B
:1078E000115001C013E0812B80933E0581E00E947E
:1078F000C15284E1F0CF83E29EE10E94841282E8CB
:10790000DF91CF911F910F91FF90EF90DF90CF907B
:10791000BF90AF909F908F900C941B5D8091BF079C
:10792000823021F483E08093BF0707C01330A9F4AD
:1079300002C00E9446310E94911287E1CCCF81E0C3
:107940000E941B5D83E00E941B5D82E00E941B5D24
:1079500081E08093FB0710921A0840E060E080917C
:10796000E7010E944A15C82F882331F08091FB0758
:10797000811102C00E94713BC093FB0790913C01B2
:1079800080912B05981710F4C6E001C0C4E080E098
:107990000E94EA104C2F406860E185E20E94880F47
:1079A00046E568E186E20E94F3588091BF0788238C
:1079B000A1F0823011F426E001C024E04091C80714
:1079C0005091C907022F60E18DE50E94180F20E059
:1079D00040E068E183E30E94021000E02091E501AD
:1079E00049E158E060E186E20E9418598091E40183
:1079F00080FF06C045E158E060E188E30E945259EB
:107A0000D0E08FE1E82E8D2F0E94EF0EE82FF0E0FE
:107A1000E05FF74FC4916D2F809177050E946D1143
:107A200097FD03969C013595279535952795243E1E
:107A30000CF424EEF22E4CE1421714F4BCE1FB2EC0
:107A40008FEF8D0F46E38230C8F464E08C2F0E94E4
:107A5000E759D13021F08091E40180FD0CC043E072
:107A60006EE18FEF8C0F0E94E75943E06EE181E0F9
:107A70008C0F0E94E7596E2D6F1913C06BE385EED2
:107A80008C0F0E94E4590FEF0C0F43E06AE3802F44
:107A90000E94E45943E06CE3802F0E94E459CF0D2B
:107AA0006BE347E08C2F0E94F31DDF5FD43009F0B9
:107AB000AACF123008F08AC0EBE5EE2EE7E0FE2EEA
:107AC00000E0F9E1DF2EABE1CA2EF701C191D191BF
:107AD0007F01802F8370113041F19E01D7FF02C0DA
:107AE000215E3F4F75E0359527957A95E1F7AE0118
:107AF000421B530B9A01D7FF02C0C158DF4FAE01A2
:107B0000440F452F441F550B420F531F602F66959E
:107B10006695660F660F660F685D8C9D802D11243B
:107B200020E28F5D0E94435B4CC0043018F492E267
:107B3000A92E02C0BEE5AB2EB82EBB0CBB0CB80EF6
:107B4000A6E28A2E8B0C8091E90181FF03C060E0E0
:107B500075E002C060E074E0AE01D7FF04C04427C6
:107B600055274C1B5D0BD49EF001D59EF00D1124C2
:107B7000CF019E5F0E94BA69962E59E1561714F400
:107B8000F9E19F2E25E543E3682D87EE8A0D0E94DB
:107B9000B45945E064E26B0D8A2D0E94E7591C162A
:107BA0001D0614F4A39401C0A91867E26B0D492DBA
:107BB0008A2D0E94E4596B2D6B5D492D8A2D0E9400
:107BC000E4590F5F083009F080CF30C0123021F542
:107BD0000E946E2460911A08662329F0862F880F70
:107BE000680F660F6D5F80E00E94583180911A081F
:107BF0008F5F682F660F680F660F81E0DF91CF916E
:107C00001F910F91FF90EF90DF90CF90BF90AF90BA
:107C10009F908F900C9458314091CA075091CB0798
:107C200004E024E068E28CE30E94180FDF91CF911A
:107C30001F910F91FF90EF90DF90CF90BF90AF908A
:107C40009F908F900895982F80918107292F281B4E
:107C500019166CF462171CF4892F861B09C03AEFC1
:107C6000360F23172CF4892F861B8A5F01C080E012
:107C7000809381070895BF92CF92DF92EF92FF9297
:107C80000F931F93CF93DF93C82E4EE0682F81E1AF
:107C900098E00E94C4218BE69FE00E941D1E182FD1
:107CA00080911E080E940A0FEC0120E0488160E0EC
:107CB00086E0810F0E94AE0FD090110866E08D2DF6
:107CC0000E94233E18E0F12CBB24B394409181071D
:107CD0004F0DEE24E394D412E12C50E04F305105C7
:107CE00008F045C1FA01E55AFF4F0C940F6A63E6AC
:107CF0007FE0812F0E944C592E2D20614981612FF8
:107D000084E50E948D0FEE2009F431C14CE261E060
:107D100089810E946A1289832AC16BE57FE0812FE5
:107D20000E944C590DE723E84A81612F80E60E94AA
:107D30007B1D8A831CC18F8186FF03C041E55FE004
:107D400002C04AE45FE0612F8CE00E9452590DE7C7
:107D500023E84885612F80E60E947B1D888707C144
:107D60008F812E2D4EE35FE0612F83FB882780F902
:107D70000E94BB259F8180FB93F90DC08F812E2D22
:107D800042E35FE0612F86FB882780F90E94BB25D4
:107D90009F8180FB96F99F83EAC08F8181702E2D91
:107DA0004CE25FE0612F9B2D981B892F0E94BB2521
:107DB0009B2D981B8F8190FB80F98F83D8C00F81FA
:107DC00007FB002700F9002319F046E25FE002C03C
:107DD00040E25FE02E2D612F8CE00E942C59EE20B6
:107DE00059F08F8187FB882780F961E00E946D122E
:107DF0009F8180FB97F99F838F8187FB882780F97C
:107E0000081709F4B4C01C82B2C08F8187FF09C073
:107E100004E62CE94C81612F80E60E947B1D8C8357
:107E2000A6C02E2D4C81612F82E10E94D826EE2023
:107E300009F49DC046E160EF8C810E946A128C8338
:107E400087300CF494C090E6C91291C0875080939B
:107E50001F088BE092E30E94DC1989C068E17FE093
:107E6000812F0E944C590E2D2E2D4B81612F8EE4B7
:107E70000E94C6268B837BC06FE07FE0812F0E942B
:107E80004C590F810295037049F0402F50E02E2D80
:107E90002064612F84E50E94435B07C02E2D4BE5D3
:107EA00053E0612F8EE40E942C59EE2009F45FC04C
:107EB00063E0802F0E946D1283708295807F9F8186
:107EC0009F7C1CC067E07FE0812F0E944C592F816E
:107ED000269523700E2D4DEE5EE0612F8EE40E94FC
:107EE0001859EE2009F443C08F81869562E08370B3
:107EF0000E946D128370880F9F81997F982B4BCFC2
:107F00004D8142954F7021EE3EE06E2D812F0E94F3
:107F1000D11B8295807F9D819F700BC04D814F70DA
:107F200027ED3EE06E2D812F0E94D11B8F709D8129
:107F3000907F982B9D831BC04E8142954F702BECF8
:107F40003EE06E2D812F0E94D11B8295807F9E8105
:107F50009F700BC04E814F7021EC3EE06E2D812F43
:107F60000E94D11B8F709E81907F982B9E83F394EB
:107F7000185F87E0F812AACEDF91CF911F910F9181
:107F8000FF90EF90DF90CF90BF9008957F928F92F7
:107F90009F92AF92BF92CF92DF92EF92FF920F9398
:107FA0001F93CF93DF93C82F8CE491E10E941D1E95
:107FB00050E1E52E0BE02EEB31E146E06C2F87E13E
:107FC00098E00E94B321E0901708EA9466E08E2DB5
:107FD0000E94233EC03611F0C43669F4E7FC0BC0A2
:107FE000E0921F088C2F0E941B5D1092B3018BE062
:107FF00092E30E94DC19B12CC12C28E0D22EFF2480
:10800000E7FCF09435E0A32E49E0942EC09181075F
:10801000CB0D0C2F10E0D1E0E016F10609F0D0E016
:1080200088248394C83028F4812C88E38D1528F4A3
:108030005BC0E0E3ED1508F457C0C11002C0CD2EBF
:1080400002C0CC24C3942D2F49E451E16D2D80E072
:108050000E942C59A8014F5F5F4FC93010F482E194
:1080600001C087E12D2F6D2D0E94435B882051F0C8
:1080700008501109909EE001919ED00D1124CF511E
:10808000DC4F07C0A09EE001A19ED00D1124C75473
:10809000DC4F8E019AE2792EF80141918F0155272C
:1080A00047FD50956D2D872D0E94525BF5E17F0EA7
:1080B00083E97812F1CF08E00D0D882079F025963C
:1080C0001AE24991552747FD5095602F812F0E9454
:1080D000525B1B5E1E37A9F700E10D0DB394E7E07C
:1080E000BE1611F0D02E92CFC11005C0809181072D
:1080F0008F5F80938107DF91CF911F910F91FF9048
:10810000EF90DF90CF90BF90AF909F908F907F9037
:108110000895BF92CF92DF92EF92FF920F931F9339
:10812000CF93DF93C82F8BEB90E10E941D1EF9E0E7
:10813000EF2E0BE02EEB31E149E06C2F84E198E06B
:108140000E94B32110911408115066E0812F0E9403
:10815000233EB82EC03899F480E80E941B5D89E167
:1081600080937E07193019F40E94E55D05C0183030
:1081700018F4812F0E940D5E81E00E94D866E8E02D
:10818000FE2EC12EDD24C7FCD09488E0B81205C0B5
:1081900080917E078823D1F13CC0CB2DD0E0CC1656
:1081A000DD0611F401E101C000E19E012F5F3F4FA8
:1081B000442737FD4095542F72E0E72E6F2D82E162
:1081C0000E94335A80917E07811104C021E0CC16B1
:1081D000DD0609F020E0FE01EE0FFF1FE85BF44E24
:1081E000459154916F2D88E10E942C5988E0F80E3A
:1081F000B39480E4F812C9CFDF91CF911F910F9112
:10820000FF90EF90DF90CF90BF90089521E018305D
:1082100009F020E048EA50E16F2D86E0DF91CF9130
:108220001F910F91FF90EF90DF90CF90BF900C9433
:108230002C592F923F924F925F926F927F928F9222
:108240009F92AF92BF92CF92DF92EF92FF920F93E5
:108250001F93CF93DF9300D000D0CDB7DEB7282E89
:1082600083E69EE00E941D1E80915507882321F021
:108270000E94D627182F01C010E080915907811164
:108280000BC0E09058070BE02EEB31E144E0622D8B
:1082900080E198E00E94B321609010088091B301C2
:1082A000803621F08F3B31F08E32A1F4909155074A
:1082B000992319F0109255070DC09091590791110B
:1082C00009C00E941B5D1092B301611007C010929B
:1082D000550702C06620D9F3198202C081E0898364
:1082E00067E0862D0E94233E382E80915907811128
:1082F0001092B30180915507882369F011160CF490
:10830000B0C11111B0C18091B301823609F4A9C185
:10831000833609F4A8C14424439411E0512CA32CC2
:10832000B12C852D0E940A0F7C01311678F4612F43
:1083300070E06A197B096830710544F4660F660FB6
:10834000660F20E0442D81E00E94AE0F9FE195155D
:1083500008F4C7C0F701F081FA83F411C2C0C70165
:108360000A969C838B83F52CCB80DC809AE0C91A1B
:10837000D108311608F0A2C0812F90E08A199B091C
:10838000883091050CF08BC0782E770C770C770C29
:1083900080915507811115C0611213C0F0921E081B
:1083A000EA81E0931C08F981FF2331F0109256070F
:1083B00081E080935907212CEE24E39480915907A2
:1083C0008111E12C5F1459F0F60127812695237065
:1083D00000E04EE55EE0672D83E10E94185920E140
:1083E000EB81FC8139974081672D80E30E948D0FDE
:1083F0000DE723E88B809C80F8E08F1A9108F40148
:108400004081672D8DE20E947B1DF4018083EB810A
:10841000FC8137974081442329F020E0672D88E4D0
:108420000E94D00FEB81FC8136974081442379F084
:10843000F601878120E087FF06C044E6672D80E6CD
:108440000E94645804C0672D80E60E94D826F60179
:108450008681811102C040E201C043E5F6018581B9
:10846000882329F0433511F44AE201C044E4672D22
:1084700089E70E94F358809155078823F9F080918D
:108480001D088F111BC020E046E6672D88E10E9481
:108490007A59F0921E0810931008612E0FC00897A9
:1084A00069F480915507882349F080911D088F1148
:1084B00005C0809110088F5F809310081F5FF394B0
:1084C000F0E2FF1609F448C08B819C810A969C83D8
:1084D0008B83FC013A9780819A81891709F444CFF4
:1084E0003BC0611237C040921C0850921E08662D96
:1084F0006A19660F660F660F615029E049E180E056
:108500000E94555BE981EE2329F10E9441278111E8
:1085100021C060E080911E080E94241C1092550723
:108520008BE39EE30F900F900F900F90DF91CF9110
:108530001F910F91FF90EF90DF90CF90BF90AF9081
:108540009F908F907F906F905F904F903F902F9073
:108550000C94DC191F5FF52C4394F1E14F1611F0D8
:108560005F2CDFCE80915907882309F460C02092E8
:10857000B30165E085E991E10E940B2884E00E9447
:10858000E227F82E00915607602F660F660F660FE0
:10859000685F20E044E288E10E947A5981E0F812A5
:1085A00035C0013079F40E94412781110DC08091BE
:1085B0001E088F5F80931E0860E00E94241C1092AA
:1085C000550702C0023018F48BE39EE30EC0809181
:1085D0001E08043069F4809357078091B3010E940C
:1085E0001B5D1092B30189E597E20E94DC190BC074
:1085F000023031F48F5F80931E0861E00E94241CDA
:1086000081E080935507109259070BC092E0F91250
:1086100008C0109259078091B3010E941B5D10920F
:10862000B30180911E0880931D081092800711509D
:10863000109358070F900F900F900F90DF91CF91EC
:108640001F910F91FF90EF90DF90CF90BF90AF9070
:108650009F908F907F906F905F904F903F902F9062
:10866000089561E001C060E080911E080E94F62636
:1086700052CE8F929F92AF92BF92CF92DF92EF92A3
:10868000FF920F931F93CF93DF93C82F8FE290E158
:108690000E941D1E2CE0A22ECC24C3943DE2E32EAA
:1086A00030E1F32E0BE02EEB31E147E06C2F82E15D
:1086B00098E00E943C1FC0901208CA94B0905A07DC
:1086C00066E08C2D0E94233E982E48E0F42EDD2497
:1086D000C7FCD094092D10E0C016D10639F4809162
:1086E0008007882329F092E0A92E04C0A12C02C0A3
:1086F000AA24A3946BE270E18F2D0E944C5988E06C
:10870000891510F448E301C041E3490D6F2D85E060
:108710000E94F358E801CC0FDD1FC00FD11FC75DC9
:10872000DB4FBB2011F000E001C00A2D2A812F7021
:1087300040EC5FE06F2D8DE00E9418598A818F70A8
:108740000E94FC0E182F811131C091E0B91611F072
:1087500020E001C02A2D48816F2D86E30E948D0FF5
:1087600088818532B4F0BBED8B2E880E6981882D0F
:108770000E94811C9C0182E0B81611F000E001C04B
:108780000A2DA2E0EA2E482D6F2D84E60E94F81CE7
:1087900072C092E0B91611F020E001C02A2D498183
:1087A000552747FD50956F2D83E663C08130B9F49E
:1087B00081E0B81611F020E001C02A2D48816F2D0C
:1087C00086E30E94D00F92E0B91611F020E001C0BC
:1087D0002A2D49816F2D8DE40E94D00F4CC082302C
:1087E000B9F481E0B81611F020E001C02A2D4881CB
:1087F0006F2D86E30E948D0F92E0B91611F020E0F4
:1088000001C02A2D49816F2D80E50E948D0F33C054
:108810006CEB7FE08F2D0E944C59488147FF03C0CD
:10882000409580E201C080E091E0B91202C02A2D9B
:1088300001C020E0282B552747FD50954F5F5F4F23
:108840006F2D89E40E94435B498147FF03C0409537
:1088500080E201C080E092E0B91202C02A2D01C07E
:1088600020E0282B552747FD50954F5F5F4F6F2D18
:108870008BE60E94435B4A8142954F7049300CF071
:108880004F5F83E0B81611F020E001C02A2D6F2D54
:1088900088E60E94D00F80917F07882309F45EC08C
:1088A000AA2009F45BC091E0B91631F1B91698F02D
:1088B00082E0B816D1F193E0B91250C08A816FE01E
:1088C00082958F700E946D128295807F9A819F7031
:1088D000982B9A8343C08A816EE08F700E946D123C
:1088E0008F709A81907F982B9A830E94FC0E1817A4
:1088F000A9F11882198232C0113069F038F01230B3
:1089000069F0133059F543E66EEC0AC06EE28881D7
:108910000E946D1208C046E16AEE02C04EE260E0BD
:1089200088810E946A12888319C0113059F038F08A
:10893000123059F0133091F443E66EEC0BC04DE762
:1089400063E808C046E16AEE05C06EE289810E94D4
:108950006D1203C089810E946A128983939488E012
:10896000F80E90E4F912B6CEDF91CF911F910F91DE
:10897000FF90EF90DF90CF90BF90AF909F908F903F
:1089800008959F92AF92BF92CF92DF92EF92FF92A3
:108990000F931F93CF93DF93982E8091E2018F70F6
:1089A000813011F0C5E101C0C7E184ED9DE00E9476
:1089B0001D1EAA24AA94AC0EAEE0CA2EB5ECEB2E76
:1089C000BDE0FB2E0BE02EEB31E140E0692D8DE0A8
:1089D00098E00E943C1F10910D08C0905A0767E074
:1089E000812F0E94233ED82E2091290530E02F5F51
:1089F0003F4F442737FD4095542FC2E0EC2E01E154
:108A000060E08AE20E94335AD1103BC060EC7DE006
:108A100088E00E944C5900E12AE043ED51E068E013
:108A200082E40E94F658113009F031C429E040E494
:108A300067E080E40E94555B8C2D880F8C0D880FB9
:108A40002091800746E068E08E5B0E947A59809111
:108A50008007882309F41BC4CC2DD0E0CD52DE4F13
:108A600088810E94702B61E40E946D120E94802B0D
:108A70009881981709F40BC4888382E00E94C15240
:108A800006C421E02D1520F1C8E06FEA7DE08C2FAF
:108A90000E944C59123081F480E6981204C08091F3
:108AA000DD010E94AE1261E38091DD010E946D1232
:108AB0008093DD0121E001C020E04091DD0150E024
:108AC0004C5F5E4F6C2F88E50E94435BC85F04C01B
:108AD00092E0D91212C0C8E061E872E18C2F0E94C6
:108AE0004C59133009F02CC421E0C212D2C380913A
:108AF0008007811127C401E026C483E0D8121AC080
:108B0000C8E067EA7DE08C2F0E944C59143051F484
:108B100049E467EC8091DE010E946A128093DE01D5
:108B200041E001C040E021E06C2F8CE30E94021084
:108B3000C85F04C094E0D9121CC0C8E06EE97DE0B3
:108B40008C2F0E944C59153051F445E16BEE809109
:108B50004E040E946A1280934E0441E001C040E03E
:108B600022E06C2F8CE30E940210C85FC93328F00A
:108B7000ECC325E0D21224C0C8E061E872E18C2F7A
:108B80000E944C59163071F48091DF0161E08170D0
:108B90000E946D129091DF0180FB90F99093DF01AC
:108BA00001E001C000E02091DF01217048E85DE0B4
:108BB0006C2F8CE30E941859C85FC93328F0C5C3D5
:108BC00086E0D81217C0C8E021E0173009F020E095
:108BD0008091E40141E85DE06C2F81700E94BB252B
:108BE0009091E40180FB90F99093E401C85FC93350
:108BF00028F0ABC397E0D91218C0C8E021E01830C4
:108C000009F020E08091E4014AE75DE06C2F829555
:108C100081700E94BB259091E40180FB94F99093B0
:108C2000E401C85FC93328F090C328E0D2121EC007
:108C3000C8E061E77DE08C2F0E944C59193049F45F
:108C400064E08091E5010E946D128093E50101E0EE
:108C500001C000E02091E50141E55DE06C2F8CE36F
:108C60000E941859C85FC93328F06FC389E0D81231
:108C70001AC0C8E069E47DE08C2F0E944C5921E0C5
:108C80001A3009F020E0022F4091E7016C2F86E3B3
:108C90000E94C6268093E701F8E0EF2EEC0E98E3E1
:108CA0009E1530F452C32AE0D21250C0E8E0EE2EF6
:108CB00060E47DE08E2D0E944C597CE3B72EC0E02D
:108CC000D0E0CC1202C01B3061F02091E80130E00E
:108CD0000C2E02C0359527950A94E2F7022F0170F9
:108CE00001C002E0AE01485C524F21E06E2D8B2D99
:108CF0000E94F658219626E0B20E86E6B812E1CF21
:108D00001B30F9F490E6991631F020913F01309133
:108D10004001232BB1F0892D0E941B5D109280072A
:108D200021E030E00C2C01C0220F0A94EAF7809178
:108D3000E80182278093E80182E00E94C1520E94EC
:108D40005253C8E0CE0DC93310F0FFC2C8E0D09135
:108D5000E201DF702BE02D1508F4D5C062E37DE061
:108D60008C2F0E944C591C3041F4C11006C08091D8
:108D70008007882321F002E003C000E001C001E089
:108D80002D2F42E15DE06C2F84E20E941859DD2313
:108D900071F08DE08D0F8F70823008F040C068E078
:108DA0007DE08C2F0E944C5958E4E52E07C06CE002
:108DB0007DE08C2F0E944C596CE3E62E1C3049F468
:108DC00081E0C81206C080918007882321F002E06C
:108DD00003C000E001C001E02091E3012E5F4AEEF4
:108DE0005CE06C2F8E2D0E9418591C3049F492E0E3
:108DF000C91206C080918007882321F022E003C0B9
:108E000020E001C021E04091E60182E34802A00198
:108E10001124445D5E4F6C2F88E28E0D1CC0D13052
:108E2000E1F463EE7CE08C2F0E944C591C3049F435
:108E300091E0C91206C080918007882321F022E0CA
:108E400003C020E001C021E04091E301552747FD28
:108E500050956C2F8EE70E94435B1C3009F04FC089
:108E600080917F07882309F44AC08091480585FFD7
:108E700002C064E001C063E021E0C21699F0C216AE
:108E800020F082E0C81631F134C08091E2018F7089
:108E90000E946D128F709091E201907F982B9093B9
:108EA000E20127C0DD2329F08DE08D0F8F70823025
:108EB00038F444E06EEF8091E3010E946A1207C02B
:108EC000D130B9F46CE78091E3010E946D12809378
:108ED000E3010FC0DD2329F08DE08D0F8F7082300C
:108EE00040F44AE06CEF8091E6010E946A128093A0
:108EF000E6018091E2018F708D131092E301C85F4B
:108F0000C93320F022C29CE0D91278C0DD2329F0B9
:108F10008DE08D0F8F708230F8F464ED7CE08C2F43
:108F20000E944C591D3051F444E16CEE8091EC01EB
:108F30000E946A128093EC0121E201C020E240917C
:108F4000EC0185E04802A00111244F515F4F6C2FC6
:108F50008CE40E94435B4EC0D13011F568EC7CE09C
:108F60008C2F0E944C591D3009F044C020E0C110E4
:108F700007C048E16C2F80E00E947A5981E006C06A
:108F80004EE16C2F84E20E947A5980E290E89912B7
:108F900031C08093BD0C82E09CE10E94DC192AC0A4
:108FA0006FEB7CE08C2F0E944C592091E30127FD50
:108FB00004C023301CF022E001C020E02093E30134
:108FC0001D3031F480918007882321F002E003C036
:108FD00000E001C001E042EA5CE06C2F8CE30E94FB
:108FE00018591D3039F462E08091E3010E946D123E
:108FF0008093E301C85FC93308F0A7C1D13009F0FD
:1090000057C02DE02D1548F16CE97CE08C2F0E94B3
:109010004C598091E20182958695869583701E3029
:1090200029F462E00E946D1201E001C000E0282FE7
:109030002295220F220F207C9091E2019F73922BA8
:109040009093E201282F41E95CE06C2F8CE30E94B1
:109050001859C85FC93320F078C18EE0D8122AC0F1
:1090600068E87CE08C2F0E944C598091E201829547
:1090700083701F3029F462E00E946D1201E001C08C
:1090800000E0282F23702295207F9091E2019F7CA1
:10909000922B9093E201282F4DE75CE06C2F8CE33C
:1090A0000E941859C85FC93308F04FC1D0E105C00C
:1090B000DEE001C0D0E1DD1648F560E77CE08C2FF2
:1090C0000E944C591D1313C08091E40167E0829502
:1090D000869587700E946D128295880F807E909190
:1090E000E4019F71982B9093E40121E001C020E0FE
:1090F0004091E4014295469547704F5C6C2F82E7A2
:109100000E946458C85FC93308F01FC101E00D0F09
:10911000D01618F566E67CE08C2F0E944C5910138F
:109120000EC08091E90161E081700E946D12909102
:10913000E90180FB90F99093E90101E001C000E0B2
:109140002091E90121704EE55CE06C2F8CE30E94D8
:109150001859C85FC93308F0F8C082E08D0FD816DF
:10916000B0F421E0181320E08091E90144E55CE0CF
:109170006C2F869581700E94BB259091E90180FB40
:1091800091F99093E901C85FC93308F0DEC083E02C
:109190008D0FD816B0F421E0181320E08091DF0184
:1091A0004CE45CE06C2F869581700E94BB25909109
:1091B000DF0180FB91F99093DF01C85FC93308F0AC
:1091C000C4C084E08D0FD816B8F421E0181320E055
:1091D0008091DF0143E45CE06C2F82FB882780F9FB
:1091E0000E94BB259091DF0180FB92F99093DF01F3
:1091F000C85FC93308F0A9C005E00D0FD016E0F430
:1092000067E37CE08C2F0E944C59101309C064E680
:10921000809183040E946D128093830421E201C037
:1092200020E24091830450E06C2F8EE70E94435B64
:10923000C85FC93308F089C0DA5FDD1608F085C061
:1092400068E27CE08C2F0E944C591D1313C0809162
:109250004F0467E08295869587700E946D12829513
:10926000880F807E90914F049F71982B90934F04AC
:1092700001E001C000E020914F042295269527705F
:109280004EE05CE06C2F8CE60E9418595EC0C0E195
:10929000FCCBC11055C08091800700E0882311F0FD
:1092A00022E001C021E04091E0015091E1016C2FEA
:1092B00087E40E94180F133009F040C080917F07A7
:1092C0008823E1F16CE370E08091E0019091E1018D
:1092D0000E94BA69962FD82FCC2021F081E0C816C1
:1092E00091F02CC06BE3892F0E946D122CE3820257
:1092F000C00111248D0F911DD7FD9A959093E10126
:109300008093E0011BC04EE361E082E08D0F0E947C
:109310006A12D81BDE5F2091E0013091E1012D1B24
:109320003109D7FD339537FD05C03093E101209316
:10933000E00104C01092E1011092E001C85FE1CBAE
:1093400000E001C002E020E0AECFDF91CF911F919D
:109350000F91FF90EF90DF90CF90BF90AF909F90D4
:1093600008958F929F92AF92CF92DF92EF92FF92E9
:109370000F931F93CF93DF93D82E83E89AE00E9438
:109380001D1E2FE1A22E32E0C32E40E8E42E4AE05B
:10939000F42E06E022EB31E140E06D2D82E098E012
:1093A0000E943C1FF0900208C0915A0767E08F2D81
:1093B0000E94233E182F883139F48AE18F1510F06E
:1093C0001FEF01C011E0185E11113AC065E77AE0A5
:1093D00088E00E944C5900E12AE04DE455E068E045
:1093E00082E40E94F65881E0F81220C429E040E4AB
:1093F00067E080E40E94555B8C2F880F8C0F880FEC
:109400002091800746E068E08E5B0E947A59809147
:109410008007882309F40AC4D0E0C35BDA4F88814F
:109420000E94702B61E40E9475120E94802B98812B
:10943000981709F4FBC3888381E00E94C152F6C3E8
:10944000123050F5D8E0C0913F05C695C695C69537
:10945000C7706EE67AE08D2F0E944C5982E0F812B8
:1094600011C066E08C2F0E947512C82F8770880F7C
:10947000880F880F90913F05977C982B90933F051C
:1094800001E001C000E02C2F42E45AE06D2F8CE592
:109490000E941859D85F03C0123021F5D8E0C0915E
:1094A0004B05C43008F0C4E067E37AE08D2F0E94DA
:1094B0004C5983E0F8120CC064E08C2F0E947512A6
:1094C000C82F843009F487E080934B0501E001C088
:1094D00000E02C2F43E05AE06D2F82E40E941859DF
:1094E000D85F03C0133001F5D8E0C0915805C95FBB
:1094F0006CEF79E08D2F0E944C5984E0F81207C080
:1095000067E08C2F0E947512C82F21E401C020E46F
:109510004C2F50E06D2F86E60E94435BC750C093EE
:109520005805C8E0CD0F03C01430F9F4C8E06DEE63
:1095300079E08C2F0E944C5985E0F8120AC044E66D
:1095400061E0809149050E9472128093490521E4EF
:1095500001C020E44091490550E06C2F86E60E944E
:10956000435BC85FC93320F063C31530F1F4C8E032
:109570006CED79E08C2F0E944C5986E0F81209C0FE
:1095800065E080914A050E94751280934A0521E4A6
:1095900001C020E440914A0550E06C2F86E60E940D
:1095A000435BC85FC93320F043C3163009F5C8E0F8
:1095B00063ED79E08C2F0E944C5987E0F8120CC0C3
:1095C0004DE26AE080912A050E94721280932A057A
:1095D0000E94EA5B21E401C020E440912A0550E0AA
:1095E0006C2F86E60E94435BC85FC93320F020C31E
:1095F0001730F1F4C8E063EC79E08C2F0E944C59ED
:1096000088E0F8120AC048E768E280912B050E94C2
:10961000721280932B0521E401C020E440912B05B8
:109620006C2F86E60E94720FC85FC93320F000C31A
:10963000183019F5C8E060EB79E08C2F0E944C5986
:1096400089E0F8120AC04EE666EF809141050E945B
:1096500072128093410521E001C020E04091410554
:10966000552747FD5095465F5F4F6C2F80E70E945E
:10967000435BC85FC93320F0DBC21930B9F4C8E0DE
:1096800021E08AE0F81220E0809142054FE959E09C
:109690006C2F81700E9490259091420580FB90F97B
:1096A00090934205C85FC93320F0C2C21A30C1F49A
:1096B000C8E021E08BE0F81220E08091420543E908
:1096C00059E06C2F869581700E94902590914205FB
:1096D00080FB91F990934205C85FC93320F0A8C27E
:1096E0001B30C9F4C8E021E08CE0F81220E0809142
:1096F000420544E859E06C2F82FB882780F90E94DC
:1097000090259091420580FB92F990934205C85FA5
:10971000C93320F08DC21C30C9F4C8E021E08DE0CF
:10972000F81220E08091420546E759E06C2F83FB58
:10973000882780F90E9490259091420580FB93F93B
:1097400090934205C85FC93320F072C21D30F1F416
:10975000C8E069E679E08C2F0E944C598EE0F8123F
:109760000AC046E16AEE80912D050E947212809334
:109770002D0521E001C020E040912D056C2F80E6F1
:109780000E94D00FC85FC93348F052C21E3029F082
:10979000D8E000E090E1C92E4CC0C8E021E08FE0A5
:1097A000F81220E08091480548E559E06C2F86FBCF
:1097B000882780F90E9490259091480580FB96F9B2
:1097C00090934805D8E0DC0FD93318F331C201116A
:1097D00033C068E479E08D2F0E944C5901112FC0ED
:1097E000C0914405FC102EC068E78C2F0E947512B2
:1097F000C82F21E0CC2341F1206485E0C89FA0015F
:1098000011246D2F86E60E94435B43E76D2F809104
:10981000810C0E94F35801111EC0C0934405D85F0B
:10982000D93308F005C281E08C0D0F5F8231B1F0B1
:10983000C82E1C15C0F7CBCF68E379E0CCCFC09120
:109840004C05D0CF20E0D6CF4BE553E06D2F86E618
:109850000E942C59E0CFC0934C05E1CF1231B0F4F7
:1098600021E0F81220E0809142054AE259E06D2F94
:10987000829581700E94B0259091420580FB94F9F9
:1098800090934205D85FD93308F0D2C182E08C0DA5
:109890001817B0F421E0F81220E0809148054EE15D
:1098A00059E06D2F829581700E94B02590914805F6
:1098B00080FB94F990934805D85FD93308F0B8C17C
:1098C00083E08C0D1817A8F421E0F81220E08091B5
:1098D0003F054DE059E06D2F81700E94B0259091B9
:1098E0003F0580FB90F990933F05D85FD93308F08E
:1098F0009FC184E08C0D1817B0F421E0F81220E02D
:1099000080913F054BE053E16D2F869581700E9459
:10991000B02590913F0580FB91F990933F05D85F6A
:10992000D93308F085C185E0E82EEC0C1E1508F04F
:109930003EC062E079E08D2F0E944C5907E8802EEE
:1099400002E1902EC2E4AA24A394809157058A21B3
:1099500001E009F400E021E0A4016D2F8C2F0E94AA
:10996000F658AA0CCA5F8FEF881A980AC23769F7AF
:10997000FE1019C029E042E36FEF6D0F81E40E94F1
:10998000555B80E6D81619F08EE6D8120CC08D2DE6
:109990000E941B5D0E94DA10809357051092800789
:1099A00081E00E94C152D85FD93308F041C186E0FE
:1099B0008C0D1817B8F421E0F81220E080913F05D3
:1099C00043EF58E06D2F82FB882780F90E94B02575
:1099D00090913F0580FB92F990933F05D85FD93372
:1099E00008F026C187E08C0D1817B8F421E0F812B2
:1099F00020E080913F0587FB882780F945EE58E0FD
:109A00006D2F0E94B02590913F0580FB97F99093B0
:109A10003F05D85FD93308F00BC188E08C0D1817CB
:109A2000B8F421E0F81220E0809142054BED58E0B7
:109A30006D2F85FB882780F90E94B0259091420503
:109A400080FB95F990934205D85FD93308F0F0C0B8
:109A500089E08C0D1817B8F421E0F81220E080910D
:109A6000480587FB882780F94FEC58E06D2F0E944E
:109A700090259091480580FB97F990934805D85F11
:109A8000D93308F0D5C08AE08C0D1817B8F421E05E
:109A9000F81220E08091420547EC58E06D2F86FBDC
:109AA000882780F90E94B0259091420580FB96F9A5
:109AB00090934205D85FD93308F0BAC08BE08C0D83
:109AC0001817B8F421E0F81220E08091480549EB1E
:109AD00058E06D2F85FB882780F90E949025909192
:109AE000480580FB95F990934805D85FD93308F075
:109AF0009FC08CE08C0D1817A8F421E0F81220E02C
:109B000080915C054FEA58E06D2F81700E9490258E
:109B100090915C0580FB90F990935C05D85FD933F8
:109B200008F086C08DE08C0D181768F5EE24E394DC
:109B3000F812E12C60EA78E08D2F0E944C59E091F8
:109B40004505F0E0E056FC4F0491CCE6E02FE370D1
:109B5000F0E0E556F74F44912E2D6D2F8C2F0E948B
:109B6000645806950695C650C43581F7EE2039F045
:109B700067E1809145050E94751280934505D85F85
:109B8000D93308F055C00EE00C0D101708F050C086
:109B900045E958E06D2F86E00E945259D83328F0ED
:109BA00018E01D0F193378F043C014E2C0E02C2FE9
:109BB00044ED51E16D2F812F0E941F58CF5F185E39
:109BC000C430A9F7EDCFF01215C08091800788232B
:109BD00099F063E0809140050E94751290914005D4
:109BE000891761F0909148059F779093480580937D
:109BF000400504C020E003C021E001C022E0409104
:109C000040054F5C612F82E10E946458D4E2C0E0BD
:109C10008C2F0E94EF0E20E0482F612F8D2F0E9485
:109C20008D0FCF5FD85EC43099F702C0D0E10BCC66
:109C3000DF91CF911F910F91FF90EF90DF90CF9028
:109C4000AF909F908F9008953F924F925F926F9246
:109C50007F928F929F92AF92BF92CF92DF92EF92BC
:109C6000FF920F931F93CF93DF93D82E82E491E15D
:109C70000E941D1ED1E1AD2ECC24C39410E4E12E30
:109C800011E1F12E0BE02EEB31E145E06D2D86E187
:109C900098E00E943C1FF0901608FA94E0905A0752
:109CA00066E08F2D0E94233E882E2FE02F15A0F016
:109CB000EF2DF0E0EE0FFF1FE55AF84F4081518184
:109CC00057FF02C04F5F5F4F5595479544525A4F1B
:109CD00060E08EE40E94525B80E8D81225C02FE03D
:109CE0002F1510F14F2D50E0FA01E819F109EE0F90
:109CF000FF1FE55AF84F20813181E11015C085E042
:109D0000849FF001859FF00D1124E35DFC4F82815B
:109D1000882319F03195219531093483238382E01A
:109D20000E94C1520E945253E8E0CE2EFAE0AF2EBC
:109D3000B12C80E1881609F4F3C0882D0E94110F20
:109D4000EC01E82DF0E0EE0FFF1FE55AF84F80819F
:109D500091814A812B813C81442319F031952195D1
:109D60003109821B930B833391051CF0411109C00B
:109D7000D5C08E3C9F4F1CF4442319F0CFC01DE288
:109D800001C01FE755245394580C20E0452D6C2D3D
:109D900080E00E94AE0F412F6C2D8BE40E94F3589F
:109DA0008091E90181FF03C06DE7662E02C054E691
:109DB000652E912C44244A944C0C362C3194F81086
:109DC00008C0E91006C080918007811105C021E01C
:109DD00004C020E0712C09C022E080917F07882315
:109DE000C9F37724739410925501809183048823DA
:109DF00081F00B811C810115110579F090E080172D
:109E0000910754F0919581959109081719072CF441
:109E100003C000E010E001C08C01C801B5010E9440
:109E2000BA6982E09816D9F183E0981609F45BC00C
:109E300081E09816B1F020624B815C816C2D8DE23F
:109E40000E94435B772009F45EC022E048EE53E0B5
:109E500068E17CEF8B819C810E94B3119C838B8392
:109E600052C088818456AB01480F511D87FD5A9519
:109E700043388FEF580714F443E85FEF6C2D88E404
:109E80000E94435B772009F43EC088818456888312
:109E900049E1632D0E946A128C59888334C08981FC
:109EA0008C59AB01480F511D87FD5A954E3751050E
:109EB00014F04DE750E06C2D86E60E94435B012BC9
:109EC00031F029E048E3642D82E30E94555B77205E
:109ED000D1F089818C598983462D67EE0E946A12E0
:109EE0008456898310C04A816C2D8CE60E94301FF5
:109EF000772049F061E08A810E946D1291E0811122
:109F000001C090E09A83939424E0921258CF88E0A5
:109F10008C0D8034A1F1C82E852C0BCF1EE732CFDB
:109F2000C1E020E1F212C0E080917E07811125C0DE
:109F30002C2F4FE251E16C2D82E10E942C59CC2351
:109F4000F1F080E8D8121BC089E180937E0780E899
:109F50000E941B5DDF91CF911F910F91FF90EF90B9
:109F6000DF90CF90BF90AF909F908F907F906F9039
:109F70005F904F903F900C94713B20E0DACFDF91DF
:109F8000CF911F910F91FF90EF90DF90CF90BF90F6
:109F9000AF909F908F907F906F905F904F903F9089
:109FA00008956F927F928F929F92AF92BF92CF92BD
:109FB000DF92EF92FF920F931F93CF93DF93C82FFF
:109FC00088E990E10E941D1E41E1A42E52E0C52EB9
:109FD00065E9E62E60E1F62E0BE02EEB31E148E07C
:109FE0006C2F83E198E00E943C1FA0901308AA9474
:109FF00090905A0766E08A2D0E94233EB82E18E002
:10A00000CA2CDD24C7FCD094B11027C065E870E1EC
:10A01000812F0E944C59A11015C080918007882380
:10A0200011F0C2E001C0C1E080914F0460E18F7186
:10A030000E946D128F7190914F04907E982B909397
:10A040004F0401C0C0E040914F044F7150E02C2FED
:10A05000612F8CE60E94435B5DC180914F048F713C
:10A0600000E1081BEB2CF12CE701CC0FDD1FC25BDC
:10A07000DB4F20E04B2D612F80E00E94AE0F0B15CF
:10A0800008F4C3C0812CCE14DF0441F4981006C03C
:10A0900080918007811105C001E004C000E0712CAF
:10A0A00007C002E080917F078823C9F37724739467
:10A0B0008881811021C0807C803421F0803821F497
:10A0C00046E503C041E401C043E5202F612F8EE146
:10A0D0000E946458772009F493C0888162E08295D9
:10A0E0008695869583700E946D128295880F880FE1
:10A0F000807C98819F7330C091E0891230C0982F86
:10A10000907C903819F026E1622E02C099E1692E08
:10A11000482F440F440F4595459547314CF029EEA3
:10A12000240F4EE650E1612F8AE20E94185905C0C3
:10A13000202F612F8AE20E94D00F772009F460C09F
:10A140008881880F880F462D6AEE859585950E9437
:10A150006A128F739881907C982B988351C0982FA6
:10A16000907C4981903491F447FD03C04F3024F432
:10A1700001C040E0242F01C02FE029834FE152E1CC
:10A18000612F80E60E9418594FE017C0903841F5C2
:10A19000880F880F89359CF047FD04C049301CF0BA
:10A1A00049E001C040E0498321E0240F4DED52E138
:10A1B000612F80E60E94185949E060E01BC04F36CD
:10A1C0000CF04FE64983552747FD509540585F4FA7
:10A1D000202F612F80E60E94435B4FE660E80AC0B3
:10A1E000552747FD5095202F612F80E60E94435B45
:10A1F0004DE763E8772021F089810E946A12898304
:10A20000839483E088123FCF85C06BE670E1812F95
:10A210000E944C59812CCE14DF0441F4981006C0E2
:10A2200080918007811105C001E004C000E0712C1D
:10A2300007C002E080917F078823C9F377247394D5
:10A240008881811014C0482F4F71202F612F8EE11B
:10A250000E94D00F772009F459C0888145E160E061
:10A260008F710E946A128F719881907E1CC091E05C
:10A2700089121CC0282F2295269527704FE350E1A4
:10A28000612F8CE30E941859772009F43FC0888120
:10A2900066E08295869587700E946D128295880F80
:10A2A000807E98819F71982B988330C08295869587
:10A2B000877090E04981069774F0493008F049E0D2
:10A2C000498321E0240F4DED52E1612F80E60E9489
:10A2D000185949E010C04B3F38F450E0202F612F4F
:10A2E00086E60E94435B06C0485F202F612F84E50D
:10A2F0000E94631D4FEF772049F050E0898122E0F2
:10A3000060E070E090E00E94B3118983839483E061
:10A31000881281CFB394185F103409F075CEDF91A5
:10A32000CF911F910F91FF90EF90DF90CF90BF9052
:10A33000AF909F908F907F906F9008951F93CF93D1
:10A34000DF93EC011AE088810E94702B0E94802B21
:10A3500089931150C1F7DF91CF911F91089590918A
:10A360003F08982B90933F08F8948091830C90912C
:10A37000840C789490933E0880933D080895EDEF07
:10A38000F4E080E090E021913191820F931F25E06D
:10A39000E531F207C1F7089581E6ECEFF4E0DF0163
:10A3A0001D928A95E9F78BE08093FC0489E1809304
:10A3B0002A058AE580932B0581E080934005EDEF27
:10A3C000F4E020E032E080E093E021933193958740
:10A3D0008487938F828FB5E0EB30FB07B1F74AE0BB
:10A3E00050E068E673E18DE495E00E94216A0E94E6
:10A3F000BF5190932805809327050895EF920F93FE
:10A400001F93CF93C82F29E233E0E3EDF1E0DF01A2
:10A41000C9011D920197E9F74AE050E06DE573E14B
:10A42000CF010E94216A8C2F90E06AE070E00196D3
:10A430000E94BA69605D6093D801805D8093D90104
:10A4400080E00E940D5E61E06C0F88ECE82E09E26E
:10A4500013E023ED31E042E084E398E00E948D5761
:10A46000CF911F910F91EF9008950F931F93CF936A
:10A47000DF93EB01042F803138F561E0680F84E34E
:10A4800098E00E94C55510E0A80160E270E0CE019E
:10A490000E94426A4AE050E0BE0184E398E00E94D4
:10A4A00049560A9789F484E398E00E94B755C00F93
:10A4B000D11F009749F06AE070E00E94BA69805DA0
:10A4C0008A93862F972FF5CFDF91CF911F910F9110
:10A4D00008958F5F0C946C55FF920F931F93CF9349
:10A4E000DF93CDB7DEB72F970FB6F894DEBF0FBE60
:10A4F000CDBF01E0080F102F1031C8F4FF24F394F2
:10A50000F10E8F2D0E946C5581110FC0602F84E3D6
:10A5100098E00E94C55561E0610F28E532E042E015
:10A520008BE298E00E94315706C01F2DE5CF103115
:10A5300069F780E01AC04FE050E0BE016F5F7F4FC7
:10A5400084E398E00E94E255882351F0482FBE0131
:10A550006F5F7F4F8BE298E00E94AE56A895EBCFDD
:10A560008BE298E00E945C5781E02F960FB6F8943A
:10A57000DEBF0FBECDBFDF91CF911F910F91FF9036
:10A58000089581110C94AF510895EF920F931F938A
:10A59000CF9340913F08442309F47FC0811110C03C
:10A5A000F8948091830C9091840C789420913D08CC
:10A5B00030913E08821B930B8436910508F46DC0E0
:10A5C00080912108811169C0C42FC47042FD02C06E
:10A5D00081E001C083E08093210810923F0840FF92
:10A5E00026C024E1E22E01E610E02CEF34E041E049
:10A5F00061E182E298E00E948D578136910519F45D
:10A6000061E180E029C080912808823051F4809176
:10A610003F0881602BC080912808823001F1C11170
:10A620003AC060E083E793E10E947F1934C041FFA4
:10A6300032C094E1E92E09E213E023ED31E042E07B
:10A6400061E182E298E00E948D578932934019F7C8
:10A650008091290561E18F5F0E947A551CC080912D
:10A660003F08C11102C0826001C0866080933F082C
:10A67000F8948091830C9091840C7894845691097D
:10A6800090933E0880933D088091BF0C833019F46D
:10A69000A8951092BF0C10922108CF911F910F9195
:10A6A000EF90089580913F08882359F081E00E943F
:10A6B000C5528091BF0C8330A9F7A8951092BF0CAA
:10A6C000F1CF0895EF92FF920F931F93CF93DF93F3
:10A6D000C82F803108F07FC061E0680F84E398E004
:10A6E0000E94C55529E233E0E3EDF1E0DF01C90145
:10A6F0001D920197E9F749E253E0BF0184E398E036
:10A700000E9449568F3F910509F018F48C2F0E9442
:10A71000FE5183ED91E00E949E5180917B04811156
:10A7200007C08091E401869583708E5F80937B04DF
:10A730000E9446310E9491128091C304823008F039
:10A740004AC010E0812F0E940A0FEC0189818150DC
:10A75000843018F40E94EF0E89831F5F103291F746
:10A76000C9E2D4E000E010E08A818F700E94FC0E04
:10A77000882381F08230B9F4D801A65DBB4F7D01FA
:10A780008C91882339F085302CF481500E94EF0E93
:10A79000F70180838881882331F0853024F481504B
:10A7A0000E94EF0E888323960D5F1F4F0432110520
:10A7B000D9F660E08BE493E10E947F1982E08093F8
:10A7C000C3040E94AF51DF91CF911F910F91FF9071
:10A7D000EF900C945253DF91CF911F910F91FF9006
:10A7E000EF900895EF920F931F93CF93DF930E9402
:10A7F0005955882399F10E94CF5487FD2FC060E0FE
:10A8000084E398E00E94C55581E6ECEFF4E0DF01B7
:10A810001D928A95E9F741E650E0BF0184E398E094
:10A820000E9449568DE495E00E949E518091FC045F
:10A830008B3058F480917A01816080937A018BE0AB
:10A840008093FC0481E00E94AF51C0912705D09114
:10A8500028050E94BF51C817D90721F161E08BE399
:10A8600093E10E947F1989E293E10E9422110E94E4
:10A8700034550E94CC5138ECE32E01E610E02CEF69
:10A8800034E041E060E084E398E00E948D57813637
:10A89000910529F060E08AE193E10E947F1980E050
:10A8A0000E94FE5180912905DF91CF911F910F9158
:10A8B000EF900C94625340E450E060E070E080E47C
:10A8C00098E00C94285C41E050E062E070E082E4A3
:10A8D00098E00C94285CCF93DF931F92CDB7DEB73E
:10A8E000698390E1899FB001112441E050E0CE01DD
:10A8F00001960E94285C0F90DF91CF910895CF932D
:10A90000DF931F92CDB7DEB790E1899FB00111248C
:10A9100041E050E0CE0101960E94496A89810F9082
:10A92000DF91CF910895CF93DF93D82FC82F8C2F2D
:10A930000E947F54882329F08C2F0E947F54C82FB7
:10A94000F6CF609142088C2F0E946B54D09342083E
:10A95000DF91CF910C946354CF93C0914208CC23E4
:10A9600059F08C2F0E947F54809342080E946354B8
:10A9700060E08C2F0E946B548C2FCF910895CF9361
:10A98000DF9380914208C0E0D0E0882321F02F9629
:10A990000E947F54FACFCE01DF91CF910895DF92CC
:10A9A000EF92FF920F931F93CF93DF9380E8E3ED35
:10A9B000F1E0DF011D928A95E9F7C4E4D8E0F12CBB
:10A9C000B4E1FB1205C08091420802E418E002C025
:10A9D0008E01888190E0E12CDD24D394DF0C009778
:10A9E00001F19C01245031092C37310530F4FC0170
:10A9F000ED52FE4F2081222371F0EE2029F060E01D
:10AA00008E2D0E946B5404C0F80110820E945B548A
:10AA100080E090E0E4CFD082E82E0E947F5490E066
:10AA2000DECFF3942396F5E1FF12CACFC4E0D0E065
:10AA3000FE01ED52FE4F8081811109C060914208F4
:10AA40008C2F0E946B54C09342080E94635421963D
:10AA5000C038D10569F780E0DF91CF911F910F9148
:10AA6000FF90EF90DF900895CF9380E4E0E4F8E06A
:10AA7000DF01982F1D929A95E9F794E09093400892
:10AA80008093410880E18093430884E0C1E0C80FCF
:10AA90006C2F0E946B54CF3711F08C2FF7CF60E0F2
:10AAA0008FE70E946B5484E080934208CF910C940E
:10AAB0005B5440E450E060E070E080E498E00E9485
:10AAC000496A80914008843029F481E090914108DE
:10AAD000903409F080E0089590E0FC01EE0FFF1F34
:10AAE000E80FF91FE05CF74F81E09481911101C0FC
:10AAF00080E00895CF93DF9390E0EC01CC0FDD1F51
:10AB0000C80FD91FC05CD74F8C819D81AE8170E08A
:10AB1000FB01EE0FFF1FE60FF71FE05CF74F2481EC
:10AB2000358146812C833D834E8384839583A68320
:10AB3000DF91CF910C945B54CF9390E09C01220F56
:10AB4000331F280F391FF901E05CF74FC481F90169
:10AB5000EC5BF74F1082118212820E945B54CC236F
:10AB600021F08C2FCF910C949354CF910895FC0138
:10AB7000808190E0FC01EE0FFF1FE80FF91FEB5BF7
:10AB8000F74F918180819F700895CF93DF93FC01EF
:10AB900060831282118270E0CB01880F991F860FAB
:10ABA000971FEC01C05CD74F2C8123831482158240
:10ABB0001682FC01EA5BF74F808182958F70DF91EE
:10ABC000CF910895AF92BF92CF92DF92EF92FF9212
:10ABD0000F931F93CF93DF931F92CDB7DEB78C01F6
:10ABE000FC01808190E0FC01EE0FFF1FE80FF91FD0
:10ABF000EB5BF74F80812181922F9F70F8012181BB
:10AC00003281821B930B7A018417950708F47C012B
:10AC10005B016701C114D10429F1F8018381882304
:10AC200009F164816F5F648370E0F0E18F9F600DD4
:10AC3000711D112441E050E0CE0101960E94496A45
:10AC40008981F50181935F01F80184818F3030F0B3
:10AC5000148283810E947F54F8018383F1E0CF1A2C
:10AC6000D108D8CFF801818192818E0D9F1D8C195A
:10AC70009D09928381838E2D8C190F90DF91CF9146
:10AC80001F910F91FF90EF90DF90CF90BF90AF900A
:10AC900008957F928F929F92AF92BF92CF92DF9250
:10ACA000EF92FF920F931F93CF93DF934C016B01B1
:10ACB0008A01C0E0D0E05C0125E0A20EB11CC01703
:10ACC000D107E8F5F40185818F7781F0F4014581A2
:10ACD000F42FFF777F2E2F2F30E0C8018C1B9D0BA8
:10ACE0008217930760F4702E7C1A09C041E050E08F
:10ACF000B501C4010E94E255813041F320C0E72C28
:10AD0000F12CC6018C0F9D1F47FF06C0A70160E014
:10AD100070E00E94426A0CC0A701BC01C4010E94FD
:10AD2000E255871529F0FE01E80FF11DCF0108C09B
:10AD3000CE0DDF1DF401858187198583C0CFCE013B
:10AD4000DF91CF911F910F91FF90EF90DF90CF9007
:10AD5000BF90AF909F908F907F900895AF92BF92D9
:10AD6000CF92DF92EF92FF920F931F93CF93DF93D7
:10AD7000EC018B01D42E8B81811111C089819A81C4
:10AD8000892B69F4E880F12C0E94AC548B83F70185
:10AD9000EE0FFF1FEE0DFF1DE05CF74F8483CD2CFF
:10ADA0008FE0A82ECC2009F445C02F813885F89477
:10ADB0008091830C9091840C7894281B390B37FF79
:10ADC00002C082E004C08B81811103C081E08E83C8
:10ADD00031C09C819F3078F01C820E947F54811189
:10ADE00006C00E94AC54682F8B810E946B548B81EB
:10ADF0000E947F548B838B81882341F36C819A2D31
:10AE0000961BBC2C9C1508F4B92EEB2CF12C70E091
:10AE100090E1899F600D711D11246F5F7F4FA70125
:10AE2000C8010E94285C0E0D1F1D8C818B0D8C8328
:10AE3000CB18B8CF6D2D70E06C19710929813A815A
:10AE4000260F371F3A8329838D2D8C19DF91CF91DF
:10AE50001F910F91FF90EF90DF90CF90BF90AF9038
:10AE60000895EF92FF920F931F93CF93DF93EC011E
:10AE7000F62EE42E89010E94C5556F2D70E0FB016E
:10AE8000EE0FFF1FE60FF71FEB5BF74F1082E29408
:10AE900030EFE322E182F8944091830C5091840CCE
:10AEA0007894400F511F58874F83DF91CF911F91A6
:10AEB0000F91FF90EF9008951F93CF93DF93EC01D4
:10AEC000888190E0FC01EE0FFF1FE80FF91FEB5B9C
:10AED000F74F898180839A819F708181807F892B40
:10AEE00081838B81882329F00E947F54182F811140
:10AEF0000BC010E00E945B54112359F0812FDF91A9
:10AF0000CF911F910C94935460E08B810E946B54FD
:10AF1000F1CFDF91CF911F9108957F928F929F92F1
:10AF2000AF92BF92CF92DF92EF92FF920F931F9357
:10AF3000CF93DF931F92CDB7DEB76C0159012E2D51
:10AF400030E00E94315719824501E12CF12C772421
:10AF50007394F40181914F019981811108C071109E
:10AF60004EC08081811105C0772473941CC071107C
:10AF70000AC080E09F3718F4E016F10679F57720D3
:10AF800089F0782E01C0712C992341F19068998342
:10AF900041E0BE016F5F7F4FC6010E94AE56813017
:10AFA000E1F027C0782E9923C9F041E0BE016F5F20
:10AFB0007F4FC6010E94AE568130D9F44981B70156
:10AFC000641B71096A0D7B1DC6010E94AE569981F2
:10AFD000891719F0981B99830CC0198289818F5F9A
:10AFE0008983FFEFEF1AFF0A0E151F0508F0B1CF96
:10AFF00008C089818F778701081B110902C0872D3E
:10B00000B9CFC6010E945C57C8010F90DF91CF9164
:10B010001F910F91FF90EF90DF90CF90BF90AF9076
:10B020009F908F907F90089580E094E0E1E8F8E0B1
:10B03000DF019C011D9221503040E1F70895FF92FD
:10B040000F931F93CF93DF93FA0174913196A491DC
:10B05000B0E0179693E0B595A7959A95E1F71A2F6A
:10B06000DA011396FA0132964491249FA00DB11D86
:10B07000112466956695669590E0F0E86F9F800DC7
:10B08000911D112420E030E060E08F57974F472F4B
:10B0900050E0611798F40A2FEC01C20FD31FFD0195
:10B0A000FE2EF01AF71620F4F490F9923196F8CFAC
:10B0B000A40FB51F6F5F20583F4FEBCFDF91CF91AB
:10B0C0001F910F91FF900895CF93DF93382F463152
:10B0D0002CF4842F880F840F880F82C086E0830FA2
:10B0E00020FD08C021FD02C090E005C09091820CB7
:10B0F00096FFFACF91E0669566956695A32FB0E02E
:10B1000050E8659FA00DB11D1124AF57B74F22FF26
:10B1100040C04E3211F08CE0830F24ED240F2F300D
:10B1200010F44B5211C02FEB240F2A3110F441536D
:10B130000BC02FE9240F2A3110F4465305C04F35B8
:10B1400011F44AE201C040E0E4E14E9FA001112465
:10B1500041575C4E6BE062302CF0FA0174913A96E4
:10B16000E49102C070E0E0E04F5F5F4F992311F07F
:10B170007095E0959D012F573F4F21583C4030F48A
:10B180007C93ED01C058DF4FE8831196615018F7AA
:10B1900027C023FF07C0892F81958D9385E0830FFA
:10B1A00031E001C030E025E04202F0011124ED5A07
:10B1B000F74E25E04491332311F0243039F05CE060
:10B1C000A138B50718F4911140954D93215031964F
:10B1D0002111F0CFECE0A138BE0710F491959C93BB
:10B1E000DF91CF91089520E00C946458EF92FF9284
:10B1F0000F931F93CF93DF93F62E122F902F907102
:10B20000E92EEA01112369F0EE2011F0488102C015
:10B21000FE014491202F6F2D0E94645811502196F9
:10B22000F1CFDF91CF911F910F91FF90EF90089593
:10B230000F93FA0194914F5F5F4F929F400D511D04
:10B240001124292F0E94F6580F9108950F9300E0C2
:10B250000E94F6580F910895FF920F931F93CF937A
:10B26000DF93062F122F922F9071F92EFA01FF20F3
:10B2700011F0408101C04491EF012196442331F047
:10B28000212F602F0E946458FE01F1CFDF91CF91F2
:10B290001F910F91FF900895AB0120E0682F80E08F
:10B2A0000C942C5920E00C942C59FF920F931F936F
:10B2B000CF93DF93082FF62EEA0114E1180F1550F3
:10B2C0004C2F4F704A301CF0495C28E002C0405DB2
:10B2D00020E06F2D812F0E94645824E0D695C795F9
:10B2E0002A95E1F71013EBCFDF91CF911F910F91CA
:10B2F000FF900895222321F09091820C96FD0895ED
:10B30000480F669566956695E82FF0E090E8699F8E
:10B31000E00DF11D1124EF57F74F8E1B982F9E0F54
:10B32000941720F4908190959193F8CF0895962FDB
:10B33000969596959695E82FF0E080E8989FE00D19
:10B34000F11D1124EF57F74F8CE0E138F80758F45E
:10B35000677081E090E0062E01C0880F0A94EAF73A
:10B36000908198279083089547FF02C0840F4195EC
:10B37000962F969596959695E82FF0E080E8989F01
:10B38000E00DF11D1124EF57F74F677031E001C058
:10B39000330F6A95EAF74423B1F08CE0E138F807FF
:10B3A00090F4822F90E020FF08C020812327208383
:10B3B00095958795282F206803C095958795282F08
:10B3C00041503196E8CF08952FEF0C94B459962F41
:10B3D000969596959695282F30E0F90180E8989FEC
:10B3E000E00DF11D1124EF57F74F962F940F96950E
:10B3F0009695969580E8989F200D311D11242F5722
:10B40000374F862F8770A1E0B0E001C0AA0F8A9560
:10B41000EAF7A1958081A827A083E217F30750F4EB
:10B42000E058FF4F8CE0E138F807E0F49081909508
:10B430009083F3CF8CE0E138F807A0F4842F9927AC
:10B4400087FD9095860F911D68E070E00E94BA69B3
:10B4500021E030E001C0220F8A95EAF72195808132
:10B460008227808308953F924F925F926F927F92DE
:10B470008F929F92AF92BF92CF92DF92EF92FF9204
:10B480000F931F93CF93DF93182FB62E802F05FFB6
:10B4900004C004FF04C002E003C000E001C001E0FA
:10B4A000982F9F77C92EE7FE04C0E1946624639429
:10B4B00001C0612C57FF0AC05095409530952195E9
:10B4C0003F4F4F4F5F4F7724739401C0712C82FF21
:10B4D00006C09CE09093810CCAE0DC2E05C096E08B
:10B4E0009093810CB5E0DB2E86FF28C071101D0DF6
:10B4F000283E83E038074105510514F01D0D05C0B5
:10B50000243631054105510514F01D0D05C02A30C2
:10B510003105410551050CF01D0D002381F002306D
:10B5200031F424363105410551054CF41D0D2A3006
:10B530003105410551051CF41D0D01C01D198091F7
:10B54000810C810F8093810C023011F490EFC90EB1
:10B5500088248394F2E09F2EA12CFF24E7FCF09432
:10B56000A6E05A2E5B0CE82DF0E0EE16FF060CF478
:10B5700060C06AE070E0C9010E94BA69382EEB0130
:10B58000E0E34E2E480E2C2D442D6B2D812F0E9472
:10B590006458081131C0C2FE1AC08FEF830D83308A
:10B5A00008F49394CE016AE070E00E94BA69823098
:10B5B00011F08430E9F484E3481204C0AA24A3946F
:10B5C000A10E17C0AA24AA94A10E939412C07EEFD4
:10B5D000472E410E8FEF810FC0FE05C047E06B2D57
:10B5E0000E94E75903C0652D0E949759142D01C090
:10B5F000A12E209709F000E09E01442737FD4095D9
:10B60000542F211531054105510581F4002331F0F6
:10B61000023059F491E0981540F008C0C4FE09C00A
:10B62000611004C080EFC80E01C000E01D198394B2
:10B630009ACFAA2061F0492D6CE06B0D8A2D0E94F3
:10B64000E459492D6DE06B0D8A2D0E94E459772055
:10B6500039F02C2D4DE26B2D812F8D190E946458ED
:10B6600080E0DF91CF911F910F91FF90EF90DF90DD
:10B67000CF90BF90AF909F908F907F906F905F9092
:10B680004F903F900895EF920F93022F9A01442715
:10B6900037FD4095542F95E0E92E0E94335A0F91C3
:10B6A000EF90089520E00C94435B0F931F93CF938A
:10B6B000DF93182FC62F042FD22F422F0E94E75955
:10B6C000023038F04D2F6C2F8FEF800F810F0E94CA
:10B6D000E75902501F5F6FEF6C0F6D0F402F812FE6
:10B6E0000E94E459402F6C2F812FDF91CF911F9141
:10B6F0000F910C94E4590F931F93CF93DF93182F5E
:10B70000C62FD22FE42FF0E03297053608F004E67A
:10B710000E9FC0010F9F900D112464E670E00E94FF
:10B72000BA69062F2D2F6C2F812F0E94555B0023A5
:10B7300069F0D150DC0FCF5F1F5FCD1738F4402F79
:10B740006C2F812F0E94E459CF5FF7CFDF91CF910B
:10B750001F910F910895A998AB98AC988BBBAD9AA7
:10B76000AD98AB9AA99A0895CF93DF9381E0809327
:10B770008008AA982AE02A95F1F700C0AA9A8CEDD1
:10B7800095E0E5E0EA95F1F7000001970097C9F729
:10B79000C3E8D3E1FE0184910E94AB5B2196F3E103
:10B7A000CF38DF07B9F789E180932A051092800826
:10B7B000DF91CF910895CF93C82F81E080938008C7
:10B7C00081E80E94AB5B8C2F0E94AB5B10928008DB
:10B7D000CF91089580912A050C94DB5B1F93CF9342
:10B7E000DF9381E08093800810E0C1E8D8E084E036
:10B7F0000E94AB5B80E10E94AB5B812F806B0E945B
:10B80000AB5BA998AB9AAC98FE01CE0180589F4FD4
:10B8100020812BBBAD9AAD9821812BBBAD9AAD9801
:10B8200022812BBBAD9AAD9823812BBBAD9AAD98ED
:10B830003496E817F90761F7EF01AB9AA99A1F5FF1
:10B840001830A9F610928008DF91CF911F910895CA
:10B85000BF92CF92DF92EF92FF920F931F93CF93FD
:10B86000DF937B018A01080F191FEC01E81AF90A1E
:10B870006701CC0EDD1EC017D107C1F0B9908091D1
:10B8800021088270E19B05C08823E1F30E940F1A12
:10B89000F6CFDFBACEBAE09A8DB3B81649F3BDBA87
:10B8A0008FB7F894E29AE19A8FBFE2CFDF91CF9100
:10B8B0001F910F91FF90EF90DF90CF90BF90089570
:10B8C0008091B20C1092B20C0895FC0180818F70AF
:10B8D000880F611181608F709081907F982B908389
:10B8E00081818F5F81838281882351F09F7041F431
:10B8F000833621F0842F80628093B20C11821282F1
:10B900008281883069F148F4813091F188F0823089
:10B9100039F1843009F03FC023C08F35C1F018F4ED
:10B920008031F1F00895813649F0823671F1089541
:10B9300080818F708F3079F581E62BC0406640930F
:10B94000B20C10929306109292068FE522C081816C
:10B95000803211F4406816C08832E9F480E119C0E1
:10B960009181903328F090E095958795828311829C
:10B97000828190E00197218130E082239323892BFB
:10B9800051F440644093B20C08958181803418F0E2
:10B9900088E082831182089540916300282F30E06F
:10B9A0002F3031056CF4F901EE0FFF1FE20FF31F8A
:10B9B000EB57F34F90819F7081E09F3051F52AC083
:10B9C00090E0FC013F97E930F10518F5E659FF4F8B
:10B9D0000C940F6A91B1947019C091B1927016C015
:10B9E000942F10C0942F9095987010C043FF11C0F1
:10B9F00091B102C091B19095907408C091B19071CD
:10BA000005C091B1917002C091B1907281E0911125
:10BA100001C080E008958F7090E08F30910551F063
:10BA2000FC01EE0FFF1FE80FF91FEB57F34F82E603
:10BA30008283118208958F7090E08F30910549F0D4
:10BA4000FC01EE0FFF1FE80FF91FEB57F34F83E6E2
:10BA500082830895EF92FF920F931F93CF93DF930A
:10BA60008091830C9091840C01969093840C809328
:10BA7000830C8093820C96B390958091B30C8823AD
:10BA800021F0282F2877292349F4892F807609F07F
:10BA900050C093FD4AC094FF4AC080E1182F166041
:10BAA00019238093B30CC5E8DCE0F12C11FB662769
:10BAB00060F94F2DCE010E94655CF3941695239694
:10BAC00086E0F812F3CFE0B2E094C3EDDAE100E0F3
:10BAD00010E0FC1AFE0184914C2F4F0D8E2161E085
:10BAE00009F460E0C8018956934F0E94655C219675
:10BAF0000D5F1F4F0831110569F79091B80161E0A2
:10BB0000C92FC07295FF60E04EE08FEA9CE00E9472
:10BB1000655C86B390E0809590958E7799278C2B05
:10BB200051F089E08093540106C088E0B7CF80E0EF
:10BB3000B5CF80E6B3CFDF91CF911F910F91FF90EA
:10BB4000EF90089595E0899FD0011124A754BC4F30
:10BB5000CB010596FB0124912D933196E817F90747
:10BB6000D1F708950F931F93CF93DF93182FCDEE46
:10BB7000D1E090E08881181738F0882329F09032BE
:10BB8000E9F09F5F2A96F6CF9032C1F02FE130E0C6
:10BB9000291B31090AE0029FA001039F500D1124C7
:10BBA000BE01CE010A960E94306AFE0111920A95EA
:10BBB000E9F7188384E68A83CE0102C08DEE91E016
:10BBC000DF91CF911F910F91089580E491E0EDEE08
:10BBD000F1E0DF019C011D9221503040E1F7089512
:10BBE00088E2E9EBF3E0DF011D928A95E9F788E44A
:10BBF000E1EEF3E0DF011D928A95E9F7089590E008
:10BC00000197FC01EE0FFF1FE80FF91FE75DFB4FE7
:10BC10006F7062834083218308958F929F92AF92C9
:10BC2000BF92CF92DF92EF92FF920F931F93CF9329
:10BC3000DF9300D000D0CDB7DEB7182F19821A825B
:10BC40001B821C82E0914505F0E0E056FC4F46E087
:10BC500050E0A1E0E491EE2EF12C21E030E0C701AC
:10BC6000042E02C0959587950A94E2F78370992770
:10BC7000BC016F5F7F4FE1E0F0E0EC0FFD1F8E0F26
:10BC80009F1F6217730711F4FC01A0832F5F3F4FC2
:10BC900025303105B1F7AF5F42505109A530E9F6C3
:10BCA00011111BC00E94E55D89810E94B25D21E0F7
:10BCB000FC0121838A810E94B25D22E0FC01218384
:10BCC0008B810E94B25D23E0FC0121838C810E9464
:10BCD000B25D24E0FC01218399C1113071F48B81A4
:10BCE0000E94B25DFC0188E081838CE9828313832A
:10BCF0008781897F8460878389C11230E9F58B81D0
:10BD00000E94B25DFC0118E011834CE9F42EF2822E
:10BD100085E183838781897F846087838EE00E94A9
:10BD2000B25D02E2FC0101838EE00E94B25DFC0183
:10BD30001183F28284E183838781897F8460878392
:10BD40008EE00E94B25DFC01118381E083838781D4
:10BD5000897F8460878382E08093490483E08093B5
:10BD600047048DE98093480481E080934C0400935C
:10BD70004A0410924B044AC11330F1F40E94E55D6D
:10BD80001981812F0E94B25DFF24F394FC01F1829E
:10BD9000812F0E94B25D12E0FC0111832CE9228305
:10BDA0000A81802F0E94B25DFC01F182802F0E94E7
:10BDB000B25DFC0111832AC11430E9F40E94E55DF3
:10BDC0000A81802F0E94B25D32E0F32EFC01F182E5
:10BDD000802F0E94B25DFC0111830C81802F0E9494
:10BDE000B25DFC01F182802F0E94B25DFC011183E3
:10BDF0002CE922830BC1153009F0A8C00E94E55D33
:10BE00000E94F05D81E00E94B25D5AE0C52EFC0107
:10BE1000C18282E00E94B25D6BE0D62EFC01D1822D
:10BE200083E00E94B25D7CE0F72EFC01F18284E0A9
:10BE30000E94B25DAA24A394FC01A18285E00E9425
:10BE4000B25DFC0103E00183A4E0BA2EB38287E077
:10BE5000848387818160878385E00E94B25DFC01D5
:10BE600001831383B8E08B2E84828781816087836E
:10BE700085E00E94B25DFC01018386E0E82EE3824A
:10BE800099E0992E948287818160878385E00E9462
:10BE9000B25DFC0181828CE98283A3828781897FE4
:10BEA0008460878386E00E94B25DFC0191828EE10E
:10BEB000828388EF83838BE00E94B25DFC01018363
:10BEC00026E4A22EA282B382C48287818160878306
:10BED0008BE00E94B25DFC010183A2821383D482B5
:10BEE0008781816087838BE00E94B25DFC010183C2
:10BEF000A282E382F4828781816087838091E90155
:10BF00008F7180628093E9018FE18093EA016FEE87
:10BF10007AE180E00E94A25D6AEE7AE181E00E940F
:10BF2000A25D65EE7AE182E00E94A25D60EE7AE1B8
:10BF300083E00E94A25D6BED7AE184E00E94A25D45
:10BF40006BED7AE185E00E94A25D60C01630B1F42D
:10BF500086E00E94B25DFC01118382E3828388EF58
:10BF6000838304E6008786E00E94B25DFC011183B2
:10BF70008EEC828388E08383008748C0173009F005
:10BF800045C08FE00E94B25D14E2FC01118328E8F5
:10BF9000268380E10E94B25DFC0189E081830EE688
:10BFA00002838AE0838380E10E94B25DFC0148E065
:10BFB000F42EF18282E982838BE083838781897FFB
:10BFC0008460878380E10E94B25DFC01F18202837C
:10BFD0008CE083838781897F846087838BE0809373
:10BFE0002B0483E28093290410932A0491E0909318
:10BFF0002E0480932C0499E690932D0492E0909364
:10C00000310480932F0487E98093300482E00E94FA
:10C01000C1520F900F900F900F90DF91CF911F9111
:10C020000F91FF90EF90DF90CF90BF90AF909F90D7
:10C030008F900C9452530F931F93CF93DF93909153
:10C04000E90191FF03C060E075E002C060E074E0C8
:10C050001091E401129516951770882331F0A8E02D
:10C06000BDE0833021F420E103C0A0ECBCE028E077
:10C070009091E301990F910F920F4091E60124E610
:10C080004202A0011124485A5D4F0091EC01E8EEF4
:10C09000F3E09F010203E001039FD00D11249E01F4
:10C0A00028533045241B350BFD01882339F0329687
:10C0B0004D935C93833011F418EF190FCC27DD27D3
:10C0C000C61BD70B1917F0F4A12FB0E0AA0FBB1FA6
:10C0D000A55AB84F0D90BC91A02D6A177B070CF4A0
:10C0E000DB01AC17BD070CF4DE01A854B44F2A1BCA
:10C0F0003B0BA41BB50BB183A083538342831F5F0B
:10C100003496E0CF283293E2390710F428E233E284
:10C1100031832083DF01882371F01296285E33403B
:10C120003093BC0C2093BB0C1D921C92DF91CF91DD
:10C130001F910F910895149653834283F5CF1F9357
:10C14000CF93DF93182F20EC3CE030932501209310
:10C150002401C09112018C2F877461F08091E3015A
:10C16000882321F0813021F4C0E906C0C0E804C072
:10C17000C8E902C0C7FF06C087E10E94CC5C8823E3
:10C1800009F471C0C7FD71C040E060E085E10E9424
:10C190004A15882309F469C0C062C09312018091D6
:10C1A00029058F5F80931301E5E1F1E0ABE5B7E08E
:10C1B00090E06DE0911729F14D915D91649F9001A0
:10C1C000659F300D112485E0359527958A95E1F717
:10C1D0003E5F37FD06C02F3F83E038072CF4822FE7
:10C1E00005C080E030E002C08FEF33E0EF0121971F
:10C1F000292F220F220F232B288380839F5F3296C3
:10C20000D9CFA2E1B1E09D91E0912401F091250107
:10C2100029E080E130E0492F4170341302C0805F93
:10C2200004C081508083319680E1969590682150BA
:10C2300011F0342FF0CF815FEF018993D093250166
:10C24000C093240181E0A032B807E9F611828FEF94
:10C25000808380EC9CE09093230180932201DF9106
:10C26000CF911F910895CF778DCFCF7D96CF1F921D
:10C270000F920FB60F9211242F938F939F93EF93EA
:10C28000FF9388B391E0892788BBE0912201F09168
:10C2900023012191F0932301E0932201822F90E06A
:10C2A00097BD86BD293C08F0C09A8091BF0C816083
:10C2B0008093BF0CFF91EF919F918F912F910F90E1
:10C2C0000FBE0F901F9018951F920F920FB60F92EE
:10C2D00011242F933F938F939F93EF93FF9388B3F2
:10C2E00091E0892788BBE0912401F09125018081AC
:10C2F00028B539B580FD03C0205E3F4F02C0205FE6
:10C300003F4F39BD28BD90E095958795009769F41A
:10C31000CF010196909325018093240181818111A1
:10C3200005C087B7877F87BF01C080838091BF0C1E
:10C3300081608093BF0CFF91EF919F918F913F910E
:10C340002F910F900FBE0F901F901895EDE7F0E022
:10C350008081857E808317981F9AAAE8B0E01C929E
:10C3600010928B0082E88C93808180628083089594
:10C37000EDE7F0E080818F7D8083179AAAE8B0E036
:10C380001C9210928B008AE08C938081886180835C
:10C3900008951F920F920FB60F9211248F939F93BF
:10C3A000EF93FF938091500D882321F01F9A1092F4
:10C3B000500D04C01F9881E08093500DE091100152
:10C3C000F091110180819181909387008093860084
:10C3D0008091BB0C9091BC0C90938500809384005D
:10C3E00082819381892B11F0329607C08091E901F7
:10C3F00081708093500DE8E0FDE0F0931101E0932F
:10C4000010018091BF0C81608093BF0CFF91EF9170
:10C410009F918F910F900FBE0F901F901895E4EB96
:10C42000FCE0208126952695282B208381818F5F33
:10C430008183843048F0A281B381CD01019693833A
:10C4400082832C93108211820895882339F0809181
:10C45000BA0C8F5F8093BA0C80E803C01092BA0CBC
:10C4600080EC0E940F628091BA0C8530B8F7089575
:10C47000CF93DF93C82FE091B90CE827F0E0EE0FDF
:10C48000FF1FE85AF44E259134915091B80C40E0CA
:10C49000242735273093B90C2093B80CD8E08C2F83
:10C4A00080780E942562CC0FD150C9F7DF91CF91DF
:10C4B0000895CF9380EC0E940F62C6E080E80E944E
:10C4C0000F62C150D9F780ECCF910C940F6280318C
:10C4D000E0F4E82FF0E0EE0FFF1FE55AF84F20815F
:10C4E0003181C901880F991F820F931F97FD039611
:10C4F00095958795959587959C5F1816190644F430
:10C500008E3F27E092073CF4089580E094E0089580
:10C5100081E090E008958EEF97E00895CF92DF924A
:10C52000EF92FF920F931F93CF93DF93C091E2019D
:10C53000CF708091480585FF04C08091CF018111A3
:10C54000C4E08091BE0C8C1709F47EC0C093BE0C71
:10C550001EBC1DBC1CBC87B7837C87BF80917D003F
:10C560008E7F80937D008CE386BF8FE380937C0079
:10C57000C23061F118F4C13089F003C0C53008F44D
:10C5800041C00E94A66180E49CE99BBD8ABD87B73B
:10C59000806187BF1FBC8AE08EBD56C00E94A66125
:10C5A00088E59BE199BD88BD80EA9FE09093790082
:10C5B0008093780087B7886087BF80917D00816015
:10C5C00080937D001FBC82E08EBD49C00E94A661A1
:10C5D00088EC90E090937900809378008CE291E071
:10C5E0009DBD8CBD80EE9BEA97BD86BD87B78062FE
:10C5F00087BF80917D00816080937D001FBC8AE1B0
:10C600008EBDD5C0C43029F484E00E941B60C09860
:10C610000DC080E49CE99BBD8ABD87B7806187BF60
:10C620001FBC8AE08EBD83E00E941B6080E593EC16
:10C63000909387008093860088E893E1909385002B
:10C64000809384000E94B861C13049F008F4BBC0F7
:10C65000C23009F4ACC0C33009F4B5C0BFC078948F
:10C66000F090520D87B7877F87BF80917D008E7FC6
:10C6700080937D00E4EBFCE080EC9CE0909325014E
:10C680008093240181EC9CE0938382831582148241
:10C690001082118216828FEF8093C00C0E94596223
:10C6A0008091E3010E9438629091BD0C8091E2017B
:10C6B00090FF08C0282F207C8695869586958670E9
:10C6C000822B01C0807C892B0E94386280E00E940E
:10C6D0003862E090E401E294E694F7E0EF228F2DD7
:10C6E0008170D82EF0FE02C088E0E80EE8E0CE2E81
:10C6F000CE0C8E2D0E9467628C01D110185F802FA6
:10C700000E94386281E08E0D0E946762EC01D110B8
:10C71000D85FE394E3949C2F9295907F812F8F7044
:10C72000892B0E943862CE0174E0969587957A95A0
:10C73000E1F70E943862EC10DCCF80E00E943862A2
:10C74000C091B80C8091B90C0E9438628C2F0E9465
:10C7500038620E9459628091B50C882321F080E0F4
:10C760000E940F62F8CFE091B60CF091B70C1082E6
:10C77000E8E7F0E0808191819C012854344F39BD75
:10C7800028BD805B994B91838083C09A88E086BFE7
:10C7900081E080937C0087B7886087BF80917D00AF
:10C7A000816080937D00F394F092520D17C07894CD
:10C7B00086E0DF91CF911F910F91FF90EF90DF9076
:10C7C000CF900C949F6080E0DF91CF911F910F91EB
:10C7D000FF90EF90DF90CF900C941B60DF91CF9192
:10C7E0001F910F91FF90EF90DF90CF9008951F92CF
:10C7F0000F920FB60F9211242F933F934F935F9395
:10C800006F937F938F939F93AF93BF93CF93DF9358
:10C81000EF93FF938CB59DB52091510D222321F00C
:10C82000C09A1092510D04C0C09821E02093510D80
:10C83000C0912001D0912101FE01219131913BBD98
:10C840002ABDF0932101E0932001EEE0F1E0282FD2
:10C850003181381708F481833081231708F48083ED
:10C860008A819B81892BD9F480EC9CE090932101F3
:10C87000809320018091E901809581708093510D12
:10C8800087B78F7E87BF0E948E628091E2018F7092
:10C8900011F0833021F487B7806187BF789480914D
:10C8A000BF0C81608093BF0CFF91EF91DF91CF911E
:10C8B000BF91AF919F918F917F916F915F914F91B8
:10C8C0003F912F910F900FBE0F901F901895809160
:10C8D000E2018F70865F8093BE0C0C948E621F9273
:10C8E0000F920FB60F9211242F933F934F935F93A4
:10C8F0006F937F938F939F93AF93BF93EF93FF9328
:10C900008091E2018F708230C1F480E492EA97BD99
:10C9100086BD80917800909179008F3F910538F421
:10C9200088E598E9909379008093780008C088ECB6
:10C9300090E090937900809378000E948E62FF913E
:10C94000EF91BF91AF919F918F917F916F915F9187
:10C950004F913F912F910F900FBE0F901F90189500
:10C960001F920F920FB60F9211242F933F934F9364
:10C970005F936F937F938F939F93AF93BF93EF9347
:10C98000FF938091E2018F7078949091BE0C98177C
:10C9900071F0943061F48091CF01882321F080916F
:10C9A000480585FD03C00E948E6203C084E00E949A
:10C9B0001B60FF91EF91BF91AF919F918F917F91FC
:10C9C0006F915F914F913F912F910F900FBE0F90FC
:10C9D0001F901895FC01A5E6B0E08C918B7F8C939D
:10C9E000148215821082118216A617A608950C943F
:10C9F000EA6421E0FC018481811101C020E0822FE2
:10CA00000895FC0121818081281B277098E0921BEA
:10CA100081E0933008F480E00895CF93DF93FC0128
:10CA200084818823F1F08150848382819381890FEE
:10CA3000828386A58823F1F187A59FEF980F97A79A
:10CA4000882331F08091650084608093650032C056
:10CA5000809165008B7F8093650080914A0587A750
:10CA600029C01B98809165008B7F8093650085812C
:10CA7000882319F0815085831DC080819181891799
:10CA8000C9F090E0EF01C80FD91F2E8122832E89B3
:10CA900024832E8523832E8D258328A926A717A6D8
:10CAA0002EA13FEF320F3EA3211104C001968770E3
:10CAB00099278083DF91CF910895EF92FF920F9392
:10CAC0001F93CF93DF93EC01F62E142FE22E0E94DA
:10CAD0000165882309F44FC080913F05887309F4EC
:10CAE0004AC0302F3295369536953370402F4F70AF
:10CAF000333009F43FEFFF2021F090914905965F14
:10CB0000F90E803129F48BEA189F112D112402C0EF
:10CB1000883111F4169509C0883211F4110F05C03F
:10CB2000803319F4812F880F180F288104FF0DC05E
:10CB3000FA821C83ED8205FB882780F98EA71FA649
:10CB40003B8329834423B9F001C04F5FE981F0E0C2
:10CB5000CF01019687709927281769F0EC0FFD1F08
:10CB6000F682168BE68E05FB002700F900AB4150DC
:10CB700046A336878983DF91CF911F910F91FF9054
:10CB8000EF9008950F931F93CF93DF93EC01062F3F
:10CB9000642F80913F0586958695869587703881AC
:10CBA0002981321300C110E00332110508F0FBC0E7
:10CBB000F801ED58FF4F0C940F6A00E32AC000E320
:10CBC00021E0CFC002EA22E04AE064E6E9C00AE2DE
:10CBD00022E045E06FE5CE010E945D6501E22AE0BA
:10CBE00045E06FE5CE010E945D650AE222E045E086
:10CBF0006FE5D6C002EC23E04AE060E5CE010E947A
:10CC00005D6502E423E04AE06CE3CE010E945D65CD
:10CC100000E221E06FC001E221E045E066E4CE01E0
:10CC20000E945D6522E04FE062E3CE010E945D65F7
:10CC300022E04FE06BC002E221E045E06EE6CE016B
:10CC40000E945D6503E221E045E09FC000E025E031
:10CC500045E062E3CE010E945D6525E045E06AE5BE
:10CC6000CE010E945D6502E024E043E06EE698C0DC
:10CC700003E22AE045E060E5CE010E945D6501E245
:10CC800024E145E060E5CE010E945D6503E22AE013
:10CC900045E03CC002E625E044E16AE081C002E2F2
:10CCA0002AE044E062E3CE010E945D6501E224E1F6
:10CCB00048E066E4CE010E945D6502E22AE048E0B9
:10CCC00062E3CE010E945D6501E224E144E04EC0D2
:10CCD0000AE22AE002C002E222E345E04CC001E29F
:10CCE00003C002E201C003E22AE044E160E058C070
:10CCF00002E122E04AE03AC002E423E044E16CE3CE
:10CD0000CE010E945D6502EE23E044E160E548C08B
:10CD100000E321E048E22AC0813009F444C000E188
:10CD200021E04AE06BE43CC08130E9F100E121E020
:10CD30004AE061E435C000E121E046E031C000E3B3
:10CD4000D8CF813081F100E1D4CF00E112C003E3FC
:10CD500003C002E301C001E323E04FE00CC001E3A4
:10CD600029E144E103C000E321E04EE166E418C09C
:10CD700001E321E04AE068E713C002E321E04AE072
:10CD80006AE70EC003E321E04AE06CE709C000E572
:10CD900020E04AE062E804C000ED20E04AE062E3FF
:10CDA000CE010E945D65DF91CF911F910F91089593
:10CDB00046E4682F8BE791E00C94C26590914B0597
:10CDC00091FF03C0862F0C94B3120C94D866CF92B7
:10CDD000DF92EF92FF920F931F93CF93DF93EC01BB
:10CDE000062F142F47FF03C0842F0E94B312D7FFD2
:10CDF00006C0D195C195D1098AE10E94B3120023E2
:10CE000071F0023019F464E670E002C06AE070E08C
:10CE1000CE010E94BA69262FC22FD72FF82E64E6C2
:10CE200070E0CE010E94BA699B01FB01EC01611523
:10CE30007105A1F16A307105CCF06AE070E0C901BA
:10CE40000E94BA696B017C01653171051CF48EE6A4
:10CE50008C0D05C08CE88C0D0E94AE128EE60E94EF
:10CE6000B312F701309769F001E001C000E084E6F9
:10CE70008E0F0E94B312011104C0209751F18C2F24
:10CE80000BC0209731F1CE016AE070E00E94BA69D0
:10CE90009E01281B390BC901845714C084570E9476
:10CEA000AE120023B1F0023081F46AE070E08F2D01
:10CEB00090E00E94BA69C82F86E0860F0E94B312E4
:10CEC0008CE88C0F0E94AE1204C086E08F0D0E9489
:10CED000B31211165CF4812FDF91CF911F910F9146
:10CEE000FF90EF90DF90CF900C94B312DF91CF9131
:10CEF0001F910F91FF90EF90DF90CF90089586B330
:10CF000080958E7708958FEF8ABB1BBA91E897BB07
:10CF10009EE798BB9EE394BB91EC95BB11BA82BB94
:10CF200088E082B987EF83B91092610010926200A5
:10CF300084E1809364008BEF80936500D4B714BEC6
:10CF40000E94B45B80E487B985E886B987E083BF37
:10CF50008CE981BF82E085BD87B7836487BF1FBC32
:10CF60008AE08EBD10928B0082E880938A008091C7
:10CF70007D00806280937D00789484EE9BE39093A3
:10CF80004B0180934A0189E10E94DB5B0E94F253CE
:10CF9000D09029050E947F67C0E081FD05C086957D
:10CFA000CF5FC730D1F71FC0C630E9F08C2F0E9489
:10CFB00069528823C1F0C09329058C2F0E946253C7
:10CFC00081E00E94C1520E94145824E04DEA51E0D1
:10CFD00060E086E10E942C5988E10E94EA100E94DC
:10CFE000EE5B0E94A7100E94EA5B81E0809338010B
:10CFF0000E946B161092380180915805895F0E943B
:10D00000B612D3FD1AC18091420584FF05C08091FC
:10D010003F0582FD4FC044C080914B05882321F01D
:10D020006CE187E00E94DE660E944A160E94145856
:10D0300020E04FEB53E060E080E00E941F588091B9
:10D04000480584FD08C000E12AE04DE455E068E3AE
:10D0500080E00E94F6580E94EE5B0E94EA5B0E940C
:10D06000A7100E94D70E0E94A2138C01F894C091C1
:10D07000830CD091840C7894C057DE4F0E94EE5BF5
:10D080000E944A160E94D70E0E94A2137C010E94A1
:10D090007F678111BCCFE016F10609F4F5C0B7CF68
:10D0A0000E94BF54883C910528F460E08EE991E02D
:10D0B0000E947F190E94D70E809175059091760588
:10D0C0006EE070E00E94A66960933C0180913F058C
:10D0D00080FD3DC080914005817012E0181B0E94C8
:10D0E000D70EE12FF0E0EE0FFF1FE450FB4F218140
:10D0F00032818091420580FF06C03195219531092A
:10D10000458D568D02C047855089241B350BE9019A
:10D110006096812F0E94BC13C817D907C4F46FE82A
:10D1200071E08DE791E00E94AE100E94EE5B0E94DC
:10D13000A7100E94D70E0E944A16812F0E94BC138E
:10D14000C817D90724F40E947F67882391F3C09100
:10D15000570580913F0581FD53C08C2F887388301F
:10D1600041F0803131F0803221F0C77CC860C0933B
:10D17000570501E00E94DA10182FD82FDC2767E648
:10D1800071E08BE093E10E94AE10D0FF04C060E03C
:10D1900082E00E94D010D1FF04C061E087E10E94CC
:10D1A000D010D2FF04C062E08CE20E94D0108D2F1C
:10D1B000887371F013FF02C063E007C014FF02C060
:10D1C00064E003C015FF04C065E081E40E94D01054
:10D1D000D6FF04C066E086E50E94D010D7FF04C0E9
:10D1E00067E08BE60E94D0100E94EE5B01110E9466
:10D1F000A7101C1729F00E947F67882309F44FC0ED
:10D2000080913F05887B29F460E087E591E00E94EA
:10D210007F1980917A01882351F060E08CE291E0DF
:10D220000E947F1980917A018E7F80937A010E94FB
:10D23000A7108091DD010E94AE1260E08BE597E0BF
:10D240000E9464330E9467642DE088E190E00FB68D
:10D25000F894A89581BD0FBE21BD83E19DE2909316
:10D260004D0180934C010E94EA5B80912905D816FC
:10D2700029F081E00E94C1520E94525381E08093C4
:10D28000D0010E940F1AFDCFF8948091830C9091E9
:10D29000840C7894C817D90709F0F0CEB8CE0E9454
:10D2A0004A1600E067CF8BE791E00C94F7640E9488
:10D2B0005F69332312F48A1B9B0B0C947069A29F45
:10D2C000B001B39FC001A39F700D811D1124911D5A
:10D2D000B29F700D811D1124911D08950E945F69F8
:10D2E000B7FF0895821B930B08950E945F69A59F65
:10D2F000900DB49F900DA49F800D911D1124089551
:10D30000B7FF0C9475690E947569821B930B089591
:10D31000DB018F939F930E947569BF91AF91A29F8C
:10D32000800D911DA39F900DB29F900D1124089523
:10D3300087FB082E062687FD819567FD61950E9473
:10D34000156A0EF4919507FC81950895AA1BBB1BE5
:10D3500051E107C0AA1FBB1FA617B70710F0A61BF5
:10D36000B70B881F991F5A95A9F780959095BC0116
:10D37000CD01089597FB072E16F4009407D077FD92
:10D3800009D00E94A66907FC05D03EF490958195CE
:10D390009F4F0895709561957F4F0895A1E21A2ED1
:10D3A000AA1BBB1BFD010DC0AA1FBB1FEE1FFF1F49
:10D3B000A217B307E407F50720F0A21BB30BE40B99
:10D3C000F50B661F771F881F991F1A9469F76095E0
:10D3D0007095809590959B01AC01BD01CF0108959A
:10D3E000052E97FB1EF400940E94076A57FD07D094
:10D3F0000E94CE6907FC03D04EF40C94076A509546
:10D400004095309521953F4F4F4F5F4F0895909530
:10D410008095709561957F4F8F4F9F4F0895EE0FC8
:10D42000FF1F0590F491E02D0994991B79E004C049
:10D43000991F961708F0961B881F7A95C9F7809553
:10D440000895FB01DC014150504048F005900D92D9
:10D450000020C9F701C01D9241505040E0F70895E7
:10D460006817790768F4FB01DC01E40FF51FA40FCE
:10D47000B51F02C002900E9241505040D8F7089557
:10D480000C94596ADC0101C06D9341505040E0F7A3
:10D490000895DC01CB01FC01E199FECF06C0FFBB82
:10D4A000EEBBE09A31960DB20D9241505040B8F764
:10D4B0000895FB01DC0102C001900D9241505040E3
:08D4C000D8F70895F894FFCF9E
:10D4C800F000B503B603B703B80364000A02FF000F
:10D4D800080DFF0000AA05FF09FF0DFF135414AA49
:06D4E800C00CC00CC00CDA
:00000001FF
